:100000000C94D5280C9406290C9406290C940629E6
:100010000C9406290C9406290C9406290C940629A4
:100020000C9406290C9406290C9406290C94062994
:100030000C9406290C9406290C9406290C94062984
:100040000C9406290C94FBC40C9406290C940629E4
:100050000C9406290C9406290C943EBD0D945F2641
:100060000C9406290C94168E0C94E08D0C940629A1
:100070000C9406290C9406290C9406290C94062944
:100080000C9406290C9406290C9406290C94062934
:100090000C9406290C9406290C9406290C94062924
:1000A0000C9406290C9406290C9406290C94062914
:1000B0000C9406290C9406290C9406290C94062904
:1000C0000C9406290C9406290C9406290C940629F4
:1000D0000C9406290C9406290C9406290C940629E4
:1000E0000C940629084AD73B3BCE016E84BCBFFD69
:1000F000C12F3D6C74319ABD56833DDA3D00C77FF8
:1001000011BED9E4BB4C3E916BAAAABE0000008090
:100110003F05A84CCDB2D44EB93836A9020C50B91F
:10012000918688083CA6AAAA2ABE000000803F004B
:100130000D9499220C94ED540C9491A80D94A22244
:100140000D9457240C94F4600C9451AF0C947E6180
:100150000C9479290D94D4230D9443240C9496A8DF
:100160000C948DB20C94EA2E0C9443AA0C947C61EE
:100170000D942F240D94C2220C94B1380C94C954C0
:100180000C94B7540C94B72B0C94852D0D948722A6
:100190000C94872D0C9415290C9489340D940C24FF
:1001A0000C94A4AD0C9444670C945BAF0C94E42DB8
:1001B0000C94BAAA0C94EFAC0C94998E0C94E15464
:1001C0000C94D7AB0C947C8E0C9469E80C9445612C
:1001D0000C948A8E0C9495B20D9439240C9455AAE3
:1001E0000C944FAA0C945AE80D94C7230C94D32A6C
:1001F0000C94A5B20C9456AF0C9408290C945BAAED
:100200000C9404B00C9432FD0C9472E80C94CDB2B2
:100210000D94A6220C94E6AF0C94B62B0C9449B125
:100220000C9481410C94E7540C94C7AF0C940337A1
:100230000C94C5B20C94BD540C9431FD0C94ADBB20
:100240000C9463E40D94C7220D94DE230C94CF54D8
:100250000C9420610C944F290C94B5290C94813E88
:100260000C9434FD0D9495220C94AF8E0C94B154E3
:100270000C94BDB20C9466E80C9436B10C9449AA67
:100280000D94AC220C94518E0C944B2D0C94ECE6F6
:100290000C949D8E0C94A1610C946FE80C943A76AA
:1002A0000C94422D0C94B6E60D949C220C94A18ED5
:1002B0000C94492D0D9491220C940EB00D9416249B
:1002C0000C9414AA0D94B4220C947FE80C94044866
:1002D0000C9439290C94D5540C9447610C94252D19
:1002E0000C9431B10C948D290C940D430D94FA2388
:1002F0000C9485B20D94CF230D9402240C9480614C
:100300000C941B2E0C94928E0D94BA220C9428E21D
:100310000C94D62A0D94BE220C94EE2D0D94C82276
:100320000C94C12E0D948D220C94F3540C943BB17B
:100330000D9420240C946CE80C94A42D0C94B935E5
:100340000C94A2310C9452B10C94DA2D0C949DB201
:100350000C943C2E0D9461240C94B5B20D94B022F3
:100360000C94A1290D94DB3B0C9478E80D944D245A
:100370000C9449610C9465290C942E760C9451527E
:100380000C94AFA80C94DD290C94DEFD0C94704EF7
:100390000C94C9290C947D3A0C9485E80C94226144
:1003A0000C94F7A90C94A58E0C94A3610C9463E8AB
:1003B0000C94EB290C94DB540C94FC2C0C9482E8E8
:1003C0000C94A5610C94C7510C94C3540C94FFAFCA
:1003D0000D94E8230C9422AA0C94784A0D94C1330E
:1003E0000C94682D0C94582E0C942CB10D94CC22A6
:1003F0000C94A98E0C9475E80C9439400D94F2235A
:100400000C947DE80C94ADB20C9409B04E414E4969
:100410004E495459494E46CDCCCC3D0AD7233C17C2
:10042000B7D13877CC2B329595E6241FB14F0A000F
:100430000020410000C84200401C4620BCBE4CCAFF
:100440001B0E5AAEC59D74434F4D4D554E49434109
:1004500054494F4E0044525952554E004552524F46
:10046000525300494E464F004543484F0045727273
:100470006F722077726974696E6720746F204545CA
:1004800050524F4D210A00627573793A20706175A0
:1004900073656420666F7220696E7075740A0062FD
:1004A0007573793A2070617573656420666F722088
:1004B000757365720A00627573793A2070726F63A2
:1004C000657373696E670A004B494C4C2063617514
:1004D00073656420627920746F6F206D7563682086
:1004E000696E6163746976652074696D65202D207D
:1004F00063757272656E7420636F6D6D616E643AC0
:100500002000506C656173652072657365740050DE
:1005100052494E5445522048414C54454400706F56
:100520007765726F6666004B494C4C45442E20003F
:100530005072696E7465722068616C7465642E20F7
:100540006B696C6C28292063616C6C6564210A00FE
:100550006563686F3A004572726F723A00486F7453
:10056000656E6420746F6F20636F6C640A00507254
:1005700065737320627574746F6E20286F72204DDE
:100580003130382920746F20726573756D650A00EB
:10059000496E736572742066696C616D656E742056
:1005A000616E6420707265737320627574746F6E0F
:1005B00020286F72204D313038290A00507265733F
:1005C0007320627574746F6E20286F72204D313005
:1005D000382920746F2068656174206E6F7A7A6C98
:1005E000650A00706175736564004D3630303A20DD
:1005F000546F6F20636F6C6400486F74656E642085
:10060000746F6F20636F6C640A00726573756D653B
:100610006400496E736572742066696C616D656E05
:100620007420616E642070726573732062757474D7
:100630006F6E20286F72204D313038290A000A0A67
:10064000426564204C6576656C20436F7272656309
:1006500074696F6E204D61747269783A00202B00C6
:100660000A436F7272656374656420426564204852
:1006700065696768742076732E2042656420546F24
:10068000706F6C6F67793A0A00202B000A4265642C
:100690002048656967687420546F706F6772617075
:1006A00068793A0A2020202B2D2D2D204241434BE2
:1006B000202D2D2B0A2020207C20202020202020CF
:1006C000202020207C0A204C207C20202020282B49
:1006D00029202020207C20520A2045207C20202018
:1006E00020202020202020207C20490A2046207C19
:1006F00020282D29204E20282B29207C20470A2025
:1007000054207C20202020202020202020207C20FD
:10071000480A2020207C20202020282D292020204D
:10072000207C20540A2020207C20202020202020F3
:10073000202020207C0A2020204F2D2D2046524FA3
:100740004E54202D2D2B0A2028302C30290A00341D
:1007500074682070726F626520706F696E742C20EF
:1007600064697374616E63652066726F6D20706C6E
:10077000616E653A2000202844525952554E290096
:10078000473239204175746F20426564204C65768C
:10079000656C696E67003F20284C2C522C462C4219
:1007A00029206F7574206F6620626F756E64732EDA
:1007B0000A003F50726F626520706F696E7473201B
:1007C00028592920697320696D706C61757369629D
:1007D0006C652028322D32292E0A003F50726F623C
:1007E0006520706F696E7473202858292069732002
:1007F000696D706C61757369626C652028322D3289
:10080000292E0A003F2856296572626F7365206C95
:100810006576656C20697320696D706C61757369AC
:10082000626C652028302D34292E0A002020536D5B
:100830006F6F7468696E6720286D6D293A202020DB
:100840002020202020202020202020202020530095
:1008500020204261636B6C6173682044697374612A
:100860006E636520286D6D293A20202020202020ED
:100870002000202846312E30203D2066756C6C2CDF
:100880002046302E30203D206E6F6E65290A0020F4
:1008900020436F7272656374696F6E20416D6F756E
:1008A0006E742F466164652D6F75743A2020202088
:1008B0002046006163746976653A0A00696E0042F9
:1008C00061636B6C61736820436F727265637469F6
:1008D0006F6E2000000020002300260029002C005D
:1008E0002F003200000100000301060109014D61E3
:1008F00063726F20746F6F206C6F6E672E0A0047F3
:1009000032380020496E76616C69642065787472B3
:1009100075646572200020746F6F206C6F6E6720A5
:10092000657874727573696F6E2070726576656E26
:100930007465640A0020636F6C6420657874727556
:1009400073696F6E2070726576656E7465640A00F7
:10095000536C6565702E2E2E004D31313720486F57
:100960007420456E642048656174696E672E2E2E72
:100970000A4D31303420533137302054300A473259
:1009800038204F310A473120593235205A31302032
:1009900046353030300A4D31313720526577697035
:1009A000696E67206E6F7A7A6C650A54300A473137
:1009B00020582D3137205932352046353030300A15
:1009C0004D31303920523137302054300A473120F0
:1009D0005A310A473120582D3137205932352046B7
:1009E000343030300A473120582D313720593935CD
:1009F0002046343030300A473120582D31372059C5
:100A000032352046343030300A473120582D3137C6
:100A1000205939352046343030300A473120582D9E
:100A20003137205932352046343030300A473120B2
:100A3000582D3137205939352046343030300A4767
:100A40003120582D3137205932352046343030305E
:100A50000A473120582D3137205939352046343056
:100A600030300A473120582D313720593235204651
:100A7000343030300A473120582D3137205939353C
:100A80002046343030300A473120582D3137205934
:100A900032352046343030300A473120582D313736
:100AA000205939352046343030300A4731205A3108
:100AB000350A4D3130362053323535200A47302043
:100AC00058302059300A4D313039205231363020DB
:100AD00054300A4D3130370A004D31303420533113
:100AE00037302054300A4D313137204C6576656CF3
:100AF000696E67205820417869730A473020583161
:100B000035302046393939390A473238205A300AC7
:100B10004D313137204C6576656C696E6720646FA6
:100B20006E652E0A4731320A4D3130392052313646
:100B3000300A4D3131372050726F62696E67206222
:100B400065640070726F62655F72657769706500D9
:100B50004175746F6C6576656C206661696C65645F
:100B6000004D31313720426564206C6576656C69D3
:100B70006E67206661696C65642E0A4730205A31C1
:100B8000300A47302045300A4D333030205032355E
:100B900020533838300A4D33303020503530205310
:100BA000300A4D3330302050323520533838300A37
:100BB0004D333030205035302053300A4D333030F3
:100BC0002050323520533838300A47342053310012
:100BD00070726F62655F6661696C6564004D31318A
:100BE000372050726F626520737563636573736637
:100BF000756C0A00205A3A200020593A20004265BC
:100C00006420583A200020204261636B3A20002083
:100C10002052696768743A200020204C6566743A57
:100C200020002020546F703A200053696465733AA5
:100C30000A00205A0020580043656E7465723A0A13
:100C4000002020546F703A200020204261636B3AEC
:100C50002000202052696768743A200020204C65EB
:100C600066743A20004261636B6C6173683A0A00F3
:100C70002058004E6F7A7A6C6520546970204F7549
:100C80007465722044696D656E73696F6E733A0A9C
:100C900000205A0020580020506F736974696F6EED
:100CA000616C204572726F723A0A00436C69636B23
:100CB00020746F20726573756D652E2E2E004E6F39
:100CC000206D6F76652E00456E642066696C652028
:100CD0006C6973740A00426567696E2066696C65A9
:100CE000206C6973740A00286E6F2066696C652930
:100CF0000043757272656E742066696C653A2000F7
:100D00005344207072696E74696E672062797465ED
:100D100020004E6F74205344207072696E74696EA7
:100D2000670A002E0A0044656C6574696F6E206660
:100D300061696C65642C2046696C653A20004669DF
:100D40006C652064656C657465643A005072696E08
:100D5000742074696D653A200050726F7465637415
:100D600065642050696E0A0025301D0C2829243145
:100D70001C0B4527232F1B0A1E4443222B1A4142DA
:100D8000033809FF36030806020200010A537461A2
:100D900074733A2046696C616D656E742075736575
:100DA000643A20002C204C6F6E67657374206A6F64
:100DB000623A2000546F74616C2074696D653A204A
:100DC0000053746174733A20002C204661696C658D
:100DD000643A20002C2046696E69736865643A2085
:100DE000005072696E74733A200053746174733AE0
:100DF0002000486F74656E6420436F6F6C696E6786
:100E00002E2E2E00486F74656E64204865617469EB
:100E10006E672E2E2E006F666600680463045C0405
:100E20005504470444454255473A004D313133207B
:100E300053006F6B0054415A20576F726B686F728A
:100E400073652045646974696F6E204F46462E00B5
:100E50004348414D4245525F54454D5045524154DF
:100E6000555245004D4F54494F4E5F4D4F444553E9
:100E700000544845524D414C5F50524F54454354E5
:100E8000494F4E004155544F5245504F52545F53B5
:100E9000445F5354415455530050524F4D50545F8A
:100EA000535550504F525400454D455247454E43BF
:100EB000595F50415253455200434153455F4C499D
:100EC0004748545F4252494748544E455353005493
:100ED0004F47474C455F4C494748545300534F4692
:100EE00054574152455F504F574552004255494C67
:100EF000445F50455243454E54004C4556454C497D
:100F00004E475F44415441005A5F50524F424500A2
:100F10004155544F4C4556454C005052494E545F34
:100F20004A4F420050524F47524553530041555487
:100F30004F5245504F52545F54454D5000564F4C00
:100F4000554D455452494300454550524F4D00427E
:100F5000494E4152595F46494C455F5452414E53A8
:100F60004645520053455249414C5F584F4E5F58D9
:100F70004F4646004649524D574152455F4E414DFE
:100F8000453A4D61726C696E20204649524D574179
:100F900052455F56455253494F4E3A322E302E300D
:100FA0002E3134342045585452554445525F5459DB
:100FB00050453A6C7574656669736B20534F555292
:100FC00043455F434F44455F55524C3A68747470D3
:100FD000733A2F2F636F64652E616C6570686F6262
:100FE0006A656374732E636F6D2F646966667573CB
:100FF000696F6E2F4D41524C494E2050524F544F05
:10100000434F4C5F56455253494F4E3A312E302094
:101010004D414348494E455F545950453A54415A11
:1010200020576F726B686F727365204564697469CD
:101030006F6E2045585452554445525F434F554EAC
:10104000543A3120555549443A3565653739386643
:10105000622D343036322D346433352D383232340B
:101060002D3565383436666662343561350A002FB1
:101070002F20004D31343520533C696E6465783E35
:10108000206F7574206F662072616E67652028304E
:101090002D31290A00205400205200416363656C01
:1010A00065726174696F6E3A205000205A002059B1
:1010B00000580020204D61783A2000205A00205925
:1010C00000580020204D696E3A2000536F6674204E
:1010D000656E6473746F70733A200020466C6F778E
:1010E0003A200050726F6265205A204F6666736521
:1010F000743A200020643A0020693A0020703A00D7
:10110000496E76616C696420657874727564657285
:101110000A0020643A0020693A0020703A006469AD
:101120007300656E0043290A0061626C65642028C3
:101130006D696E2074656D702000436F6C6420656E
:10114000787472756465732061726520004F46463D
:10115000004F4E00426564204C6576656C696E6791
:1011600020004661696C656420746F20656E616261
:101170006C6520426564204C6576656C696E670A13
:1011800000426564204C6576656C20436F72726521
:101190006374696F6E204D61747269783A004545D9
:1011A00050524F4D204F4B0A003F5A206F7574200C
:1011B0006F662072616E676520282D3220746F2063
:1011C00035290A0050726F6265205A204F66667397
:1011D00065743A20003F4B2076616C7565206F7511
:1011E00074206F662072616E67652028302D313063
:1011F000292E0A00416476616E6365204B3D0049EB
:101200006E76616C69642065787472756465720AC3
:10121000004361703A0047322F47332062616420F7
:10122000706172616D65746572730A00220A0065EF
:101230006E7175657565696E672022002042002019
:1012400050006F6B00526573656E643A2000535412
:101250004F505045442E20005072696E74657220C4
:1012600073746F707065642064756520746F206599
:1012700072726F72732E20466978207468652065DB
:1012800072726F7220616E6420757365204D3939FA
:101290003920746F20726573746172742E20285423
:1012A000656D706572617475726520697320726511
:1012B0007365742E205365742069742061667465AB
:1012C000722072657374617274696E67290A004EC8
:1012D0006F20436865636B73756D20776974682050
:1012E0006C696E65206E756D6265722C204C617341
:1012F00074204C696E653A20004E6F204368656328
:101300006B73756D2077697468206C696E65206EEB
:10131000756D6265722C204C617374204C696E652A
:101320003A2000636865636B73756D206D69736D3A
:10133000617463682C204C617374204C696E653A4B
:1013400020004C696E65204E756D62657220697370
:10135000206E6F74204C617374204C696E65204E52
:10136000756D6265722B312C204C617374204C6951
:101370006E653A20004D313130004D333100534419
:101380002072656164206572726F720A00446F6E2C
:1013900065207072696E74696E672066696C650A93
:1013A000002569730025696D20256973002569682A
:1013B0002025696D202569730025696420256968E9
:1013C0002025696D202569730025697920256964C8
:1013D000202569682025696D202569730020573A0A
:1013E0000042656420636F6F6C696E672E2E2E005D
:1013F0004265642068656174696E672E2E2E002335
:10140000646566696E652044454641554C545F00ED
:1014100000626564004B6420004B6920004B702023
:1014200000504944204175746F74756E652066697B
:101430006E69736865642120507574207468652036
:101440006C617374204B702C204B6920616E64209A
:101450004B6420636F6E7374616E74732066726F79
:101460006D2062656C6F7720696E746F20436F6EBC
:1014700066696775726174696F6E2E680A005049FB
:1014800044204175746F74756E65206661696C6582
:1014900064212074696D656F75740A00486F746506
:1014A0006E6420544845524D414C2052554E415790
:1014B00041590042454420544845524D414C205228
:1014C000554E4157415900546865726D616C205208
:1014D000756E6177617900486F74656E6420486548
:1014E0006174696E67206661696C65640042656459
:1014F0002068656174696E67206661696C65640067
:1015000048656174696E67206661696C6564005046
:101510004944204175746F74756E65206661696C0D
:101520006564212054656D70657261747572652003
:10153000746F6F20686967680A00204B643A200066
:10154000204B693A2000204B703A20000A20436C5F
:10155000617373696320504944200A002054753A2E
:101560002000204B753A2000206D61783A20002041
:101570006D696E3A200020643A2000206269617330
:101580003A2000504944204175746F74756E65208F
:1015900073746172740A00504944204175746F7409
:1015A000756E65206661696C6564212054656D7097
:1015B0006572617475726520746F6F206869676801
:1015C0000A00504944204175746F74756E65206639
:1015D00061696C656421204261642065787472756C
:1015E000646572206E756D6265720A004572723AAA
:1015F000207574663820666F6E74206E6F74206973
:101600006E697469616C697A65642E004572723A1C
:10161000207574663820666F6E74206E6F74206952
:101620006E697469616C697A65642E00304848306F
:1016300025753A2530327500253032753A2530321D
:101640007500253364002534640025202000252002
:101650000020202020004572723A207574663820E0
:10166000666F6E74206E6F7420696E697469616C48
:10167000697A65642E001FFFFFFFFFFFFF60000017
:10168000000001FF400000000000FF80000000009B
:10169000007F83CF00000C303F87FF80000C301F9D
:1016A000867980000C000F8C30C7838C30E78C303B
:1016B000CFC7CC31F38C30DCECEC33B98C30D86C48
:1016C0006C33198C30D06C0C33198C30D86C0C33D3
:1016D000198C30DC6C0E3B198C30CF7C079F198C39
:1016E00030C77C038F19400000000000026000003A
:1016F000000000061FFFFFFFFFFFF86F6F6F000085
:101700000047414D45204F56455200107CFEFEFEDD
:1017100044402480000031800000248044400400C4
:101720000E000E007FC0FFE0FFE0FFE0FFE01FC003
:101730007FF0DDD8FFF87FF006000F001F8036C075
:101740003FC009001680294006000F001F8036C0E8
:101750003FC0168020401080104008801FC03760B6
:101760007FF05FD050500D80104048905FD0777070
:101770007FF01FC0104020200F007FE0FFF0E670D8
:10178000FFF0198036C0C0300F007FE0FFF0E67038
:10179000FFF0198036C019800A003B2045455052A1
:1017A0004F4D20496E6465783A200055706461742D
:1017B000696E67207A6F666673657420696E20456E
:1017C0004550524F4D3A200001FC0007FF000F0723
:1017D000800E01C00001C00000E00800E01C00E035
:1017E0003E00E07F00E01C00E00E00E00E01C007BC
:1017F00083C003FF8000FE0000FE0003FF8007831C
:10180000C00E01C00E00E01C00E07F00E03E00E0E2
:101810001C00E00800E00000E00001C00E01C00F65
:10182000078007FF0001FC000E000E000E000E00F6
:101830000E000E000E000E007FC03F801F000E0045
:10184000040004000E001F003F807FC00E000E0049
:101850000E000E000E000E000E000E00FFFFFF7FB8
:1018600080FFC0FFC0FFC07F807F80FFC0FFC0FF40
:10187000C03F001E000C0050726F6265205A204F5E
:101880006666736574004C6F6164206D6D004C6F0B
:101890006164206D6D00556E6C6F6164206D6D002C
:1018A000556E6C6F6164206D6D00416476616E638E
:1018B00065204B00416476616E6365204B00416496
:1018C00076616E6365642053657474696E67730036
:1018D0005654726176206D696E005654726176209E
:1018E0006D696E00566D696E00566D696E00566DBD
:1018F0006178204500566D6178204500566D61780D
:10190000205A00566D6178205A00566D6178205932
:1019100000566D6178205900566D61782058005648
:101920006D6178205800416476616E636564205370
:10193000657474696E677300416D6178204500417C
:101940006D6178204500416D6178205A00416D61DC
:1019500078205A00416D6178205900416D617820EE
:101960005900416D6178205800416D617820580020
:10197000412D74726176656C00412D7472617665DB
:101980006C00412D7265747261637400412D726543
:10199000747261637400416363656C0041636365E5
:1019A0006C00416476616E6365642053657474698C
:1019B0006E67730056652D6A65726B0056652D6AF9
:1019C00065726B00567A2D6A65726B00567A2D6AC5
:1019D00065726B0056792D6A65726B0056792D6AB7
:1019E00065726B0056782D6A65726B0056782D6AA9
:1019F00065726B00416476616E6365642053657443
:101A000074696E6773004573746570732F6D6D0034
:101A10004573746570732F6D6D005A7374657073C0
:101A20002F6D6D005A73746570732F6D6D0059734F
:101A3000746570732F6D6D005973746570732F6DBD
:101A40006D005873746570732F6D6D0058737465F5
:101A500070732F6D6D00416476616E636564205311
:101A6000657474696E67730046696C616D656E7448
:101A7000004261636B6C6173680053746570732F0F
:101A80006D6D004A65726B00416363656C657261E0
:101A900074696F6E0056656C6F6369747900436F8B
:101AA0006E66696775726174696F6E00536D6F6FF2
:101AB0007468696E6700536D6F6F7468696E670054
:101AC0005A005A005900590058005800436F72726A
:101AD000656374696F6E00436F7272656374696FDA
:101AE0006E004D61696E004C6F61642073657474A3
:101AF000696E677300526573746F72652066616901
:101B00006C736166650053746F72652073657474DD
:101B1000696E67730050726F6265205A204F666667
:101B200073657400416476616E6365642053657407
:101B300074696E6773004D61696E004D37303220F5
:101B4000542564004D363030204230205425640046
:101B50004D373032203B2564004D3730312054253D
:101B600064004368616E67652066696C616D656ECF
:101B700074005072656865617420437573746F6D8D
:101B8000005072656865617420414253005072656F
:101B90006865617420504C410050726568656174DD
:101BA00020437573746F6D004261636B00456E6412
:101BB0002066696C616D656E74206368616E67652F
:101BC000005075726765206D6F7265000043686133
:101BD0006E67696E672046696C616D656E7400554D
:101BE0004E4C4F41442046494C414D454E54004CCB
:101BF0004F41442046494C414D454E540020204E13
:101C00006F7A7A6C653A200020005061726B696EC1
:101C1000672E2E2E00746F207374617274006669D3
:101C20006C616D656E74206368616E6765005761F5
:101C3000697420666F720066696C616D656E7420F0
:101C4000756E6C6F6164005761697420666F720015
:101C5000506C6561736520776169742E2E2E004E7D
:101C60006F7A7A6C652068656174696E6700746F5D
:101C70002068656174206E6F7A7A6C6500507265B9
:101C8000737320627574746F6E00746F20636F6E6F
:101C900074696E756500616E64207072657373207F
:101CA000627574746F6E00496E7365727420666934
:101CB0006C616D656E740066696C616D656E742033
:101CC0006C6F6164005761697420666F7200746F95
:101CD00020726573756D65207072696E7400507244
:101CE00065737320627574746F6E00506C656173F8
:101CF0006520776169742E000066696C616D656EA0
:101D000074207075726765005761697420666F7220
:101D100000536E346B3300496E76616465727300F4
:101D2000427269636B6F7574004D61696E003E208D
:101D300000457874727564656420746F74616C3AE0
:101D400000256C642E25696D003E20004C6F6E6787
:101D5000657374206A6F622074696D653A003E2075
:101D600000546F74616C207072696E742074696DB8
:101D7000653A00436F6D706C657465643A2000507D
:101D800072696E7420436F756E743A200047616DFE
:101D90006573005072696E74657220537461747358
:101DA000004669726D776172652056657273696F5E
:101DB0006E004D61696E003F0053746F7020707249
:101DC000696E74004261636B0053746F70004D3232
:101DD0003520500A4D3234005072696E74207061A3
:101DE00075736564005061757365207072696E74F7
:101DF00000726573756D65004D3234005072696E06
:101E0000742066726F6D205344004368616E67658D
:101E10002053442063617264004D32310041626F8F
:101E20007574205072696E746572004368616E67E4
:101E3000652066696C616D656E74004368616E67EC
:101E4000652066696C616D656E74004D36303020BA
:101E5000423000436F6E66696775726174696F6EB8
:101E60000054656D7065726174757265004D6F76B2
:101E7000656D656E7400526573756D65207072696D
:101E80006E74004E6F205344206361726400547579
:101E90006E650053746F70207072696E74005061CB
:101EA000757365207072696E7400496E666F207379
:101EB000637265656E004D6F76652058004D6F76D4
:101EC000652059004D6F7665205A0045787472750B
:101ED00064657220004578747275646572200041F3
:101EE00075746F20686F6D6500473238004D6F76EE
:101EF00065205A004D6F76652059004D6F7665203C
:101F000058004D6F76656D656E740044697361624B
:101F10006C65207374657070657273004D383400A1
:101F20004175746F2063616C696272617465004D04
:101F3000313137205374617274696E672041757452
:101F40006F2D43616C6962726174696F6E0A5430FF
:101F50000A4D323138205431205834332059302042
:101F60005A300A4732380A4D313137204C65766590
:101F70006C696E67205820417869730A4730205891
:101F80003135302046393939390A473238205A300C
:101F90000A4D313137204C6576656C696E67206477
:101FA0006F6E652E0A4731320A4D31313720436159
:101FB0006C6962726174696E672E2E2E0A47343224
:101FC000350A4D3530300A4D3131372043616C6967
:101FD00062726174696F6E206461746120736176EE
:101FE0006564004175746F20686F6D650047323815
:101FF000004C6576656C20582061786973004D311E
:102000003137204C6576656C696E672058204178C1
:1020100069730A473020583135302046393939390B
:102020000A473238205A300A4D313137204C657614
:10203000656C696E6720646F6E652E0A004D6F7661
:10204000652061786973004D61696E003F005374CB
:10205000617274207072696E74200043616E6365F2
:102060006C005072696E740043616E6E6F7420650F
:102070006E746572207375626469723A2000022E74
:102080002E004D61696E00436F6F6C646F776E0058
:1020900046616E20737065656420310046616E2074
:1020A00073706565642031004265640042656400B8
:1020B0004E6F7A7A6C65004E6F7A7A6C65004D616E
:1020C000696E0042616279737465702058004261E4
:1020D00062797374657020590050726F6265205A7E
:1020E000204F66667365740042616279737465702F
:1020F0002059004261627973746570205800466C03
:102100006F7700466C6F770046616E20737065656F
:102110006420310046616E20737065656420310073
:1021200042656400426564004E6F7A7A6C65004EC9
:102130006F7A7A6C650053706565640053706565ED
:1021400064004D61696E000000007E006000600068
:1021500060F87ECC60CC60CC60F860CC00CC00CC69
:1021600000CC0000000000000000000000000000A3
:1021700000000000000000000000000000FE7FFEE4
:102180007F06600000000000000000F00FF81FF85C
:102190001FF81FF00FF00FF81FF81FF81FE007C01F
:1021A000038001000000000000FE7F0E70266472B4
:1021B0004E7A5E324C8241324C7A5E724E26640E0A
:1021C00070FE7F000000000000FE7F0E70C663C23C
:1021D0004382411A58BA5D1A588241C243C6630EFF
:1021E00070FE7F00000000000088088808101120A1
:1021F0002220221011880888081011000000000019
:102200000000000000000000002022101188088853
:102210000810112022202210118808000000000060
:1022200000000000000000436172642072656D6F61
:10223000766564004361726420696E7365727465CB
:1022400064004C756C7A426F742054415A20726558
:102250006164792E005072696E74696E672E2E2E3D
:10226000005072696E7420706175736564006361FB
:102270006E63656C005072696E742061626F727477
:102280006564000000914300009A430040964300BB
:10229000005CC20000F0C1000000C0290A002062FA
:1022A000797465733B2063726320005365747469AD
:1022B0006E67732053746F72656420280045455023
:1022C000524F4D206461746173697A652065727242
:1022D0006F722E0A00290A002062797465733B2010
:1022E00063726320002073746F7265642073657479
:1022F00074696E67732072657472696576656420AF
:102300002800202863616C63756C61746564292101
:102310000A0020213D2000454550524F4D20435298
:1023200043206D69736D61746368202D2028737478
:102330006F7265642920002053697A653A2000494C
:102340006E6465783A2000204D61726C696E3D566E
:102350003637290A00454550524F4D207665727335
:10236000696F6E206D69736D6174636820284545DF
:1023700050524F4D3D00454550524F4D20496E69DA
:102380007469616C697A65640A0048617264636F9C
:102390006465642044656661756C7420536574746B
:1023A000696E6773204C6F616465640A00282300BE
:1023B0000028230000C80000002823000000009629
:1023C00043000096430000F0410000C8410000C8EF
:1023D000420000C8420000FA430080CF433A0A009E
:1023E00020204D3630332000205300205A00205941
:1023F0000020580020204D343235204600426163D1
:102400006B6C61736820636F6D70656E7361746966
:102410006F6E3A0A002055004C0046696C616D658C
:102420006E74206C6F61642F756E6C6F6164206CCC
:10243000656E677468733A0A0020204D3930302089
:102440004B004C696E65617220416476616E636514
:102450003A0A0020204D383531205A005A2D50724A
:102460006F6265204F6666736574002044002049E2
:102470000020204D333034205000204400204900FB
:1024800020204D3330312050005049442073657472
:1024900074696E67733A0A002046002042002048A3
:1024A0000020204D3134352053004D617465726930
:1024B000616C2068656174757020706172616D6512
:1024C000746572733A0A0020204D34323020530074
:1024D0004175746F20426564204C6576656C696E49
:1024E000673A0A00204500205A0020590020580071
:1024F00020540020530020204D323035204200204F
:10250000453C6D61785F655F6A65726B3E0020587F
:102510003C6D61785F785F6A65726B3E20593C6DF7
:1025200061785F795F6A65726B3E205A3C6D6178B5
:102530005F7A5F6A65726B3E00416476616E6365C7
:10254000643A20423C6D696E5F7365676D656E74B9
:102550005F74696D655F75733E20533C6D696E5F96
:1025600066656564726174653E20543C6D696E5F9A
:1025700074726176656C5F66656564726174653EF0
:102580000020540020520020204D323034205000D2
:10259000416363656C65726174696F6E2028756E46
:1025A0006974732F7332293A20503C7072696E74CB
:1025B0005F616363656C3E20523C72657472616357
:1025C000745F616363656C3E20543C747261766530
:1025D0006C5F616363656C3E0A00204500205A0011
:1025E00020590020204D3230312058004D6178694B
:1025F0006D756D20416363656C65726174696F6EA2
:102600002028756E6974732F7332293A0A002045A9
:1026100000205A0020590020204D3230332058002D
:102620004D6178696D756D2066656564726174656C
:10263000732028756E6974732F73293A0A005374D6
:102640006570732070657220756E69743A0A002097
:10265000204D3134392043203B20556E697473205E
:10266000696E2043656C736975730A0020286D6D6F
:1026700029002020473231202020203B20556E6940
:10268000747320696E206D6D006F70656E0054521A
:1026900049474745524544003A20007A5F6D6178CA
:1026A000007A5F6D696E00795F6D696E00785F6DAD
:1026B000696E005265706F7274696E6720656E6432
:1026C00073746F70207374617475730A00205A3AC2
:1026D0000020593A0020436F756E7420583A00204C
:1026E000453A00205A3A0020593A00583A00486FBB
:1026F0006D652025732573257320666972737400D8
:102700002066697273740A00486F6D6520000000CE
:102710005CC20000F0C10040964300004842000047
:1027200048420000F0415761726E696E673A204876
:102730006F6D696E672042756D70204469766973AC
:102740006F72203C20310A000202040000A0400009
:1027500000A040000000400080AC430000A94300FE
:10276000409743FFFF0124F4D43050C38E20C2A20F
:102770004017828B7011127A910D816CD90AA86171
:10278000E108C7586607615143061E4B5D05C14508
:10279000A7041A411104093D9803713931034036E9
:1027A000DB0265339102D4305402802E1D02632C6B
:1027B000EE01752AC501B028A001102781018F25DF
:1027C00064012B244B01E0223401AC211F018D2038
:1027D0000D01801FFC00841EED00971DDF00B81C5A
:1027E000D200E61BC600201BBC00641AB200B2195E
:1027F000A8000A19A0006A189900D1179100401783
:102800008B00B516840031167E00B31579003A1599
:102810007300C7146F0058146A00EE136600881323
:10282000630025135E00C7125B006C12570015127F
:102830005400C111510070114F0021114B00D610EE
:1028400049008D1047004610440002104200C00F9E
:102850004000800F3E00420F3C00060F3B00CB0EB5
:102860003800930E37005C0E3500270E3400F30D50
:102870003200C10D3100900D3000600D2E00320D80
:102880002D00050D2C00D90C2B00AE0C2900850C59
:1028900029005C0C2700350C27000E0C2600E80BE5
:1028A0002400C40B2400A00B23007D0B23005A0B33
:1028B0002100390B2100180B2000F80A1F00D90A4B
:1028C0001E00BB0A1E009D0A1D00800A1D00630A2F
:1028D0001C00470A1B002C0A1B00110A1A00F709EA
:1028E0001A00DD091900C4091900AB091900920981
:1028F00017007B091800630917004C0916003609F8
:102900001600200916000A091500F5081500E00850
:102910001400CC081400B8081400A408140090088F
:1029200013007D0812006B081300580812004608B7
:1029300012003408110023081100120811000108C8
:102940001100F0071000E0071000D0071000C007CA
:102950001000B0070F00A107100091070E008307B9
:102960000F0074070F0065070E0057070E00490798
:102970000E003B070D002E070E0020070D00130769
:102980000D0006070D00F9060C00ED060D00E0062F
:102990000C00D4060C00C8060C00BC060C00B006E7
:1029A0000C00A4060B0099060C008D060B00820695
:1029B0000B0077060B006C060B0061060A00570639
:1029C0000B004C060A0042060A0038060A002E06D2
:1029D0000A0024060A001A060A0010060900070663
:1029E0000A00FD050900F4050900EB050900E205F0
:1029F0000900D9050900D0050900C7050900BE0571
:102A00000900B5050800AD050800A50509009C05ED
:102A10000800940508008C050800840508007C0562
:102A20000800740508006C050700650508005D05D1
:102A30000700560508004E0507004705070040053A
:102A4000080038050700310507002A05070023059F
:102A500007001C050600160507000F0507000805FE
:102A6000060002050700FB040600F5040700EE045B
:102A70000600E8040600E2040700DB040600D504B3
:102A80000600CF040600C9040600C3040600BD0406
:102A90000600B7040600B1040500AC040600A60455
:102AA0000600A00405009B040600950405009004A0
:102AB00006008A04050085040500800406007A04E7
:102AC000050075040500700405006B04050066042C
:102AD0000500610405005C0405005704050052046C
:102AE00005004D04050048040500430405003E04AC
:102AF00004003A04050035040500300404002C04E9
:102B0000050027040400230405001E0404001A0421
:102B1000040016040500110404000D040400090457
:102B200005000404040000040400FC030400F8038E
:102B30000400F4030400F0030400EC030400E803C1
:102B40000400E4030400E0030400DC030400D803F1
:102B50000400D4030400D0030400CC030400C80321
:102B60000300C503030024F404D9201BC40C5C0E2D
:102B70009804C4095F0265077101F405F900FB04BC
:102B8000B30048048700C1036900580355000303DC
:102B90004500BE023A008402310053022A00290295
:102BA000250004022000E4011C00C8011900AF0147
:102BB00017009801140084011300710110006101D5
:102BC000100051010E0043010D0036010B002B01D6
:102BD0000B0020010B00150109000C010900030185
:102BE0000800FB000800F3000800EB000700E40009
:102BF0000600DE000600D8000600D2000600CC0069
:102C00000500C7000500C2000500BD000400B900B2
:102C10000400B5000400B1000400AD000400A900E8
:102C20000400A5000300A20003009F0004009B0015
:102C30000300980003009500020093000300900039
:102C400003008D0002008B00030088000200860054
:102C5000020084000300810002007F0002007D006A
:102C600002007B000200790002007700010076007C
:102C700002007400020072000100710002006F0087
:102C800002006D0001006C0002006A000100690092
:102C90000200670001006600010065000100640099
:102CA00002006200010061000100600001005F009D
:102CB00002005D0001005C0001005B0001005A00A1
:102CC00001005900010058000100570001005600A2
:102CD00001005500010054000100530000005300A2
:102CE00001005200010051000100500001004F009E
:102CF00001004E0000004E0001004D0001004C009C
:102D000001004B0000004B0001004A000100490097
:102D10000100480000004800010047000100460093
:102D2000000046000100450000004500010044008D
:102D30000100430000004300010042000000420087
:102D400001004100000041000100400001003F007F
:102D500000003F0001003E0000003E0001003D0079
:102D600000003D0001003C0000003C0000003C0071
:102D700001003B0000003B0001003A0000003A0067
:102D8000010039000000390001003800000038005F
:102D90000000380001003700000037000100360055
:102DA000000036000000360001003500000035004C
:102DB0000000350001003400000034000000340041
:102DC0000100330000003300000033000100320036
:102DD000000032000000320001003100000031002C
:102DE0000000310001003000000030000000300021
:102DF00001002F0000002F0000002F0000002F0016
:102E000001002E0000002E0000002E0001002D0009
:102E100000002D0000002D0000002D0001002C00FE
:102E200000002C0000002C0000002C0001002B00F2
:102E300000002B0000002B0000002B0001002A00E6
:102E400000002A0000002A0000002A0001002900DA
:102E500000002900000029000000290000002900CE
:102E600001002800000028000000280000002800C1
:102E700000002800010027000000270000002700B4
:102E800000002700000027000100260000002600A7
:102E9000000026000000260000002600010025009A
:102EA000000025000000250000002500000025008E
:102EB0000000250001002400000024000000240080
:102EC0000000240000002400010023000000230073
:102ED0000000230000002300000023000000230066
:102EE0000000230001002200000022000000220058
:102EF000000022000000220000002200010021004A
:102F0000000021000000210000002100000021003D
:102F1000000021000000210001002000000020002E
:102F20000000200000002000000020000000200021
:102F3000000020000000200001001F0000001F0012
:102F400000001F0000001F0000001F0000001F0005
:102F500000001F0001001E0000001E0000001E00F7
:102F600000001E000000C23100001C260000F41901
:102F70000000D80F0000EB080000C004000075023C
:102F80000000400100004D6963726F7374657073D7
:102F900020756E617661696C61626C650A0045310D
:102FA0003A200045303A20005A3A2000593A200091
:102FB0004D53312C4D53322C4D53332050696E7389
:102FC0000A583A2000626564002C20737973746596
:102FD0006D2073746F70706564212048656174653D
:102FE000725F49443A2000426564206865617469F3
:102FF0006E67206661696C65640048656174696E1E
:1030000067206661696C6564004245442054484508
:10301000524D414C2052554E41574159005468651C
:10302000726D616C2052756E6177617900486F74C2
:10303000656E642048656174696E67206661696CBD
:1030400065640048656174696E67206661696C65D6
:103050006400486F74656E6420544845524D414C7D
:103060002052554E4157415900546865726D616C4C
:103070002052756E61776179001000AD0330016AEE
:103080000150022B0170030A019004F500B005E520
:1030900000D006D800F007CE001009C500300ABEE7
:1030A00000500BB700700CB100900DAB00B00EA635
:1030B00000D00FA200F0109D00101299003013955F
:1030C000005014920070158E0090168B00B0178778
:1030D00000D0188400F0198100101B7E00301C7B8A
:1030E00000501D7900701E7600901F7300B0207094
:1030F00000D0216E00F0226B00102469003025669C
:1031000000502663007027610090285E00B0295CA3
:1031100000D02A5900F02B5600102D5400302E51AB
:1031200000502F4E0070304B0090314800B03245B7
:1031300000D0334200F0343E0010363B00303737C9
:10314000005038330070392E00903A2900B03B23EC
:1031500000D03C1B00F03D1100103F0100F03F008B
:1031600000486F74656E64204572723A204D415874
:1031700054454D50004572723A204D415854454DCA
:103180005020424544004D415854454D50207472E2
:103190006967676572656400486F74656E64204591
:1031A00072723A204D494E54454D50004572723A64
:1031B000204D494E54454D5020424544004D494E06
:1031C00054454D50207472696767657265640020CC
:1031D0002F002042403A0020403A0020573A007C1D
:1031E0003C3E5E2B3D3F2F5B5D3B2C2A225C00105A
:1031F00000C90210012C014001220170011801B028
:10320000010E01F00104015002FA00B002F000309A
:1032100003E600D003DC009004D2007005C800A0D3
:1032200006BE000008B400B009AA00D00BA00060E0
:103230000E960060118C000015820020197800C0E5
:103240001D6E00A0226400B0275A00902C50000090
:10325000314600E0343C0010383200903A280060DB
:103260003C1E00A03D1400803E0A00203F000043A9
:10327000616E6E6F74206F70656E20737562646925
:1032800072200053442063617264206F6B0A006FE8
:1032900070656E526F6F74206661696C65640A00B8
:1032A000766F6C756D652E696E6974206661696CE8
:1032B00065640A00534420696E6974206661696C14
:1032C0000A004D3234004D323320257300577269A5
:1032D00074696E6720746F2066696C653A20002EF1
:1032E0000A006F70656E206661696C65642C20460B
:1032F000696C653A20002E0A006F70656E20666169
:10330000696C65642C2046696C653A200046696CDE
:10331000652073656C65637465640A002053697A7F
:10332000653A200046696C65206F70656E65643A89
:103330002000667265736800646F696E67002066BE
:10334000696C653A20004E6F772000454E4420534B
:103350005542524F5554494E450A002220706F7312
:10336000002220706172656E743A220053554252F9
:103370004F5554494E452043414C4C20746172676F
:1033800065743A2200747279696E6720746F2063E5
:10339000616C6C207375622D67636F64652066696C
:1033A0006C6573207769746820746F6F206D616E2F
:1033B00079206C6576656C732E204D4158206C65C4
:1033C00076656C2069733A310A0000000A0B020925
:1033D0000C0D0E08070304010000000000000000AF
:1033E00000000000000000000000000000000000DD
:1033F000000000000000121110000000000000009A
:1034000000000000000000000000000000000000BC
:1034100000000000000000000000000000000000AC
:10342000473238205A002020506C616E6E6572421F
:10343000756666657242797465733A20002046723B
:103440006565204D656D6F72793A2000436F6D7030
:10345000696C65643A204E6F76203130203230320C
:10346000300A00207C20417574686F723A2028462B
:10347000616D6520334420496E632E2C204C756CA1
:103480007A426F7420476974205265706F73697453
:103490006F7279290A0000204C61737420557064A2
:1034A000617465643A2000322E302E302E3134346F
:1034B0000A004D61726C696E0020536F667477610B
:1034C00072652052657365740A00205761746368E1
:1034D000646F672052657365740A002042726F77CB
:1034E0006E206F75742052657365740A00204578EC
:1034F0007465726E616C2052657365740A00506F5A
:1035000077657255700A0073746172740A00617590
:10351000746F25632E67006572726F72207772690F
:1035200074696E6720746F2066696C650A00446F69
:103530006E6520736176696E672066696C652E0A18
:10354000004D323900456E6473746F7073202563CB
:1035500020256320256320256300205A3A00205946
:103560003A0020583A00656E6473746F7073206877
:1035700069743A20004739310A4730205A313520E2
:10358000463630300A4739300A4730205831373014
:1035900020593239302046333030300A4D313137FE
:1035A000205072696E742061626F727465642E00BF
:1035B0004D6F766520302E3032356D6D004D6F7653
:1035C0006520302E316D6D004D6F766520316D6D4B
:1035D000004D6F76652031306D6D004D6F76652042
:1035E0006178697300486F74656E6420746F6F2032
:1035F000636F6C6400457874727564657220004D69
:103600006F7665205A004D6F76652059004D6F76B4
:1036100065205800000000000000000000000000CD
:10362000000000000000000000000000000000009A
:10363000000000000000000C000000000000000C72
:103640000000000000000012000000000000002345
:103650000000000000000021000000000000004CFD
:10366000800000000000005E80000000000000926A
:1036700040000000000000A1400000000000012107
:10368000200000000000027F900000000000020007
:1036900010000000000007FFF80000000000040018
:1036A00008000000000008000400000000000800FE
:1036B0000600000000001000020000000000301EA4
:1036C000010000000000207F81000000000041FF99
:1036D000E0800000000043FCF08000000000873B19
:1036E0007840000000018EDBFC60000000010FEB61
:1036F000CC20000000021FEDB610000000021FDE0B
:10370000B6100000000439CD7F080000000436E048
:10371000FF08000000087EC0BB84000000187F0086
:103720005D86000000107FC0ED82000000203CC0DC
:103730007301000000203B337F01000000701BE795
:103740007E03800000C81DEEDE04C00000880FDE8E
:10375000DC04400001240FDF3C092000012607DBC8
:10376000F8192000027203E7F0139000025101FFE4
:10377000E02290000489007F802448000904801E14
:10378000004824000BFE400000DFF4001000400061
:10379000008002001FFFFFFFFFFFFE00000000008F
:1037A0000000000000000000000000000000000019
:1037B000000000001022103C3C0E1F0010221004DC
:1037C00022110400102210082211040010221008F7
:1037D0003C110400102210102211040010221020AD
:1037E000221104001E1C1E3C3C0E040000000000C0
:1037F00000000000000000000000000000000000C9
:1038000000000000000000000000000000000000B8
:1038100000000000000000000000000000000000A8
:103820000000000000000000000000000000000098
:103830000000000000000000000000000000000088
:103840000000000000000000000000000000000078
:1038500000004175746F6C6576656C206661696CFB
:1038600065640A004175746F6C6576656C206661ED
:10387000696C656400220A00556E6B6E6F776E206E
:10388000636F6D6D616E643A20220020746F6F204B
:103890006C6F6E6720657874727573696F6E2070D7
:1038A000726576656E7465640A0020636F6C6420CF
:1038B000657874727573696F6E2070726576656E67
:1038C0007465640A00204500205A00205900204DEC
:1038D00039322058002E0A006F70656E20666169CB
:1038E0006C65642C2046696C653A2000000022005B
:1038F000250028002B002E003100340002010000BA
:10390000050108010B0100002100240027002A0006
:103910002D003000330001010000040107010A01FD
:1039200005050505070508080808020202020A0A3B
:103930000808040404040101010101010101030359
:10394000030303030303040707070C0C0C0C0C0C04
:103950000C0C0202020206060606060606060B0B01
:103960000B0B0B0B0B0B07070A0A0A0A0A0A0505C1
:103970000504040408080102102020080810204053
:103980001020408002010201080402010102040823
:1039900010204080804020100804020180040201B1
:1039A00080402010080402010804020101020408FA
:1039B00010204080010204081020408010080408F4
:1039C000801020400440801020400480486F7465BF
:1039D0006E6420544845524D414C2052554E41573B
:1039E00041590042454420544845524D414C2052D3
:1039F000554E4157415900546865726D616C2052B3
:103A0000756E61776179002F2F616374696F6E3A0B
:103A10000001050800FF060121023520FFFF07FF16
:103A200006FF0900502216568080808000801533E2
:103A300053A0A0A00257575050F850F850500257CA
:103A4000572070A07028702013355580A040A0200A
:103A500002475740A0A040A0A0502513538080806B
:103A6000122656408080808040122656804040407A
:103A700040800245559060F060900255552020F836
:103A80002020113353604080044151F011335340E2
:103A9000E04002465610102040808012365640A06A
:103AA000A0A0A04012365640C0404040E00246561A
:103AB0006090106080F0024656F020601090600226
:103AC00046562060A0F02020024656F080E010907C
:103AD000600246566080E0909060024656F01020EA
:103AE00020404002465660906090906002465660CA
:103AF0009090701060122555C0C000C0C01136569D
:103B00006060006040801236562040808040200374
:103B10004353F000F0123656804020204080123689
:103B20005640A020400040015858304898A8A8901E
:103B30004030024656609090F09090024656E090D9
:103B4000E09090E002465660908080906002465679
:103B5000E090909090E0024656F080E08080F00285
:103B60004656F080E0808080024656609080B0909B
:103B7000600246569090F0909090123656E0404089
:103B80004040E002465670202020A0400246569059
:103B9000A0C0A0A0900246568080808080F002469F
:103BA0005690F0F090909002465690D0F0B0B090C1
:103BB000024656609090909060024656E09090E0E9
:103BC0008080014757609090D0B06010024656E068
:103BD0009090E0909002465660904020906012369F
:103BE00056E0404040404002465690909090906091
:103BF000024656909090906060024656909090F0E9
:103C0000F0900246569090606090900256568888D8
:103C100050202020024656F010204080F0123656E8
:103C2000E080808080E002465680804020101012A4
:103C30003656E020202020E016325240A0014151AB
:103C4000F016225280400244547090907002465602
:103C50008080E09090E0123454608080600246568C
:103C600010107090907002445460B0C060024656CC
:103C7000205040E040400145556090701060024681
:103C8000568080E09090901236564000C04040E050
:103C90001137572000202020A040024656808090F7
:103CA000E09090123656C040404040E0025454D05C
:103CB000A8A8A8024454E0909090024454609090C8
:103CC00060014555E090E08080014555709070108E
:103CD00010024454A0D0808012345460C020C0022E
:103CE00046564040E040502002445490909070125C
:103CF0003454A0A0A04002545488A8A850024454B0
:103D0000906060900145559090709060024454F02E
:103D10002040F0024757304020C020403022165645
:103D2000808080808080024757C02040304020C083
:103D300006425250A0FFFFFFFFFFFFFFFFFFFFFF04
:103D4000FFFFFFFFFFFFFFFFFFFFFFFFFFFFFFFF83
:103D5000FFFFFFFFFFFF0900502216568000808002
:103D600080800146562070A0A07020024656205048
:103D7000E04050A002555588705070880256568811
:103D800050F820F820221757808080008080800221
:103D900047577080E0907010E0173151A0025656DE
:103DA00070A8C8C8A87014355560A06000E003432F
:103DB0005350A050123353E02020143151E00256EA
:103DC0005670E8D8E8D870173151E015335340A049
:103DD0004012355540E04000E014355540A02040E9
:103DE000E0143555C020C020C01622524080014545
:103DF00055909090E08002565678E8E8682828248C
:103E0000115180112252408014355540C04040E08D
:103E100014355540A04000E0034353A050A0024792
:103E200057808080A060F0200247578080A0D0108B
:103E3000207002475780408060A0F0201236564024
:103E4000004080A04002475740206090F0909002D0
:103E5000475720406090F0909002475760906090E4
:103E6000F0909002475750A06090F0909002475712
:103E700090006090F0909002475760906090F090B2
:103E80009002465670A0A0F0A0B001475760908005
:103E9000809060400247574020F080E080F0024769
:103EA000572040F080E080F00247576090F080E0BB
:103EB00080F00247579000F080E080F01237578082
:103EC00040E0404040E01237572040E0404040E0B2
:103ED00012375740A0E0404040E0123757A000E0C2
:103EE000404040E00256567048E848487002475744
:103EF00050A090D0B0909002475740206090909092
:103F00006002475720406090909060024757609051
:103F1000609090906002475750A06090909060022F
:103F2000475790006090909060123353A040A002D9
:103F3000465670B0B0D0D0E00247574020909090E5
:103F400090600247572040909090906002475760E1
:103F50009090909090600247579000909090906061
:103F60000257571020885020202002465680E090AB
:103F700090E0800246566090A0A090A00247574073
:103F80002000709090700247572040007090907011
:103F90000247572050007090907002475750A00081
:103FA0007090907002465650007090907002475783
:103FB00060906070909070025454F068B078113541
:103FC00055608080604002475740200060B0C0606C
:103FD00002475720400060B0C06002475760900021
:103FE00060B0C060024656500060B0C060123757E3
:103FF000804000C04040E0123757204000C04040A1
:10400000E012375740A000C04040E0123656A000F2
:10401000C04040E0024757A040A0107090600247A7
:104020005750A000E09090900247574020006090C9
:1040300090600247572040006090906002475760B0
:1040400090006090906002475750A0006090906090
:104050000246569000609090601235554000E00096
:104060004002445470B0D0E0024757402000909086
:104070009070024757204000909090700247576020
:104080009000909090700246569000909090700131
:10409000485820400090907090600147578080E021
:1040A00090E08080014757900090907090600105EB
:1040B0000700FE0500FB01F220FFFE05FE05FE02E3
:1040C00000400215258080800080053242A0A002B9
:1040D000556550F850F8500146562070C030E02029
:1040E00002556590102040480255656080689068D0
:1040F00005122280800225354080808040022535CF
:104100008040404080043343A040A003334340E05C
:10411000400122324080043141E0021121800255E9
:1041200065081020408002455560909090600225FF
:1041300035C040404040024555E0106080F00245E7
:1041400055E0106010E00245552060A0F0200245C7
:1041500055F080E010E00245556080E09060024537
:1041600055F0102040400245556090609060024537
:104170005560907010600313238000800214248027
:104180000080800235452040804020033343E0001A
:10419000E00235458040204080024555E010600037
:1041A000400255657088B8A870024555609090F03F
:1041B00090024555E090E090E002354560808080B7
:1041C00060024555E0909090E0023545E080E08047
:1041D000E0023545E080E080800245557080B09077
:1041E000700245559090F09090023545E040404077
:1041F000E0024555301010906002455590A0C0A0D7
:104200009002354580808080E002556588D8A88876
:104210008802455590D0B09090024555609090909E
:1042200060024555E09090E0800146566090909085
:104230006010024555E09090E09002455570806016
:1042400010E0023545E040404040024555909090D6
:1042500090600245559090A0A04002556588A8A89E
:10426000A8500245559090609090024555909070EE
:104270001060023545E0204080E0022535C0808096
:1042800080C00255658040201008022535C040409E
:1042900040C005324240A0024151F0052232804028
:1042A0000244547090907002455580E09090E00276
:1042B00034446080806002455510709090700244D4
:1042C0005460B0C0600235452040E0404000465692
:1042D00070909070106002455580E09090900215AB
:1042E000258000808080002737400040404040808B
:1042F0000245558090A0E090021525808080808046
:10430000025464F0A8A8A8024454E090909002449B
:104310005460909060004656E09090E080800046A7
:1043200056709090701010023444A0C080800244F7
:104330005470C030E002354540E040402002445413
:10434000909090700244549090A040025464A8A8A9
:104350005050023444A04040A000465690909070C7
:104360001060024454F02040F00235456040804027
:10437000600215258080808080023545C040204045
:10438000C005425250A0FFFFFFFFFFFFFFFFFFFFEE
:10439000FFFFFFFFFFFFFFFFFFFFFFFFFFFFFFFF2D
:1043A000FFFFFFFFFFFFFF020040FFFFFFFFFFFFD8
:1043B000FFFFFFFFFFFFFFFFFFFFFFFFFFFFFFFF0D
:1043C000FFFFFFFFFFFFFFFFFFFFFFFFFFFFFFFFFD
:1043D000FFFFFFFFFFFFFFFFFFFFFFFFFFFFFFFFED
:1043E000FFFFFFFFFFFFFFFFFFFFFFFFFFFFFFFFDD
:1043F000FFFFFFFFFFFFFFFFFFFFFFFFFFFFFFFFCD
:10440000FFFFFFFFFFFFFFFFFF01060D00FE090199
:104410006602D620FFFE0BFE0AFE0D00602219691F
:10442000808080808080800080183363A0A0A003FB
:1044300057675050F850F850500259692078A0A0A2
:10444000702828F02002596948A85010204050A830
:104450009002586840A0A040A098906828136380FC
:104460008080113B6B2040408080808080404020D5
:10447000113B6B804040202020202040408006558A
:104480006520A870A8200455652020F8202011334D
:1044900063604080065161F811336340E040025987
:1044A0006908081010204040808002596920508817
:1044B0008888888850200259692060A02020202008
:1044C00020F80259697088880810204080F8025945
:1044D00069F80810207008088870025969101030B7
:1044E000505090F81010025969F88080B0C8080840
:1044F000887002596970888080F0888888700259B5
:1045000069F80810102020404040025969708888DE
:104510008870888888700259697088888878080847
:10452000887011386840E040000040E04011386871
:1045300040E040000060408002596908102040803F
:1045400040201008045464F80000F80259698040C3
:1045500020100810204080025969708888081020B7
:1045600020002002596970888898A8A8B080780235
:1045700059692050888888F8888888025969F048E5
:10458000484870484848F0025969708880808080A7
:10459000808870025969F048484848484848F00205
:1045A0005969F8808080F0808080F8025969F8802D
:1045B0008080F08080808002596970888080809837
:1045C00088887002596988888888F888888888125D
:1045D0003969E040404040404040E00259693810AD
:1045E00010101010109060025969888890A0C0A027
:1045F0009088880259698080808080808080F8025D
:1046000059698888D8A8A88888888802596988C87C
:10461000C8A8A89898888802596970888888888866
:10462000888870025969F0888888F08080808001CD
:104630005A6A70888888888888A87008025969F042
:10464000888888F0A0908888025969708880807076
:1046500008088870025969F8202020202020202096
:10466000025969888888888888888870025969888A
:10467000888888505050202002596988888888A8E6
:10468000A8A8A8500259698888505020505088889E
:10469000025969888850502020202020025969F84A
:1046A00008101020404080F8113B6BE08080808033
:1046B0008080808080E00259698080404020101016
:1046C0000808113B6BE0202020202020202020E043
:1046D000085363205088015161F82A226280400209
:1046E0005666700878889868025969808080F088DA
:1046F000888888F0025666708880808870025969C0
:104700000808087888888888780256667088F88053
:10471000887002596930484040F04040404000589D
:10472000687088888878088870025969808080B0AD
:10473000C8888888881238684000C040404040E0FF
:10474000004A6A10003010101010909060025969F1
:1047500080808090A0C0A09088123969C0404040FD
:1047600040404040E0025666D0A8A8A8A88802565B
:1047700066B0C8888888880256667088888888707D
:10478000005868F0888888F08080800058687888B1
:10479000888878080808025666B0C8808080800241
:1047A00056667088601088700258684040F040403B
:1047B000404830025666888888889868025666881D
:1047C00088885050200256668888A8A8A8500256AB
:1047D0006688502020508800586888888898680823
:1047E0008870025666F810204080F8015B6B182034
:1047F000202020C02020202018221969808080805D
:104800008080808080015B6BC020202020182020C9
:104810002020C008536348A890FFFFFFFFFFFFFF61
:10482000FFFFFFFFFFFFFFFFFFFFFFFFFFFFFFFF98
:10483000FFFFFFFFFFFFFFFFFFFF0D006022196971
:104840008000808080808080800358682070A8A0CD
:10485000A0A8702002596930484040E0404048B06C
:104860000356668870505070880259698888505085
:10487000F820F820202219698080808000808080C4
:1048800080124A6A609080609090601090601A3246
:1048900062A0A00359697088A8D8C8D8A8887004F5
:1048A0005767700878887800F80356662850A0A0EB
:1048B0005028045363F80808163161E00359697001
:1048C00088E8D8D8E8D888700A5161F8174464603D
:1048D0009090600357672020F8202000F807356586
:1048E00040A02040E007356540A04020C02A226259
:1048F00040800058688888888898E88080025969D4
:1049000078E8E8E8E868282828262161C0202262A3
:10491000408007356540C04040E004576770888894
:10492000887000F8035666A050282850A0025A6AE2
:1049300040C04040E00818283808025A6A40C04089
:1049400040E01028081038025A6A40A04020A048D1
:104950001828380802596920002020408088887073
:10496000025A6A40200020508888F88888025A6AD3
:1049700010200020508888F88888025A6A30480041
:1049800020508888F88888025A6A28500020508869
:1049900088F88888025A6A50500020508888F88821
:1049A00088025A6A20502020508888F88888025946
:1049B0006958A0A0A0B0E0A0A0B8005B6B70888090
:1049C0008080808088702040025A6A402000F880F1
:1049D00080F08080F8025A6A102000F88080F08011
:1049E00080F8025A6A304800F88080F08080F8022F
:1049F0005A6A505000F88080F08080F8123A6A803D
:104A00004000E04040404040E0123A6A204000E070
:104A10004040404040E0124A6A609000E040404020
:104A20004040E0123A6AA0A000E04040404040E030
:104A3000025969F0484848E8484848F0025A6A284C
:104A400050008888C8A8988888025A6A4020007058
:104A5000888888888870025A6A1020007088888840
:104A6000888870025A6A3048007088888888887000
:104A7000025A6A28500070888888888870025A6AAA
:104A80005050007088888888887003556588502049
:104A90005088015B6B08709898A8A8A8C8C8708057
:104AA000025A6A40200088888888888870025A6A7A
:104AB00010200088888888888870025A6A304800E8
:104AC00088888888888870025A6A50500088888848
:104AD00088888870025A6A10200088885020202018
:104AE0002002596980F0888888F0808080025969A6
:104AF000609090A0A0908888B00259694020007012
:104B00000878889868025969102000700878889899
:104B100068025969304800700878889868025969B5
:104B200028500070087888986802596950500070C1
:104B30000878889868025A6A304830007008788887
:104B40009868025666702870A0A85000586870884F
:104B50008080887020400259694020007088F88069
:104B600088700259691020007088F8808870025996
:104B7000693048007088F880887002596950500088
:104B80007088F8808870123969804000C0404040C9
:104B900040E0123969204000C040404040E01249E6
:104BA00069609000C040404040E0123969A0A00018
:104BB000C040404040E0025A6A502060107088882F
:104BC000888870025969285000B0C888888888028F
:104BD00059694020007088888888700259691020BF
:104BE0000070888888887002596930480070888809
:104BF00088887002596928500070888888887002F7
:104C00005969505000708888888870035767202041
:104C100000F8002020015868087098A8A8C8708083
:104C2000025969402000888888889868025969106C
:104C300020008888888898680259693048008888E8
:104C400088889868025969505000888888889868D0
:104C5000005B6B1020008888889868088870005A6C
:104C60006A8080B0C88888C8B08080005B6B505074
:104C700000888888986808887000060C00FE070283
:104C80002603BC017FFE08FE08FE0508080600009A
:104C900040F0C88888987810050808060000C0F819
:104CA0008888888888F80505050600012030F830D6
:104CB000200508080600002070F820202020E005CC
:104CC00009090600FF2070A8A8B88888702005068A
:104CD00006060001E08CEA8C8A0A0509090600FF35
:104CE000F8A88888888888A8F8050A0A0600FE209F
:104CF0005050505088A8A888700303030600034052
:104D0000A040FFFFFFFFFFFFFFFFFFFFFFFFFFFFD1
:104D1000FFFFFFFFFFFFFFFF0000000605FF010789
:104D20000706020080808080800080030303060164
:104D300005A0A0A005060606000050F85050F85047
:104D40000509090600FF2070A8A07028A87020059A
:104D50000707060000C8C8102040989805070706F6
:104D6000000040A0A040A89068010303060205804F
:104D700080800309090601FF204040808080404078
:104D8000200309090601FF80404020202040408088
:104D900005070706000020A8702070A8200505055B
:104DA0000600012020F820200203030601FFC04076
:104DB00080050101060003F8020202060100C0C0DE
:104DC000050707060000081010204040800507076F
:104DD000060000708898A8C88870030707060100BD
:104DE00040C040404040E0050707060000708808CA
:104DF000102040F8050707060000F8081030088862
:104E00007005070706000010305090F810100507D5
:104E100007060000F880F0080888700507070600FC
:104E200000304080F0888870050707060000F80809
:104E30001010202020050707060000708888708861
:104E400088700507070600007088887808106002DF
:104E50000505060100C0C000C0C00206060601FF2D
:104E6000C0C000C04080030505060101204080400D
:104E700020050303060002F800F8030505060101FA
:104E80008040204080050707060000708810202021
:104E900000200507070600007088B8A8B8807005D4
:104EA0000707060000708888F888888805070706C5
:104EB0000000F04848704848F005070706000070F9
:104EC000888080808870050707060000F048484801
:104ED0004848F0050707060000F88080F08080F859
:104EE000050707060000F88080F08080800507072E
:104EF000060000708880809888700507070600000B
:104F0000888888F8888888030707060100E0404001
:104F1000404040E0050707060000381010101090D0
:104F2000600507070600008890A0C0A090880507CC
:104F300007060000808080808080F8050707060053
:104F40000088D8A888888888050707060000888810
:104F5000C8A8988888050707060000708888888890
:104F60008870050707060000F08888F080808005BB
:104F7000070706000070888888A89068050707065C
:104F80000000F08888F0A0908805070706000070F0
:104F9000888070088870050707060000F820202028
:104FA00020202005070706000088888888888870E8
:104FB00005070706000088888888505020050707E5
:104FC00006000088888888A8A85005070706000002
:104FD0008888502050888805070706000088885078
:104FE00020202020050707060000F8081020408038
:104FF000F80309090601FFE080808080808080E05E
:10500000050707060000804040201010080309092A
:105010000601FFE020202020202020E005030306D9
:1050200000052050880501010600FEF80303030671
:105030000105804020050505060000700878887885
:105040000507070600008080F0888888F0050505C0
:1050500006000070808088700507070600000808B9
:1050600078888888780505050600007088F08070CB
:10507000050707060000304840E0404040050707AC
:105080000600FE708888887808700507070600000B
:105090008080F0888888880307070601004000C0E8
:1050A000404040E00409090601FE100030101010D5
:1050B00010906005070706000080808890E09088C7
:1050C000030707060100C04040404040E0050505D9
:1050D000060000D0A8A8A8A8050505060000B0C8CD
:1050E000888888050505060000708888887005078F
:1050F000070600FEF0888888F08080050707060014
:10510000FE78888888780808050505060000B0C87C
:1051100080808005050506000078807008F005078E
:10512000070600002020F8202020180505050600AD
:1051300000888888986805050506000088888850DA
:10514000200505050600008888A8A8500505050665
:10515000000088502050880507070600FE888888D0
:1051600050204080050505060000F8102040F80397
:1051700009090601FF2040404080404040200109CD
:10518000090602FF8080808080808080800309097A
:105190000601FF8040404020404040800503030658
:1051A000000248A890FFEE01B20111241FBECFEF0C
:1051B000D1E2DEBFCDBF00E00CBF14E0A0E0B2E062
:1051C000E8E5F2E902E00BBF02C007900D92A830BB
:1051D000B107D9F728E1A8E0B4E001C01D92A035DD
:1051E000B207E1F718E2C4EDD8E200E006C021976B
:1051F0000109802FFE010F949548C33DD10780E03F
:105200000807A9F70F9416350D941A490C9400005D
:10521000CF93DF93EC01CB01BA010F94FF400F94C1
:10522000C2466883DF91CF910895CF93DF93EC015D
:10523000CB01BA010F94FF400F94C2466883DF91FF
:10524000CF9108958091B0149091B114891B8F7003
:1052500071F49091A11692FB882780F992FD08C005
:1052600081E09091A107913019F080E0089581E0EC
:105270000895CF93DF93EC01CB01BA010F94FF4067
:1052800020E030E048EC51E40F945E410F94C246B8
:10529000688379838A839B83DF91CF910895CF932D
:1052A000DF93EC01CB01BA010F94FF4020E030E026
:1052B00048EC52E40F945E410F94C24668837983B0
:1052C0008A839B83DF91CF910895CF93DF93EC0185
:1052D000CB01BA010F94FF402AE037ED43E25CE3D3
:1052E0000F945E41688379838A839B83DF91CF919A
:1052F0000895CF93DF93EC01CB01BA010F94FF40E7
:105300002AE037ED43E25CE30F945E4168837983E2
:105310008A839B83DF91CF910895CF93DF93EC0134
:10532000CB01BA010F94FF402DEC3CEC4CEC5DE35B
:105330000F945E41688379838A839B83DF91CF9149
:105340000895CF93DF93EC01CB01BA010F94FF4096
:1053500020E030E048EC51E40F945E4168837983AB
:105360008A839B83DF91CF910895CF93DF93EC01E4
:10537000CB01BA010F94FF4020E030E048EC52E44A
:105380000F945E41688379838A839B83DF91CF91F9
:105390000895CF93DF93EC01CB01BA010F94FF4046
:1053A0002FE632E143E85AE30F945E416883798344
:1053B0008A839B83DF91CF910895CF93DF93EC0194
:1053C000CB01BA010F94FF40688379838A839B8362
:1053D000DF91CF910895CF93DF93EC01CB01BA0118
:1053E0000F94FF400F94BB4679836883DF91CF9180
:1053F0000895811118C08FEF90914307890F837032
:1054000080934307E0914207EF5FE0934207F0E0AB
:10541000EE0FFF1FE252F94F809147078083809182
:1054200045078183089581E0E7CFCF92DF92EF9225
:10543000FF921F93CF93DF931091CC06CCE9D6E077
:10544000E0E090E0F0E080E049919F5F4111192F8A
:10545000842B30E020E050E070E060E06A017B01E6
:10546000022E04C0F694E794D794C7940A94D2F716
:10547000C0FE08C0AF2FB0E0A156B94FFE2EF22AF1
:10548000FC92FF5F2F5F3F4F2530310539F7E05F1A
:105490009330D1F61093CC0650E040E020E090E04D
:1054A000B0E0A0E06C017D01042E04C0F694E79406
:1054B000D794C7940A94D2F7C0FC05C02E504F5F12
:1054C0005F4F2A3B79F72093CF062AE335E0422F3E
:1054D0003150203811F1225F6C017D01032E04C090
:1054E000F694E794D794C7940A94D2F7C0FEEFCF0E
:1054F0004093CE068091D306823039F48091D00655
:10550000181674F484E08093D006DF91CF911F9138
:10551000FF90EF90DF90CF9008952093CE06EACFD2
:105520008CEFF1CF80918A07882319F082E0809375
:105530009B0684E080936F028091570B882349F08B
:1055400090919B068FEF890F80939B0681E019163F
:105550000CF080E0089580E095E290938B068093B4
:105560008A068CE491E0909389068093880680EC0B
:105570009EEF90938D0680938C0690919A0680E220
:10558000890F863740F080EF890F20E431E03093B7
:105590008D0620938C0610928E0680938F068FEFD7
:1055A000809387060895FC0184910895FC01808111
:1055B00008959091050194709093030100000000FC
:1055C000000087FDC5C0A3980000000091E09A95F7
:1055D0000000E9F790910501909594709093030174
:1055E0000000000000009091050194709093030169
:1055F00000000000000086FDB7C0A3980000000076
:1056000091E09A950000E9F79091050190959470CA
:105610009093030100000000000090910501947038
:105620009093030100000000000085FD9BC0A3983B
:105630000000000091E09A950000E9F790910501C3
:1056400090959470909303010000000000009091E9
:10565000050194709093030100000000000084FD98
:105660007FC0A3980000000091E09A950000E9F740
:1056700090910501909594709093030100000000B3
:1056800000009091050194709093030100000000C8
:10569000000083FD63C0A3980000000091E09A958C
:1056A0000000E9F7909105019095947090930301A3
:1056B0000000000000009091050194709093030198
:1056C00000000000000082FD47C0A3980000000019
:1056D00091E09A950000E9F79091050190959470FA
:1056E0009093030100000000000090910501947068
:1056F0009093030100000000000081FD2BC0A398DF
:105700000000000081E0982F9A950000E9F7909141
:105710000501909594709093030100000000000033
:105720009091050194709093030100000000000027
:10573000A398000000008A950000E9F78091050118
:10574000809584708093030100000000000008959C
:10575000A39A3ACFA39AD4CFA39AB8CFA39A9CCFB7
:10576000A39A80CFA39A64CFA39A48CF089590E0DC
:1057700080E0089590914E09E92FF0E0EE5AFA4E3C
:1057800080839F5F953040F490934E098091320B57
:105790008F5F8093320B089510924E09F7CF8F924E
:1057A0009F92AF92BF92CF92DF92EF92FF92CF93F0
:1057B0004B015C0169017A0124E330E040EF51ECD8
:1057C000C701B6010F94AF4787FD48C023E030E022
:1057D0004AE953E4C701B6010F94F84018160CF4D7
:1057E0003DC02AE130E04CE552ECC501B4010F9414
:1057F000AF4787FD33C023E030E041E953E4C50102
:10580000B4010F94F84018164CF129E630E040E25C
:1058100051ECC501B4010F94AF4787FD1FC023E0D1
:1058200030E040E953E4C501B4010F94F840181684
:10583000ACF029E630E040E151ECC701B6010F942D
:10584000AF4787FD0BC0C1E023E030E841E953E4F6
:10585000C701B6010F94F84018160CF4C0E08C2F65
:10586000CF91FF90EF90DF90CF90BF90AF909F903F
:105870008F900895DC0112964D915D916D917C9110
:105880001597ED91FC914083518362837383089552
:105890009C018CE0EAE7F2E0D90101900D928A9533
:1058A000E1F798E0E6E8F2E0D901A05CBF4F019093
:1058B0000D929A95E1F70895CF92DF92EF92FF92C1
:1058C0000F931F93CF93DF93CDB7DEB72C970FB60F
:1058D000F894DEBF0FBECDBF2CE0EAE7F2E0DE01B8
:1058E000119601900D922A95E1F724E0629F8001C4
:1058F00011247C01E00EF11EC8018D5A9D4F6C01F0
:10590000F70124A935A946A957A9FC016081718135
:10591000828193810F944F45F60160837183828366
:105920009383E1E0F0E0EC0FFD1FE00FF11F8081B9
:105930009181A281B381F70180839183A283B38394
:1059400014AA15AA16AA17AA2C960FB6F894DEBFA9
:105950000FBECDBFDF91CF911F910F91FF90EF90C0
:10596000DF90CF9008952FEB280F2A3108F042C026
:10597000E22FF0E080918F0590919005A091910524
:10598000B091920504C0B695A795979587952A95ED
:10599000D2F780FD02C081700895EB58FA4FE08184
:1059A000EE2329F18091C90B9091CA0BE80FF92FD2
:1059B000F11D808190ED980F9A3030F08E3251F4C5
:1059C000818180538A3098F4F0936505E0936405F3
:1059D00081E008958D3211F08B3249F4818190ED90
:1059E000980F9A3088F38E3211F48281EACFF0E07A
:1059F000E0E0EACF80E008950F94FF400F94BB46AB
:105A0000CB010C94D1E1CF92DF92EF92FF926B0128
:105A10007C0120E030E0A9010F94F84020E030E064
:105A200040E05FE387FF04C020E030E040E05FEB50
:105A3000C701B6010F944F450F94BB46CB01FF90B1
:105A4000EF90DF90CF900C94D1E10F94FF400C9435
:105A5000032D0E94F4E62091810691E0821301C09B
:105A600090E0821380938106892F089563E972E0A4
:105A700084E690E00E944DE66AEB72E084E690E0F6
:105A80000C944DE60F94FF400F94C246862F0C9461
:105A900038E40C9470CECF93DF9300D01F92CDB733
:105AA000DEB70F94FF402DEC3CEC4CEC5DE30F9423
:105AB0005E4169837A838B839C83CE0101960E9429
:105AC00099DE0F900F900F900F90DF91CF91089576
:105AD000CF93DF9300D01F92CDB7DEB70F94FF4076
:105AE0002AE037ED43E25CE30F945E4169837A83F9
:105AF0008B839C83CE0101960E944ADF0F900F900A
:105B00000F900F90DF91CF9108950C9422CECF93F8
:105B1000DF9300D01F92CDB7DEB70F94FF4020E097
:105B200030E048EC51E40F945E4169837A838B83C3
:105B30009C83CE0101960E94E9DF0F900F900F9099
:105B40000F90DF91CF910895CF93DF9300D01F92F4
:105B5000CDB7DEB70F94FF4020E030E048EC52E4D0
:105B60000F945E4169837A838B839C83CE01019677
:105B70000E94E9DF0F900F900F900F90DF91CF916F
:105B80000895CF93DF9300D01F92CDB7DEB70F9467
:105B9000C2460F94FD4069837A838B839C83CE0138
:105BA00001960E94E9DF0F900F900F900F90DF9108
:105BB000CF9108950F94FF4020E030E048EC51E48D
:105BC0000F945E410C94C12D0F94FF4020E030E013
:105BD00048EC52E40F945E410C94C12DCF93DF93B7
:105BE00000D01F92CDB7DEB70F94FF402AE037ED0B
:105BF00043E25CE30F945E4169837A838B839C83E9
:105C0000CE0101960E940CE10F900F900F900F9023
:105C1000DF91CF9108959B011092D9061092D8067A
:105C20008093570B40E060E0C9010F94BD0281E012
:105C300080933614089560E77EE482E00E940B2E84
:105C400088E380939A0683E08093990680E48093AA
:105C50009806E0E9F6E01182108213821282158222
:105C60001482178216820E94AB2A82E190E0909300
:105C70003A148093391408950F94FF400F94C2464C
:105C8000862F0C9406E2CF93DF9300D01F92CDB7FE
:105C9000DEB769837A838B839C83CE0101960F9450
:105CA000D91D0F900F900F900F90DF91CF91089515
:105CB0000F94FF402FE632E143E85AE30F945E4130
:105CC0000C94432E1F93CF93DF9368E170E080E044
:105CD00090E00F944F226093DB066AE070E080E072
:105CE00090E00F944F226093DA06109142072091C2
:105CF000DB06A22F022E000CBB0BEEEDF6E030E02F
:105D0000C62F062E000CDD0B1317B9F1808192818E
:105D100089131BC0482F082E000C550B4150510908
:105D2000A417B50711F082130DC083819181482F0C
:105D300098170CF4492F64172CF089170CF4892F4D
:105D400086171CF63F5F3296DFCF7181472F072EF3
:105D5000000C550B41505109C417D50711F06713BA
:105D6000F1CF482F98170CF4492F24175CF38917AB
:105D70000CF4892F821734F3A8CFDF91CF911F91B4
:105D80000895CF9364E078E481E00E940B2E80E0D8
:105D900091E0909347078093460780E095E09093C9
:105DA0004507809344071092430710924207EEED97
:105DB000F6E01082C5E0C18381E00E94F929C0931A
:105DC000DD0610923A14109239141092DC06CF912D
:105DD0000C94622EAF92BF92CF92DF92EF92FF921D
:105DE0000F931F93CF93DF936B01E9014A3009F4BE
:105DF000B8C0453109F06AC0DB011296ED91FC9103
:105E0000F280C681D781A49A88E28A950000E9F7DA
:105E1000BF2CB29420EFB22230E1A32EAF0C48E2A7
:105E2000E42E88EF0E94D92A8E2D8A950000E9F78A
:105E3000BFE1BF1508F481C08F2D807780680E9474
:105E4000D92A8B2D0E94D92A8E2D8A950000E9F738
:105E500080E80E94D92A80E00E94D92A8E2D8A9556
:105E60000000E9F78AEF0E94D92A8E2D8A9500005A
:105E7000E9F78E01005F1F4F8881807F0E94D92A39
:105E800089918295807F0E94D92AC017D107A1F7F6
:105E90008E2D8A950000E9F7F394E0E1BE0EFA102A
:105EA000C0CFA498D6011296CD91DC91CE010F946B
:105EB000BF2681112CC2DF91CF911F910F91FF90CE
:105EC000EF90DF90CF90BF90AF900895FB010281DB
:105ED0001381423309F4D6C108F4DAC1463409F417
:105EE000C7C1473409F4CAC14B3329F589812B81D5
:105EF000D80112967C91129713963C91213009F4A7
:105F00001DC2233009F0E7C148EF480F582F91E038
:105F1000341708F490E031E0541708F030E0492FCE
:105F2000432B61E0571708F460E0462309F0FBC1FA
:105F3000932309F0F8C181E0BECF80EE8F0D806819
:105F4000807F0E94D92A8F2D8295807F0E94D92A36
:105F50008E2D8A950000E9F780E80E94D92A80E812
:105F60007BCF9C9AA4989B9AA3988091040184600B
:105F700080930401809105018095847080930301D2
:105F8000A49A88E28A950000E9F788E790E0CEE9D4
:105F9000DFE0FE013197F1F70197D9F788EF0E9412
:105FA000D92A18E2812F8A950000E9F780E20E9441
:105FB000D92A80E00E94D92A812F8A950000E9F72A
:105FC00080E00E94D92A80E80E94D92A812F8A95F0
:105FD0000000E9F780E00E94D92A80E10E94D92AD6
:105FE000812F8A950000E9F7CE010197F1F7CE01E4
:105FF0000197F1F7CE010197F1F7CE010197F1F783
:10600000CE010197F1F7CE010197F1F7CE0101978B
:10601000F1F7CE010197F1F7CE010197F1F7CE012B
:106020000197F1F7CE010197F1F7CE010197F1F752
:10603000CE010197F1F7CE010197F1F72197F1F722
:1060400080E20E94D92A80E40E94D92A812F8A9571
:106050000000E9F780E20E94D92A80E60E94D92A4E
:106060001A950000E9F7F12C00E018E2C1E0802F5A
:10607000807780680E94D92A8F2D0E94D92A812F8B
:106080008A950000E9F780E80E94D92A80E00E9402
:10609000D92A812F8A950000E9F78AEF0E94D92A30
:1060A000812F8A950000E9F7D0E280E00E94D92A8A
:1060B00080910501847080930301000000000000BE
:1060C000A398000000008C2F8A950000E9F78091CA
:1060D000050180958470809303010000000000009A
:1060E000809105018470809303010000000000008E
:1060F000A398000000008C2F8A950000E9F780919A
:106100000501809584708093030100000000000069
:10611000809105018470809303010000000000005D
:10612000A398000000008C2F8A950000E9F7809169
:106130000501809584708093030100000000000039
:10614000809105018470809303010000000000002D
:10615000A398000000008C2F8A950000E9F7809139
:106160000501809584708093030100000000000009
:1061700080910501847080930301000000000000FD
:10618000A398000000008C2F8A950000E9F7809109
:1061900005018095847080930301000000000000D9
:1061A00080910501847080930301000000000000CD
:1061B000A398000000008C2F8A950000E9F78091D9
:1061C00005018095847080930301000000000000A9
:1061D000809105018470809303010000000000009D
:1061E000A398000000008C2F8A950000E9F78091A9
:1061F0000501809584708093030100000000000079
:10620000809105018470809303010000000000006C
:10621000A398000000008C2F8A950000E9F7809178
:106220000501809584708093030100000000000048
:10623000812F8A950000E9F7D15009F036CF88EF19
:106240000E94D92A812F8A950000E9F70F5F80E12B
:10625000F80E003209F00BCF80E00E94D92A80ECC2
:106260000E94D92A1A950000E9F7A49881E023CE6C
:10627000D80115968C91888381E01DCEF80181812B
:106280008883FACFB901C8010F94A92681E013CE03
:10629000443171F0473109F04ECE1882F801828105
:1062A0008983858181508A8383818B8381E003CEBA
:1062B000D80115964C91159750E0440F551F70E08A
:1062C00060E016968D919C910F94BB48C8010F9485
:1062D000D52681E0F0CD381708F42DCE871708F4C5
:1062E0002ACEFA80E12CD12C243070F41DC0BE01DE
:1062F000C8010F94A926898198819D0D98838E0DE0
:106300008983FF0C09F417CEF7FEF6CFF0CF4D814D
:1063100050E0440F551F70E060E08E819F810F9424
:10632000BB4881E0C8CDFA8030E0F901EA56FD4F64
:10633000D0802E563D4FF901E080E6CF58E0580F4F
:10634000482FE5CDDF92EF92FF920F931F93CF93EB
:10635000DF93EC01D62E1CAD0BAD7C0184E0E80E82
:10636000F11CE98DFA8DC7011995412F480F2D2D8C
:10637000602FC7010F940F2B9BAD890F8BAF81E06E
:1063800090E0DF91CF911F910F91FF90EF90DF9000
:1063900008958F929F92AF92BF92CF92DF92EF9229
:1063A000FF920F931F93CF93DF93EC018B017A0140
:1063B0008A859B858617970731F0888199810F948C
:1063C000DB291B870A87888599850196F9F46A81FC
:1063D0008E81680F97014C81888199810F94A22B3F
:1063E0002E813F81820F932F911D9F838E8390E09A
:1063F00080E0DF91CF911F910F91FF90EF90DF90A0
:10640000CF90BF90AF909F908F900895CE80DF8007
:10641000F701008110E0002309F1A880B980602F06
:10642000C5010F94412AF501118911954701FFEF2C
:106430008F1A9F0AF40181914F01F501882341F0E1
:106440009089190F082F682FC5010F94412AF2CFA8
:10645000003279F083899189890F180FC10ED11C00
:10646000288539852C153D0508F0B1CF81E090E0F5
:10647000C0CF8089F2CFCF92DF92EF92FF926C0172
:10648000990FEE08FF084AE0C701B601F7FE0DC0FC
:106490006DE284E195E10E94A23166277727CB0166
:1064A0006C197D098E099F094AE0FF90EF90DF90FB
:1064B000CF900D94811CCF92DF92EF92FF920F93B9
:1064C0001F93CF9390910602913009F461C0662327
:1064D00051F01092540410925004109251041092F2
:1064E000520410925304C82F0F949924C090500462
:1064F000D0905104E0905204F09053049B01AC0101
:106500002C193D094E095F0969017A01F7FC40C069
:1065100020915404C7FD15C04C2F0C2E000C550BB8
:106520004C5F5F4FE22F022E000CFF0B4E175F07F0
:106530007CF144EFC42EDD24D394E12CF12C2C17F4
:1065400034F438EEC32E33E0D32EE12CF12CC60EFA
:10655000D71EE81EF91EC0925004D0925104E0925A
:106560005204F0925304022F017010E084E2809FE5
:10657000B001819F700D701B112460597C4F82E324
:1065800090E00E944DE6809154048F5F8093540404
:10659000CF911F910F91FF90EF90DF90CF900895D2
:1065A0008091640590916505009731F04AE050E0D4
:1065B00070E060E00D94F73D60E070E0CB0108957D
:1065C0000E94D032CB010895CF92DF92EF92FF92DA
:1065D0000F931F93CF93DF938B01C3E5D2E02091FC
:1065E0006702309168024091690250916A02FC0191
:1065F00060817181828193810F9449462C853D850C
:106600004E855F850F944F456C877D878E879F876A
:10661000C12CD12C76012FE532E04BE552E067E545
:1066200072E0CE010F949517DF91CF911F910F91DA
:10663000FF90EF90DF90CF900C9494CE8091640502
:1066400090916505009731F04AE050E070E060E01D
:106650000D94253F60E070E0CB0108950F931F93E8
:10666000CF9380916405909165050097E9F0FC0156
:106670008F01C1912C2F2F7D81F0C53411F0C536CB
:10668000B9F7F801108270E060E00F94993CF801CE
:10669000C083CF911F910F91089570E060E0CF917A
:1066A0001F910F910D94993C60E070E0CB01F1CF08
:1066B00080918F05827149F4809191058C7829F43D
:1066C00080919205837009F469C082E40E94B32C22
:1066D000882351F00E941E336093A4137093A51376
:1066E0008093A6139093A71383E50E94B32C88236D
:1066F00051F00E942E336093D4137093D51380937E
:10670000D6139093D71384E50E94B32C882351F0BD
:106710000E942E336093D8137093D9138093DA13A9
:106720009093DB1388E50E94B32C882351F00E94DC
:106730002E336093ED0B7093EE0B8093EF0B9093E1
:10674000F00B89E50E94B32C882351F00E942E3370
:106750006093F10B7093F20B8093F30B9093F40B17
:106760008AE50E94B32C882351F00E942E33609357
:10677000F50B7093F60B8093F70B9093F80B85E471
:106780000E94B32C882351F00E942E336093F90BA2
:106790007093FA0B8093FB0B9093FC0B08959091F0
:1067A000CB0B9817D1F00E9494CE8091CB0B88230D
:1067B00061F04BE552E067E572E083E592E00E940C
:1067C000CFDB1092CB0B0C945AD581E08093CB0B8E
:1067D00083E592E00E9436DCF6CF0895282F1092D0
:1067E0003E0B8091391490913A148130904820F0FA
:1067F00010923A141092391480918A07882331F04C
:10680000809139148093370B10923414809137148F
:106810001816BCF4082E000C990B821B91092091CC
:10682000370B022E000C330B2817390754F097FF53
:1068300002C090E080E08093370B90933A148093ED
:1068400039148091370B6623A9F090913814891779
:1068500014F48093381420913814022E000C330B5A
:106860002C5F3F4F482F082E000C550B241735077F
:106870001CF48450809338140895E0913514E63068
:1068800000F581E08E0F809335148091391490913A
:106890003A14B0E0A0E0309138142091371448E069
:1068A000E49FF0011124E85BF84F409112155091DC
:1068B00013155183408382839383A483B5833683E6
:1068C00027830895CF93DF93EC010E943D3440E08D
:1068D00060E0CE01DF91CF910D94BD0240E060E019
:1068E0008BE59AEA0D94BD02E0913514EE2379F020
:1068F000E150E093351488E0E89FF0011124E85B53
:10690000F84F47816681808191810D94BD020C947E
:106910006E34BF92CF92DF92EF92FF920F931F934C
:10692000CF93DF9361E081E00E94EE33C091381491
:1069300085E0C82ECC0E15E01C1B04E00C1B83E088
:10694000F82EFC1A82E0E82EEC1A81E0D82EDC1A30
:10695000BC2EB194C11136C08091370B8823E1F071
:1069600080916F02882359F081E09091370B91114B
:1069700080E024E046E35BE16B2D0F94CF1C0E9486
:106980002229D82FDD2309F4A0C084E0CF5FCC12E8
:10699000E1CF809337140CC080913F0B10923F0BD6
:1069A0008823F1F20E947434809134148823C1F258
:1069B000DF91CF911F910F91FF90EF90DF90CF90DB
:1069C000BF900895C13009F041C08091370B8130EC
:1069D00071F180916F02882391F281E09091370BE1
:1069E000913009F080E023E044E25BE16D2D0F94EB
:1069F000CF1C0E942229D82FC33021F68091370B5B
:106A0000833009F448C080916F02882361F081E0EF
:106A10009091370B933009F080E020E246E05BE193
:106A20006F2D0F94CF1CDD2309F465C0AECF80918C
:106A30003F0B10923F0B882361F289EB95E30E9494
:106A4000623480913414882321F2B2CFC23089F6A7
:106A50008091370B823081F080916F02882309F496
:106A60008ECF81E09091370B923009F080E023E0E7
:106A700045E15BE16E2DBBCF80913F0B10923F0B48
:106A8000882351F384E497E60E94623480913414A1
:106A9000882311F38DCF80913F0B10923F0B8823F9
:106AA00009F4B1CF0E94F8D6882341F00E94362D18
:106AB00080913414882309F4A6CF7ACF68EB71E073
:106AC00084E190E00E944DE6F3CFC430E9F5809177
:106AD000370B843091F080916F02882361F081E060
:106AE0009091370B943009F080E020E247EE5AE1B4
:106AF000602F0F94CF1C86E049CF80913F0B1092FE
:106B00003F0B882341F30E948DF9882339F00E94BE
:106B1000362D809134148823F1F24ACF68EB71E06E
:106B200084E190E00E944DE6F4CF80913F0B1092FB
:106B30003F0B882379F00E94C4EE0E94362D80918D
:106B40003414882339F034CFC530A9F68091370B3F
:106B5000853059F380916F02882369F281E090912A
:106B6000370B953009F080E020E245EF5AE1612FC4
:106B7000C0CFBF92CF92DF92EF92FF920F931F93FD
:106B8000CF93DF9361E081E00E94EE33C09138142F
:106B9000DC2E85E0C82ECC0E13E01C1B02E00C1B83
:106BA00081E0F82EFC1ABC2EB19484E0E82EEC1A99
:106BB000C1115EC08091370B882309F441C08091D8
:106BC0006F02882359F081E09091370B911180E09A
:106BD00024E04EE95AE16B2D0F94CF1C0E9422292C
:106BE0008111C0C0D5E0C43009F0BDC08091370B21
:106BF000843009F499C080916F028111A6C0D5E05C
:106C000081E08D0F8C1315C08091370B8C1709F420
:106C1000D1C080916F02882361F06C2F6D1981E0E3
:106C20009091370B9C1380E023E048E65AE10F94E3
:106C3000CF1CCF5FCC11BCCFDE5FD09337140EC01A
:106C400080913F0B10923F0B882309F4B8CF0E942C
:106C5000743480913414882309F4B1CFDF91CF913B
:106C60001F910F91FF90EF90DF90CF90BF9008950C
:106C7000C13019F58091370B813081F080916F021E
:106C8000882309F4ABCF81E09091370B913009F064
:106C900080E023E045E95AE16F2D9ECF80913F0BC4
:106CA00010923F0B882351F381EB98E30E946234EA
:106CB00080913414882311F3D1CFC23009F08BC0F6
:106CC0008091370B823081F080916F02882309F424
:106CD00085CF81E09091370B923009F080E023E07E
:106CE00048E85AE1602F78CF80913F0B10923F0B1C
:106CF000882351F38DE79AE30E9462348091341423
:106D0000882311F3ABCF80913F0B10923F0B882368
:106D100009F469C081E89EE30E94623480913414D2
:106D2000882309F460C09ACF80913F0B10923F0BEB
:106D3000882309F460CF89E390E40E946234809153
:106D40003414882309F457CF89CF81E09091370B11
:106D5000943009F080E023E04AE75AE16E2D0F9469
:106D6000CF1C4DCFD4E0DC134BCF8091370B8D1768
:106D700091F080916F02882309F442CF6C2F6D1936
:106D800081E09091370B9C1380E023E041E75AE1CA
:106D90000F94CF1C35CF80913F0B10923F0B88236F
:106DA00041F383E097E30E94623480913414882396
:106DB00001F354CF80913F0B10923F0B882309F4CD
:106DC00028CF81E891E40E946234809134148823B2
:106DD00009F41FCF43CFC33009F000CF8091370BA8
:106DE000833009F490CF80916F02882309F4F6CEA6
:106DF00081E09091370B933009F080E023E043E885
:106E00005AE1612FE9CE2F923F924F925F926F929B
:106E10007F928F929F92AF92BF92CF92DF92EF922A
:106E2000FF920F931F93CF93DF9300D0CDB7DEB7C0
:106E300061E081E00E94EE33809138148A83282E2D
:106E40008B5F898395E092199B8314E0121983E08C
:106E5000882E382C321802E0021997EDC92E9AE1DB
:106E6000D92E28EDA22E2BE0B22E412C512C32012E
:106E70004A9481E0982E92188A81811140C08091B5
:106E8000370B8823D1F080916F02882361F0622D47
:106E9000619581E09091370B911180E024E042EE02
:106EA0005AE10F94CF1C9A819F5F9A83898189133D
:106EB000E3CF86E0809337140CC080913F0B109293
:106EC0003F0B882301F30E9474348091341488238B
:106ED000D1F20F900F900F90DF91CF911F910F91F2
:106EE000FF90EF90DF90CF90BF90AF909F908F90EA
:106EF0007F906F905F904F903F902F9008959A8170
:106F0000913009F058C08091370B8130B9F08091F1
:106F10006F02882341F2FF24F3948091370B813074
:106F200009F0F12C8091D80B0E9438E49C014CECC4
:106F30005AE1692D8F2D0F94091DB5CF80913F0B1C
:106F400010923F0B882319F30F945B20E090D80B2D
:106F5000F12C0E943D3480926F02D0924E0BC09271
:106F60004D0BB0924C0BA0924B0B1092470B109212
:106F7000480B1092490B10924A0B4092430B5092CF
:106F8000440B6092450B7092460BF0923A14E092DB
:106F9000391481EB94E59093131580931215109298
:106FA000420B1092410B1092400B809134148823B5
:106FB00009F4ADCF8ECF8A81823009F0A9C08091CB
:106FC000370B8230D9F080916F02882309F46BCFA0
:106FD000FF24F3948091370B823009F0F12C6091FB
:106FE000CC0B7091CD0B8091CE0B9091CF0B0E946A
:106FF000432E9C0148EC5AE1602F9CCF80913F0BBF
:1070000010923F0B8823F9F20F945B206CEC7BE02D
:107010008AEC9AE10F94AD1F80913414882399F281
:1070200058CF8091370B8330D9F080916F0288233D
:1070300009F439CFFF24F3948091370B833009F0A2
:10704000F12C6091D00B7091D10B8091D20B90916B
:10705000D30B0E94432E9C0144EC5AE1632D6ACF6E
:1070600080913F0B10923F0B8823F9F20F945B2025
:1070700060ED7BE086EC9AE10F94AD1F80913414B3
:10708000882399F226CF8091370B8430D9F08091F4
:107090006F02882309F407CFFF24F3948091370B04
:1070A000843009F0F12C6091D40B7091D50B809154
:1070B000D60B9091D70B0E94432E9C0140EC5AE1D5
:1070C000612F38CF80913F0B10923F0B8823F9F24C
:1070D0000F945B2064ED7BE082EC9AE10F94AD1F8E
:1070E00080913414882399F2F4CE80913F0B109252
:1070F0003F0B8823D9F00F945B2063E672E086EBA8
:107100009AE10F94AD1F80913414882379F0E1CE79
:107110009A81933009F485CF943009F4B4CF953037
:1071200009F0C1CE8091370B8530F9F280916F0262
:10713000882309F4B8CEFF24F3948091370B85306F
:1071400009F0F12C609163027091640280916502F4
:10715000909166020E94432E9C014CEA5AE16B8199
:10716000E9CE7F928F929F92AF92BF92CF92DF92A1
:10717000EF92FF920F931F93CF93DF9361E081E033
:107180000E94EE33C091381465E0862E8C0ED6E056
:10719000DC1B85E0D82EDC1A84E0C82ECC1A83E0F4
:1071A000B82EBC1A82E0A82EAC1A81E0982E9C1A48
:1071B0007C2E7194C11134C08091370B8823B1F0BB
:1071C00080916F02882359F081E09091370B9111E3
:1071D00080E024E046E259E1672D0F94CF1CCF5F99
:1071E0008C12E8CF87E0809337140CC080913F0B5E
:1071F00010923F0B882321F30E9474348091341441
:107200008823F1F2DF91CF911F910F91FF90EF90C2
:10721000DF90CF90BF90AF909F908F907F90089518
:10722000C130E1F58091370B8130E1F080916F0240
:107230008823A9F211E08091370B813009F010E02A
:107240006091B8137091B9138091BA139091BB13E8
:107250000E94032D9C0148E159E1692D812F0F9473
:10726000091DBDCF80913F0B10923F0B8823F1F297
:107270000F945B20E12C10ECF12E09E714E420E0E0
:1072800030E040E85FE368EB73E18FE199E10F9450
:10729000161F80913414882349F2B4CFC23009F00C
:1072A00002C18091370B8230D1F080916F02882328
:1072B00009F495CF11E08091370B823009F010E08E
:1072C0006091BC137091BD138091BE139091BF1358
:1072D0000E94032D9C014AE059E16A2DBFCF8091A5
:1072E0003F0B10923F0B882301F30F945B20E12C9E
:1072F00010ECF12E09E714E420E030E040E85FE311
:107300006CEB73E181E199E10F94161F80913414C5
:10731000882359F277CF8091370B8330D1F0809159
:107320006F02882309F45BCF11E08091370B833023
:1073300009F010E06091C0137091C1138091C213E5
:107340009091C3130E94032D9C014CEF58E16B2DCB
:1073500085CF80913F0B10923F0B882301F30F9450
:107360005B20E12C10ECF12E09E714E420E030E082
:1073700040E85FE360EC73E183E099E10F94161F4E
:1073800080913414882359F23DCF8091370B84309B
:10739000D1F080916F02882309F421CF11E0809110
:1073A000370B843009F010E06091C4137091C5135D
:1073B0008091C6139091C7130E94032D9C014EEE3D
:1073C00058E16C2D4BCF80913F0B10923F0B8823DF
:1073D00001F30F945B20E12C10ECF12E09E714E48B
:1073E00020E030E040E85FE364EC73E185EF98E192
:1073F0000F94161F80913414882359F203CF809183
:10740000370B8530D1F080916F02882309F4E7CEE5
:1074100011E08091370B853009F010E06091D413B2
:107420007091D5138091D6139091D7130E94032D9C
:107430009C0144EE58E16D2D11CF80913F0B1092CD
:107440003F0B882301F30F945B20E12C10ECF12E0D
:1074500009E714E420E030E0A90164ED73E189EE6E
:1074600098E10F94161F80913414882361F2CACEDC
:1074700080913F0B10923F0B882329F10F945B20E2
:10748000E12C10ECF12E09E714E420E030E0A90132
:1074900068ED73E18AED98E10F94161F8091341422
:1074A000882389F0AFCEC33009F435CFC43009F456
:1074B0006CCFC53009F4A3CFC63009F090CE8091CF
:1074C000370B8630A9F280916F02882309F487CEAA
:1074D00011E08091370B863009F010E06091D813ED
:1074E0007091D9138091DA139091DB130E94032DD0
:1074F0009C0140ED58E16D2FB1CE2F923F924F92FB
:107500005F926F927F928F929F92AF92BF92CF9233
:10751000DF92EF92FF920F931F93CF93DF9300D0F0
:1075200000D0CDB7DEB761E081E00E94EE3310916C
:107530003814012F85E0810F8D83C12CD12C760169
:10754000C39487E0811B8E8386E0282E211A85E074
:10755000382E311A97E7492E9FE0592E612C712C55
:10756000111141C08091370B8823C1F080916F02C7
:10757000882361F0602F619581E09091370B911124
:1075800080E024E042EA59E10F94CF1C1F5F9D8107
:107590009113E6CF88E0809337140CC080913F0BA5
:1075A00010923F0B882311F30E947434809134149D
:1075B0008823E1F226960FB6F894DEBF0FBECDBF4A
:1075C000DF91CF911F910F91FF90EF90DF90CF90BF
:1075D000BF90AF909F908F907F906F905F904F90F3
:1075E0003F902F900895113009F07EC08091370BA5
:1075F000813021F180916F02882341F2BB24B39442
:107600008091370B813009F0B12C8091C813909193
:10761000C913A091CA13B091CB1389839A83AB830A
:10762000BC83CE0101960E94E9DF61E0601B9C01F2
:1076300046E959E18B2D0F94091DA8CF80913F0B8E
:1076400010923F0B8823B1F20F945B202AE037EDB4
:1076500043E25DE36091C8137091C9138091CA132E
:107660009091CB130F945E4120E030E040E85FE35F
:107670000F944E450F94C2464B010E943D3483E067
:1076800080936F028CE999E190934E0B80934D0BA0
:1076900088EC93E190934C0B80934B0BC092470B7B
:1076A000D092480BE092490BF0924A0B4092430B68
:1076B0005092440B6092450B7092460B90923A1494
:1076C0008092391489EC94E59093131580931215E8
:1076D0001092420B1092410B1092400B8091341487
:1076E000882309F487CF66CF123009F0D9C2809180
:1076F000370B823011F180916F02882309F446CF55
:10770000BB24B3948091370B823009F0B12C809167
:10771000CC139091CD13A091CE13B091CF13898348
:107720009A83AB83BC83CE0101960E94E9DF62E0BD
:10773000601B9C0142E859E17DCF80913F0B109284
:107740003F0B8823C1F20F945B202AE037ED43E220
:107750005CE36091CC137091CD138091CE13909126
:10776000CF130F945E4120E030E040E85FE30F94D8
:107770004E450F94C2464B010E943D3483E08093F6
:107780006F028CE899E190934E0B80934D0B8CEC3B
:1077900093E190934C0B80934B0BC092470BD0928C
:1077A000480BE092490BF0924A0B8DED93E0A0E07C
:1077B000B0E08093430B9093440BA093450BB093A0
:1077C000460B90923A14809239148FEC94E5909382
:1077D0001315809312151092420B1092410B1092C8
:1077E000400B80913414882309F485CFE3CE809137
:1077F000370B833011F180916F02882309F4C6CED4
:10780000BB24B3948091370B833009F0B12C809165
:10781000D0139091D113A091D213B091D313898337
:107820009A83AB83BC83CE0101960E94E9DF63E0BB
:10783000601B9C0140E759E1FDCE80913F0B109207
:107840003F0B8823C1F20F945B202AE037ED43E21F
:107850005DE36091D0137091D1138091D213909118
:10786000D3130F945E4120E030E040E85FE30F94D3
:107870004E450F94C2464B010E943D3410936F0257
:1078800089E799E190934E0B80934D0B80ED93E146
:1078900090934C0B80934B0BC092470BD092480BAC
:1078A000E092490BF0924A0B4092430B5092440BEA
:1078B0006092450B7092460B90923A148092391464
:1078C00089EC94E590931315809312151092420B56
:1078D0001092410B1092400B80913414882309F4CC
:1078E0008ACF68CE8091370B8430F1F080916F029F
:1078F000882309F44BCEBB24B3948091370B84309A
:1079000009F0B12C609194137091951380919613A6
:10791000909197130F94FD400E94C12D64E0601B6D
:107920009C0142E659E186CE80913F0B10923F0BBD
:107930008823E1F20F945B2060919413709195136A
:1079400080919613909197130F94FD402AE037EDA4
:1079500043E25DE30F945E4120E030E040E850E414
:107960000F944E450F94C2464B010E943D3483E074
:1079700080936F0289E699E190934E0B80934D0BB3
:1079800084E993E190934C0B80934B0B84E090E05F
:10799000A0E0B0E08093470B9093480BA093490B75
:1079A000B0934A0B84E79FE0A0E0B0E08093430BE4
:1079B0009093440BA093450BB093460B90923A14CE
:1079C0008092391483EC94E59093131580931215EB
:1079D00085E89DE29093420B8093410B1092400BFF
:1079E00080913414882309F481CFE4CD8091370B42
:1079F0008530E9F080916F02882309F4C7CDBB245C
:107A0000B3948091370B853009F0B12C60919813B5
:107A10007091991380919A1390919B130F94FD404C
:107A20000E94C12D9C0144E559E1632D03CE809154
:107A30003F0B10923F0B8823E9F20F945B2060917B
:107A400098137091991380919A1390919B130F94AE
:107A5000FD402AE037ED43E25DE30F945E4120E014
:107A600030E040E850E40F944E450F94C2464B017D
:107A70000E943D3483E080936F028BE599E19093FF
:107A80004E0B80934D0B88E993E190934C0B8093C0
:107A90004B0B84E090E0A0E0B0E08093470B909324
:107AA000480BA093490BB0934A0B84E79FE0A0E0FA
:107AB000B0E08093430B9093440BA093450BB0939D
:107AC000460B90923A148092391483EC94E590938B
:107AD00013158093121585E89DE29093420B8093D5
:107AE000410B1092400B80913414882309F482CF0B
:107AF00061CD8091370B8630E9F080916F02882349
:107B000009F444CDBB24B3948091370B863009F03F
:107B1000B12C60919C1370919D1380919E13909154
:107B20009F130F94FD400E94C12D9C0146E459E132
:107B3000622D80CD80913F0B10923F0B8823E9F29C
:107B40000F945B2060919C1370919D1380919E1304
:107B500090919F130F94FD402AE037ED43E25DE3DF
:107B60000F945E410F94C2464B010E943D3483E066
:107B700080936F028DE499E190934E0B80934D0BAF
:107B80008CE993E190934C0B80934B0B1092470B35
:107B90001092480B1092490B10924A0B88E79FE015
:107BA000A0E0B0E08093430B9093440BA093450B6F
:107BB000B093460B90923A148092391483EC94E57A
:107BC000909313158093121585E89DE29093420BD4
:107BD0008093410B1092400B80913414882309F458
:107BE0008CCFE8CC80913F0B10923F0B882309F497
:107BF0006BC00F945B206091A0137091A1138091D2
:107C0000A2139091A3130F94FD402AE037ED43E2B5
:107C10005CE30F945E4120E030E040E85FE30F94C6
:107C20004E450F94C2464B010E943D3483E0809341
:107C30006F028FE399E190934E0B80934D0B80EA96
:107C400093E190934C0B80934B0BC092470BD092D7
:107C5000480BE092490BF0924A0B8DED93E0A0E0C7
:107C6000B0E08093430B9093440BA093450BB093EB
:107C7000460B90923A14809239148DEB94E59093D0
:107C800013158093121585E89DE29093420B809323
:107C9000410B1092400B809134148823A9F08ACCB8
:107CA000133009F4A4CD143009F41CCE153009F4B6
:107CB0009DCE163009F41DCF173009F067CC8091A6
:107CC000370B873009F48ECF80916F02882309F437
:107CD0005DCCBB24B3948091370B873009F0B12C75
:107CE0006091A0137091A1138091A2139091A3139E
:107CF0000F94FD400E94C12D9C0148E359E16E8123
:107D000099CC2F923F924F925F926F927F928F9277
:107D10009F92AF92BF92CF92DF92EF92FF920F931A
:107D20001F93CF93DF9300D000D000D01F921F92FB
:107D3000CDB7DEB761E081E00E94EE33D090381419
:107D4000DE8285E08D0D8D8384E08D198B873AE08E
:107D5000832E912CA12CB12C45EF442E4FE7542EAD
:107D6000612C712C83E0282E2D1882E0382E3D18CE
:107D700081E0C82ECD18D11041C08091370B8823E7
:107D8000C1F080916F02882361F06E81619581E07E
:107D90009091370B911180E024E044EF59E10F946A
:107DA000CF1CD3949D819D11E6CF85E0809337143D
:107DB0000CC080913F0B10923F0B882311F30E945F
:107DC0007434809134148823E1F22B960FB6F89422
:107DD000DEBF0FBECDBFDF91CF911F910F91FF90FE
:107DE000EF90DF90CF90BF90AF909F908F907F905B
:107DF0006F905F904F903F902F90089591E0D9122F
:107E00003CC08091370B8130E1F080916F02882374
:107E100041F211E08091370B813009F010E0609160
:107E2000ED0B7091EE0B8091EF0B9091F00B0E9497
:107E3000032D9C0144EE59E16C2D812F0F94091DF7
:107E4000B0CF80913F0B10923F0B8823F1F20F943B
:107E50005B20E12C10E8F12E07E714E420E030E08D
:107E600040E85FE36DEE7BE08CEE99E10F94161F26
:107E700080913414882349F2A8CF82E0D812D4C06C
:107E80008091370B8230D1F080916F02882309F402
:107E900088CF11E08091370B823009F010E06091BB
:107EA000F10B7091F20B8091F30B9091F40B0E9407
:107EB000032D9C0144ED59E1632DBFCF80913F0B11
:107EC00010923F0B882301F30F945B20E12C10E804
:107ED000F12E07E714E420E030E040E85FE361EFD3
:107EE0007BE08CED99E10F94161F80913414882368
:107EF00059F26BCF8091370B833001F180916F0283
:107F0000882309F44ECF11E08091370B833009F0BC
:107F100010E08091F50B9091F60BA091F70BB091CA
:107F2000F80B89839A83AB83BC83CE0101960E94B0
:107F30004ADF9C0144EC59E1622D7FCF80913F0BD9
:107F400010923F0B8823D1F20F945B2020E030E0A9
:107F500048EC52E46091F50B7091F60B8091F70BB1
:107F60009091F80B0F945E4120E030E040E251E444
:107F70000F944E450F94C2466F83788789879A87FE
:107F80000E943D34D0926F028CEC99E190934E0B9D
:107F900080934D0B85EF9BE090934C0B80934B0BA4
:107FA0008092470B9092480BA092490BB0924A0BDB
:107FB0004092430B5092440B6092450B7092460BDB
:107FC0008F81988590933A148093391487EB94E5C8
:107FD00090931315809312151092420B1092410B3F
:107FE0001092400B80913414882309F487CFEDCE92
:107FF00080913F0B10923F0B882309F10F945B2077
:10800000E12C10E8F12E07E714E420E030E040E82E
:108010005FE369EF7BE08CEB99E10F94161F809191
:108020003414882361F0D1CE83E0D81609F462CFEE
:1080300094E0D912B6CE8091370B8430C9F280918A
:108040006F02882309F4ADCE11E08091370B8430A4
:1080500009F010E06091F90B7091FA0B8091FB0B25
:108060009091FC0B0E94032D9C0144EB59E16B8520
:10807000E4CEAF92BF92CF92DF92EF92FF920F9336
:108080001F93CF93DF9300D01F92CDB7DEB761E08F
:1080900081E00E94EE331091381485E0B82EB10EC5
:1080A00004E0011B83E0F82EF11A82E0E82EE11AC9
:1080B00081E0D82ED11AA12EA194111135C0809142
:1080C000370B8823B1F080916F02882359F081E04B
:1080D0009091370B911180E024E046E55AE16A2D3A
:1080E0000F94CF1C1F5FB112E8CF85E08093371447
:1080F0000CC080913F0B10923F0B882321F30E940C
:108100007434809134148823F1F20F900F900F9003
:108110000F90DF91CF911F910F91FF90EF90DF9023
:10812000CF90BF90AF9008951130D1F58091370B6B
:10813000813019F180916F028823A1F2CC24C3947D
:108140008091370B813009F0C12C8091A813909158
:10815000A913A091AA13B091AB1389839A83AB831F
:10816000BC83CE0101960E9499DE9C0142E45AE153
:108170006D2D8C2D0F94091DB5CF80913F0B109262
:108180003F0B8823B9F20F945B2068EA73E18CE41B
:108190009AE10F94FE1F80913414882359F2B5CFD1
:1081A000123009F083C08091370B823009F1809141
:1081B0006F02882309F496CFCC24C3948091370BA7
:1081C000823009F0C12C8091AC139091AD13A09135
:1081D000AE13B091AF1389839A83AB83BC83CE0176
:1081E00001960E9499DE9C014EE25AE16E2DC1CFAC
:1081F00080913F0B10923F0B8823C9F20F945B20B4
:108200006CEA73E188E39AE10F94FE1F80913414C5
:10821000882369F27ACF8091370B833009F18091FE
:108220006F02882309F45ECFCC24C3948091370B6E
:10823000833009F0C12C8091B0139091B113A091BB
:10824000B213B091B31389839A83AB83BC83CE01FD
:1082500001960E9499DE9C014AE15AE16F2D89CF77
:1082600080913F0B10923F0B8823C9F20F945B2043
:1082700060EB73E184E29AE10F94FE1F8091341465
:10828000882369F242CF80913F0B10923F0B8823E5
:10829000B9F00F945B2064EB73E180E19AE10F94F5
:1082A000FE1F80913414882359F02FCF133009F426
:1082B000B2CF143009F016CF8091370B843019F308
:1082C00080916F02882309F40DCFCC24C394809150
:1082D000370B843009F0C12C8091B4139091B51301
:1082E000A091B613B091B71389839A83AB83BC83F3
:1082F000CE0101960E9499DE9C0146E05AE1602F72
:1083000038CF2F923F924F925F926F927F928F92CF
:108310009F92AF92BF92CF92DF92EF92FF920F9314
:108320001F93CF93DF93CDB7DEB72C970FB6F8949A
:10833000DEBF0FBECDBF61E081E00E94EE33D09082
:10834000381485E08D0D8D8393E09D199A8782E026
:108350008D198B8722E1222E2CE0322E34EBA32EB6
:1083600038E1B32E44244A944FE7542E612C712CEB
:1083700055ED852E54E5952E81E08D198C87CD2CF9
:10838000C194D11040C08091370B8823B9F08091FF
:108390006F02882359F081E09091370B911180E0B2
:1083A00024E04EEB58E16C2D0F94CF1CD3948D81BB
:1083B000D812E7CF84E0809337140CC080913F0B34
:1083C00010923F0B882319F30E9474348091341467
:1083D0008823E9F22C960FB6F894DEBF0FBECDBF0E
:1083E000DF91CF911F910F91FF90EF90DF90CF9091
:1083F000BF90AF909F908F907F906F905F904F90C5
:108400003F902F90089581E0D81273C08091370B70
:10841000813011F180916F02882341F211E0809147
:10842000370B813009F010E08091120C9091130C01
:10843000A091140CB091150C89839A83AB83BC83F3
:10844000CE0101960E940CE19C014AEA58E16C853C
:10845000812F0F94091DAACF80913F0B10923F0BE3
:108460008823C1F220E030E048EC52E46091120C25
:108470007091130C8091140C9091150C0F945E4127
:108480000F94C2466E837F83888799870E943D340C
:1084900093E090936F02B0924E0BA0924D0B3092EE
:1084A0004C0B20924B0B1092470B1092480B1092E2
:1084B000490B10924A0B4092430B5092440B60922E
:1084C000450B7092460B8E819F8190933A14809356
:1084D000391490921315809212151092420B10923B
:1084E000410B1092400B80913414882309F492CFF1
:1084F00071CF92E0D91252C08091370B8230D1F007
:1085000080916F02882309F451CF11E08091370BDD
:10851000823009F010E060918F0770919007809190
:108520009107909192070E94032D9C0146E958E122
:108530006B858ECF80913F0B10923F0B882301F308
:108540000F945B20E12CF12C08E413E420E030E0F0
:10855000A9016FE877E080EA98E10F94161F8091F7
:108560003414882369F236CF80913F0B10923F0B71
:108570008823D9F00F945B20E12CF12C08E413E45C
:1085800020E030E0A90163E977E08EE898E10F94FC
:10859000161F80913414882341F01CCF93E0D91228
:1085A00005CF8091370B8330F9F280916F028823D9
:1085B00009F4FCCE11E08091370B833009F010E014
:1085C0006091930770919407809195079091960719
:1085D0000E94032D9C0146E858E16A8539CFEEEAF6
:1085E000F6E01282339686E0EC3CF807D1F7089566
:1085F0001092D1068AE08093CD0683E08093D00666
:108600008FE08093D306ECE9F6E08FE180838183ED
:1086100082830E94152A0C94EF4268E77AE484E191
:108620000E940B2E83E080935B0B8AE08093D70639
:1086300010925A0B0E94F84210925F0B10923A145B
:10864000109239140895109236140C947434AF9229
:10865000BF92CF92DF92EF92FF920F931F93CF932F
:10866000DF93EC015B018A01FB01199587FD16C0C0
:10867000C82ED12CF12CE12C2196F801C082D18298
:10868000E282F382CE01DF91CF911F910F91FF9093
:10869000EF90DF90CF90BF90AF900895982F907E8D
:1086A000903CA9F48F7190E0B0E0A0E06C017D01F6
:1086B00026E0CC0CDD1CEE1CFF1C2A95D1F7CE0168
:1086C0000196F50119958F73C82A2296D6CF982F57
:1086D000907F903E11F58F7090E0B0E0A0E06C01CB
:1086E0007D0186E0CC0CDD1CEE1CFF1C8A95D1F7C9
:1086F000CE010196F50119958F73C82A96E0CC0C2E
:10870000DD1CEE1CFF1C9A95D1F7CE010296F501F7
:1087100019958F73C82A2396B0CF982F987F903FD2
:1087200079F5877090E0B0E0A0E06C017D01F6E0A3
:10873000CC0CDD1CEE1CFF1CFA95D1F7CE01019686
:10874000F50119958F73C82AA6E0CC0CDD1CEE1C30
:10875000FF1CAA95D1F7CE010296F50119958F73EA
:10876000C82AB6E0CC0CDD1CEE1CFF1CBA95D1F774
:10877000CE010396F50119958F73C82A24967DCFF3
:10878000982F9C7F983FE1F5837090E0B0E0A0E0E7
:108790006C017D0156E0CC0CDD1CEE1CFF1C5A95D3
:1087A000D1F7CE010196F50119958F73C82A66E0BD
:1087B000CC0CDD1CEE1CFF1C6A95D1F7CE01029695
:1087C000F50119958F73C82A76E0CC0CDD1CEE1CE0
:1087D000FF1C7A95D1F7CE010396F50119958F7399
:1087E000C82AE6E0CC0CDD1CEE1CFF1CEA95D1F794
:1087F000CE010496F50119958F73C82A25963DCFB1
:10880000982F9E7F9C3F09F049C0817090E0B0E0B6
:10881000A0E06C017D0186E0CC0CDD1CEE1CFF1C91
:108820008A95D1F7CE010196F50119958F73C82A63
:1088300096E0CC0CDD1CEE1CFF1C9A95D1F7CE0106
:108840000296F50119958F73C82A26E0CC0CDD1C21
:10885000EE1CFF1C2A95D1F7CE010396F501199560
:108860008F73C82A36E0CC0CDD1CEE1CFF1C3A9539
:10887000D1F7CE010496F50119958F73C82A46E009
:10888000CC0CDD1CEE1CFF1C4A95D1F7CE010596E1
:10889000F50119958F73C82A2696EFCE982F907CF4
:1088A000903841F4807C803869F42196CE01F5013E
:1088B0001995F8CF8E7F8D3F28F02196CE01F501D6
:1088C0001995F8CFC12CD12C7601D7CE1F93CF9319
:1088D000DF9300D01F92CDB7DEB710E0AE014F5F3F
:1088E0005F4F63ED7AE20E94274349815A816B8191
:1088F0007C81452B462B472B11F01F5FEFCF812F3B
:108900000F900F900F900F90DF91CF911F910895CE
:108910001F93CF93DF9300D01F92CDB7DEB710E047
:10892000AE014F5F5F4F66ED7AE20E9427434981B7
:108930005A816B817C81452B462B472B11F01F5FA1
:10894000EFCF812F0F900F900F900F90DF91CF916D
:108950001F910895CF93C82F807F0E94D92A8C2F12
:108960008295807F0E94D92A88E28A950000E9F7E3
:10897000CF910895CF93DF93EC01FE01849121966E
:10898000882319F00E94AA44F8CFDF91CF9108956F
:108990000F931F93CF93C62F8C01F80181918F0104
:1089A000882331F0CC2321F00E94AA44C150F5CF96
:1089B000CF911F910F910895CF93DF93EC0189918F
:1089C000882319F00E94AA44FACFDF91CF9108952D
:1089D0000F934CE0849F402D112421E0240F20931D
:1089E0007F078CE0840F8093B10B90E0029630916A
:1089F0004C153817190621F01CF080E00F910895EE
:108A000080914E152817C8F781E0809338156623AA
:108A100051F04D5F0BE020E860E088E195E10F94B4
:108A2000A028109238158091B10B90914C158917A0
:108A300020F320914E1590917F072917F0F21092A4
:108A40004F158093501581E0D9CFEF92FF920F938D
:108A500086E7E82E86E1F82E03E127E047E064E2AE
:108A600088E195E10F94CD2B0F94332A25E733E06D
:108A70004BE265E288E195E10F94A22B2FE733E00A
:108A800047E367E088E195E10F91FF90EF900D9447
:108A9000A22BEF92FF920F931F93CF93DF93CDB74B
:108AA000DEB72C970FB6F894DEBF0FBECDBF6F3F79
:108AB00071058105910509F0C0F484E195E10E94FA
:108AC000A231E0911C15F0911D153196849190E032
:108AD0002C960FB6F894DEBF0FBECDBFDF91CF91BD
:108AE0001F910F91FF90EF90089510914F150091F5
:108AF00050152091880721110FC046E556E1602FDF
:108B0000812F0F947B2B20E030E0120F10934F1534
:108B100000935015C901DCCFE0901C15F0901D1595
:108B200028E135E13A832983212F30E03C832B83F0
:108B3000202F30E03E832D8318861F822FEF3FEFDA
:108B40003A8729871C861B869E012F5F3F4FAB010A
:108B5000BC01C7010F94C201B70188E195E10F94F0
:108B6000DB292F813885D1CFCF93DF93FC0125AD51
:108B7000211104C021E025AF0F94E026C0911A1501
:108B8000D0911B15E0914915F0914A1582E0199595
:108B9000E0914915F0914A1581E0199530E020E007
:108BA00044E1BE0188E195E10F94DC262BE435E138
:108BB00047E1BE0188E195E10F94DC26E09149157B
:108BC000F0914A1580E0DF91CF9119948091890747
:108BD000982F9370913059F081608D7F8093890731
:108BE0008AEF0E94D92A88E28A950000E9F7089561
:108BF000CF93C82F80918907982F9370933059F0A5
:108C0000816082608093890788EF0E94D92A88E278
:108C10008A950000E9F78C2FCF910C94AA44CF934A
:108C2000DF939091890792FB222720F92817C9F03A
:108C3000D1E0392F387093FFD0E020E2811124E297
:108C400092E0311101C090E0C82F822F892B0E9441
:108C5000F84580918907C0FB82F9D0FB83F98093A6
:108C60008907DF91CF91089586E20E94F8458091AF
:108C70008907846088608093890786E20E94F845AE
:108C800080918907846088608093890781E00E94D1
:108C90000F4682E00E94F845809189078F7E80937D
:108CA00089070895EF92FF920F931F93CF93DF935D
:108CB000C82F7B0180E00E940F468C2F80640E94A9
:108CC000F8450E94E645D0E0C0E0F701EC0FFD1F3B
:108CD00005911491812F0E94AA44802F0E94AA44DA
:108CE0002296C032D10589F7DF91CF911F910F9164
:108CF000FF90EF90089580E00E940F4681E00E946F
:108D0000F8456FE070E080E090E00D946624CF932A
:108D1000DF93C82FD62F81E00E940F468D2F8068E9
:108D20000E94F8458C2F8F708068DF91CF910C9452
:108D3000F845CF92DF92EF92FF920F931F93CF935C
:108D4000DF93C42E982F9170D92ED82FD695F62E5A
:108D5000F29480EFF8220CE216E1C1E0F801E49011
:108D60006F2D6C0F8D2F0E9487460E94E645CC2008
:108D7000C9F08E2DD11080E00E94AA44D11001C00C
:108D8000E12C8E2D0E94AA44CF5F0F5F1F4FC5308C
:108D900029F7DF91CF911F910F91FF90EF90DF9016
:108DA000CF90089580E00E94AA4480E0EBCF1F930B
:108DB000CF93DF93182FC62FD1E0D627611104C0BF
:108DC00081E596E10E94BA444D2F612F85E00E9413
:108DD00099464C2F612F89E0DF91CF911F910C9420
:108DE0009946DF92EF92FF920F931F93CF93DF93F9
:108DF000D82EC62FC295C07F8A01D0E1DC0F6C2F20
:108E00008D2D0E9487460E94E645F801E590F4907A
:108E10008F2D0E94AA448E2D0E94AA440E5F1F4FE0
:108E2000CF5FDC13ECCFDF91CF911F910F91FF90BB
:108E3000EF90DF900895CF93C82F80E00E940F46F7
:108E40008C2F8068CF910C94F8451F93CF93DF93BC
:108E500088E10E941B470E94E64583EE93E10E9451
:108E60008844C82F813158F483EE93E10E94DC449A
:108E7000C031B1F180E20E94AA44CF5FF9CFC09126
:108E8000E213D0E0CD51DC4ECE010E948844182F71
:108E900060E1CE010E94C844103178F48EE20E9455
:108EA000AA441F3051F08EE20E94AA446EE0611B7A
:108EB00021F083EE93E10E94C84483EE93E10E9487
:108EC00088449091E213981778F49F5FE92FF0E0BF
:108ED000ED51FC4E8081807C8038B9F39093E21391
:108EE000DF91CF911F9108951092E213F9CFA49AC8
:108EF00088E28A950000E9F7809189078E7F809348
:108F000089070895EF92FF920F931F93CF93DF93FA
:108F1000CDB7DEB72C970FB6F894DEBF0FBECDBF2E
:108F200010914F15009150152091880721111AC0FA
:108F30004CE056E1602F812F0F947B2B80E090E076
:108F4000180F10934F15009350152C960FB6F894E8
:108F5000DEBF0FBECDBFDF91CF911F910F91FF906C
:108F6000EF900895E0901C15F0901D1528E135E173
:108F70003A832983212F30E03C832B83202F30E05C
:108F80003E832D8318861F827A8769871C861B86FD
:108F90009E012F5F3F4F43ED5AE2BC01C7010F9482
:108FA0008202B70188E195E10F94DB298F819885D2
:108FB000C7CF6FEF7FEF0C9482470F9380914C15D2
:108FC000853200F580914E158B31E0F01092381506
:108FD00009E028E34BE164E288E195E10F94A028E1
:108FE00081E0809338150E94F4E6882359F085E2E9
:108FF00080934F1583E28093501581E097E10F91A4
:109000000C94D9470F910895AF92BF92CF92DF92FF
:10901000EF92FF920F931F93CF93DF930E94922AB8
:10902000882341F18091460790914707392F40915D
:1090300044075091450720914307213009F4A4C00B
:109040000CF097C0CA01C397222309F4A1C0D091A4
:109050004707C09145073D1302C0C51759F0D831E5
:1090600008F49BC01092570B68E270E080E991E031
:109070000E944DE681E08093381580914C1589302F
:1090800058F410924F1587E0809350158091D806C0
:109090009091D9060E943B3226E34CE769E082E0DA
:1090A0000F942A28F12C20914C1530E08091420732
:1090B000F81608F0D9C1EF2DF0E0AF01440F551FAD
:1090C000DA01A252B94F8C91FA01E052F94F908126
:1090D00011961C91891396C1C181EC2EC1170CF415
:1090E000E12EFE2D65E0F602C00111240E968217D6
:1090F00093070CF4B7C11C170CF4C12F75E0C7021D
:10910000C00111240A9620914E152817190609F05E
:109110000CF4A8C1DC2FDD0FDD0FDC0FD55FCA0119
:109120008252994F6C0180914C1590E0EC160CF432
:1091300099C12D2F0D2E000C330BA9014D5F5F4FF0
:10914000481759079CF080914E158217130674F04A
:10915000F6018081682F660F660F680F6C5F04E070
:1091600024E04D2F88E195E10F94A028CF5FDB5FCD
:10917000DACF223059F0C397233009F068CF9093AB
:1091800047078093460763CFC396F9CFCA01C396BA
:1091900090934507809344075ACFCA3008F062CFB6
:1091A000E0914207F0E0EE0FFF1FE252F94FD0834B
:1091B000C183809139149091DC06282F291B41F03E
:1091C0008093DC0681E012160CF080E00E94F92901
:1091D0008091DD06882309F453C081508093DD0619
:1091E00040914207443008F4EAC050E0FA01EE0F23
:1091F000FF1FE452F94F8081DA01AA0FBB1FA25270
:10920000B94FFC90425051098F118DC0D12C11964D
:109210005F016FEFA61AB60A2D2D30E0241735072F
:109220000CF0CDC08901000F111FB8016252794FB7
:10923000FB019081F801E052F94F7F0120819217E4
:1092400009F453C0392F29170CF4322F8317B4F0C7
:1092500092170CF4922F98178CF00252194FF801C4
:10926000318121E0F501908139170CF020E091E087
:109270006C9163170CF490E02913F4CED394CCCF07
:109280008091DE069091E006891327C08091DF0669
:109290009091E10621E089170CF02FEF820F809367
:1092A000DF0698139DCF309142073150309342072B
:1092B00020E0822F90E0DC01AA0FBB1FA252B94F21
:1092C000880F991FFC01E052F94F808191818D93A5
:1092D0009C932F5F321768F783CF21E089170CF03A
:1092E0002FEF820F8093DE06DCCF8913C7CF2C913E
:1092F000F5011081F7019181FB013181722F121765
:109300000CF4712F692F93170CF4632F67170CF46B
:10931000B5CF21170CF4212F39170CF4932F2917EF
:109320000CF4ACCF9FCEE12CDF0111962E2D30E056
:10933000241735070CF043C0B901660F771F8B0166
:109340000252194FF8019181FB01E052F94F21813E
:109350003C919217D9F0E92F29170CF4E22F3E1710
:109360009CF092170CF4922F931774F06252794F7D
:10937000FB01308121E038170CF020E091E0F3167A
:109380000CF490E029136ECEE394D0CF9313FCCF6E
:109390009081F8012081682FF8160CF46F2D392F79
:1093A00092170CF4322F36177CF3382F8F150CF4EC
:1093B0003F2D29170CF4922F391734F353CE809197
:1093C000DB068D1357CE8091DA068C1353CE6CEDED
:1093D00070E085E090E00E944DE668E171E085E094
:1093E00090E00E944DE68091D8069091D9060196B2
:1093F0009093D9068093D80682E08093DD060E9480
:10940000622E38CE412F440F440F140F155F412FA9
:10941000012E000C550BBA016D5F7F4F6217730769
:109420000CF120914E1524171506E4F0D82F98174B
:109430000CF4D92FC82F89170CF4C92F6D2F660F84
:10944000660F6D0F85E0E82EE60ECD175CF06C5FC1
:1094500004E024E0412F88E195E10F94A028DF5F2C
:109460006E2DF0CFF3941FCE8091DA06682F660F31
:10947000660F680F655F862F062E000C990BAC01F6
:109480004D5F5F4F4217530784F020914E15281708
:1094900019065CF09091DB06892F880F880F890FE1
:1094A00024E044E08C5F0F942A288091570B8111AF
:1094B00002C00E94DD4780913F0B10923F0B882332
:1094C00061F0DF91CF911F910F91FF90EF90DF90AE
:1094D000CF90BF90AF900C942343DF91CF911F9119
:1094E0000F91FF90EF90DF90CF90BF90AF900895D5
:1094F0006F927F928F929F92AF92BF92CF92DF92A4
:10950000EF92FF920F931F93CF93DF9384E08093AA
:109510006F0280918A07882309F45CC08091391416
:1095200090913A148E31910514F08DE190E097FFFF
:1095300002C090E080E090933A1480933914880F31
:10954000991F880F991F20915F0B422F022E000C4C
:10955000550B4817590764F42D5FAC01421B5109A4
:1095600027FD5395423051050CF499C120935F0BB0
:1095700020915F0B422F022E000C550B841795078C
:109580006CF42350422F022E000C550B481B590B34
:10959000423051050CF486C120935F0B8091570B2C
:1095A0008823C1F09091D606992349F02091D506E1
:1095B000920F9093D506933F14F41092D606823002
:1095C00008F47AC181508093570B823009F06DC145
:1095D0000E94F84280918C0782FF5EC38091D7067B
:1095E00081508093D70680913F0B10923F0B8823C8
:1095F00031F08091570B811151C31092D7068091A1
:10960000D706811102C00E94234381E08093381560
:10961000C091CD062C2F0C2E000C330B8091CC0664
:10962000A9016AE08602400D511D1124CA0102976A
:1096300040914C15481719060CF061C080914E15E9
:10964000821713060CF45BC07CE9672E76E0772E58
:10965000E0EA8E2EE2E09E2E1EE11C0F8C2F0C2ED7
:10966000000C990B9C01295F3F4F40914C1542170C
:10967000130609F0DCF520914E1528171906B4F1F0
:10968000D091D106F401C080D12CCC0CDD1CB12CC2
:10969000A12CF301808190E0B0E0A0E00A2C04C08E
:1096A000B695A795979587950A94D2F780FF16C02F
:1096B000E090D206EC0CFD2CF11C54E0EE0CFF1CEB
:1096C0005A95E1F7A701485C584E7A0108E022E07C
:1096D0004C2F6D2F88E195E10F94CD2B5FEFA51AEC
:1096E000B50AD25F65E0A616B10499F6C65F8FEFA2
:1096F000681A780A9FEF891A990AC113AFCF80912F
:10970000D606882389F080914C15883068F44EE2A3
:10971000E42E47E1F42E05E022E042E06091D50618
:1097200088E195E10F94CD2B8091570B8823C9F0E8
:1097300090914C159F33A8F490914E15973388F073
:10974000823010F081FF0DC03EE1E32E37E1F32EB1
:1097500008E022E047E360915F0B88E195E10F9418
:10976000CD2B80915A0B8823C9F06091590B862F1D
:10977000062E000C990B9C012D5F3F4F40914C151C
:109780004217130609F054F420914E1528171906B4
:109790002CF044E08091580B0F94AA27CEEAD6E033
:1097A0000CEC16E08A818823B1F06981862F062EA1
:1097B000000C990B20914C152817190609F05CF440
:1097C000029720914E15281719062CF0625043E09D
:1097D00088810F94AA2723960C171D0719F78091EB
:1097E0005E0B882329F140915D0B842F042E000C21
:1097F000990B9C012A5F3F4F50914C15521713064D
:1098000009F0B4F420914E15281719068CF020E1C8
:10981000E22E27E1F22E07E022E060915C0B88E166
:1098200095E10F94CD2B80915E0B815080935E0B60
:109830008091570B811102C00E94DD4780914C1529
:109840008A3008F03EC210924F1589E0809350157F
:109850008091D8069091D9060E943B3280915B0B93
:10986000882309F42EC2C1E090E1C92ED12C809149
:109870005B0B8C1708F425C2B6016C1B7109660FCF
:10988000660F660F8BE0E82E87E1F82E05E021E0F9
:1098900041E088E195E10F94CD2BCF5FE8CF809335
:1098A0005F0B66CE80935F0B79CE843609F092CE43
:1098B00081E08093570B8ECE8091D4068F5F80938A
:1098C000D4069091D306292F30E03595279582173D
:1098D000130609F00CF494C08091D20621E082278F
:1098E0008093D2061092D406992309F489C08091FE
:1098F000D0069091D106980F2091CF06921724F0B0
:109900002091CE062917CCF481958093D0068091C2
:10991000CD068B5F8093CD069093D1062091CC0627
:10992000082E000C990B3AE02302800D911D1124A2
:10993000C9971CF084E10F94AF1D8091D1069091DE
:10994000D006890F8093D1068091D306882309F42D
:1099500057C064E170E080E090E00F944F22672BE5
:10996000682B692B09F04CC0EEEAF6E0D0E0C0E0CD
:1099700082818111C3C06091D30670E06F5F7F4F19
:10998000072E000C880B990B0F944F226156794FCC
:10999000FB019081492F50E0F4E055954795FA95E9
:1099A000E1F7FA01E056FD4F208130E0BE01660F7D
:1099B000771FC60FD71FC255D94F9F708091D10610
:1099C000FEE09F9F800D1124F901E356FD4F908129
:1099D000890F26563D4FF90190819695890F88830E
:1099E0008091CD06FAE04F9F800D1124885F898316
:1099F00062E070E080E090E00F944F226E5F6A8337
:109A000020915A0B222349F08091590B280F209363
:109A1000590B27FF7AC010925A0BCEEAD6E00CEC15
:109A200016E08A81882339F09981890F89838034EF
:109A30000CF415C11A8223960C171D0791F780911B
:109A4000D60681111BC064EF71E080E090E00F94B6
:109A50004F22672B682B692B89F462E070E080E06D
:109A600090E00F944F22672B682B692B09F40FC1EC
:109A700081E08093D60683EF8093D50680915A0BC0
:109A8000882309F4A7CD8091D606882309F4A2CDB6
:109A90008091590B87300CF09DCD2091580B80910F
:109AA000D50628170CF496CD022E000C330B082E89
:109AB000000C990B0C96821793070CF48BCD109227
:109AC000D60610925A0B8091D8069091D9060A9624
:109AD0009093D9068093D8066AE070E088E290E01F
:109AE0000E944DE68091D5068F5F80935C0B81E0EC
:109AF00080935D0B84E080935E0B6CCD2196339652
:109B0000CA30D10509F034CF7BCF0091CD062017A4
:109B10000CF483CF022E000C330B002E000C110B23
:109B2000C8014D96821793070CF477CFC091580B5C
:109B3000AC2E0C2E000CBB08D091D106C5018D1B9C
:109B40009109D7FD93956EE070E00F948148E62E61
:109B500044E0461708F461CF201B310BC90102967F
:109B60006AE070E00F948148F62E52E0561708F430
:109B700054CF41E050E060E070E00E2C04C0440F90
:109B8000551F661F771F0A94D2F7AF2D0F2C000CBC
:109B9000BB0B8D010456194FF801D0808D2D842305
:109BA00009F43BCFCD0180569D4FFC01208130E070
:109BB000FEE0EF9ED00D1124C90183569D4FFC019C
:109BC0008081D80FCD170CF428CF26563D4FF901D0
:109BD000C0818C2F90E08D0F911DD7FD9A95A8160E
:109BE000B9060CF01ACF10925A0B942F90959D2124
:109BF000F801908323E030E02A1B3B0B8091D806CC
:109C00009091D906820F931F9093D9068093D8061E
:109C10006AE070E088E290E00E944DE69091CD0607
:109C2000FAE0FF9E900D11248C2F86958D0F8550A4
:109C300080935C0B90935D0B84E080935E0B80912E
:109C4000D30681508093D306882319F00E94152AE9
:109C5000E4CE84E18093570B0E94EF42DECE87333F
:109C60000CF4E9CE288180915F0B28170CF4E3CE29
:109C7000022E000C330B082E000C990B0A9682174B
:109C800093070CF4D8CE88E70F94AF1DD4CE8FEF96
:109C90008093D6068FE7F0CE8AE0A3CC813009F01E
:109CA000AECC80915A0B8111AACC80915F0B8B5F57
:109CB0008093580B84E38093590B8CEF80935A0B5D
:109CC0009ECCDF91CF911F910F91FF90EF90DF908D
:109CD000CF90BF90AF909F908F907F906F9008959E
:109CE000AF92BF92CF92DF92EF92FF920F931F93AA
:109CF000CF93DF930E94922A882309F409C18091AF
:109D0000391486320CF4EBC085E2282F082E000CA3
:109D1000330B30933A1420933914982F990F890FED
:109D200080939A068091570B882309F4F1C0209103
:109D30008C0630918D0600918E0610918F06020FD1
:109D4000131FC0918A06D0918B068091880690914E
:109D50008906C80FD91F01304FE7140768F0319505
:109D60002195310930938D0620938C066CED70E0BF
:109D700085E090E00E944DE6D7FFB5C0809188064F
:109D80009091890691958195910990938906809388
:109D9000880668E171E085E090E00E944DE681E090
:109DA000809387062091880630918906CE019A50CB
:109DB0008130934108F090C18D2F992787FD9A95A6
:109DC0000A9765E070E00F948148412F17FF02C0A9
:109DD00047E0410F45954595459581E090E0A0E02D
:109DE000B0E004C0880F991FAA1FBB1F4A95D2F785
:109DF000FB01EE0FFF1FE057F94F40815181EA014F
:109E0000C823D923CD2B09F44DC080959095842388
:109E100095239183808344E050E0461B570B80914B
:109E2000D8069091D906840F951F9093D9068093F8
:109E3000D80680919806815080939806811103C0BE
:109E400082E08093570B932F9095991F9927991F24
:109E500080918706881F8827881F981709F419C1E1
:109E6000319521953109309389062093880660E267
:109E700070E080E090E00F944F22DC01CB0140972E
:109E8000A109B10920918C0630918D06820F931F94
:109E900090938D0680938C0660E773E085E090E0F8
:109EA0000E944DE680918E0690918F0620918C063F
:109EB00030918D06820F931F90938F0680938E06AC
:109EC00080918A0690918B062091880630918906B0
:109ED000820F931F90938B0680938A0619C087FF89
:109EE00014CF80E012CFC13080E4D8070CF45ACFF1
:109EF0006BE470E084EF91E00E944DE6809199065A
:109F0000815080939906882309F4C0C00E94AB2A2F
:109F100081E08093381580914C158E3108F057C040
:109F200080914E158A3008F452C080E9C82E86E030
:109F3000D82ECAE0D0E0BC2E20914C15CE0104965C
:109F40002817190609F0DCF580914E158C17B8F129
:109F500010E000E0F60180819181B0E0A0E0002EE9
:109F600004C0B695A795979587950A94D2F780FF78
:109F700021C0A02EAA0CAA0CAA0CF12CE12CCE0117
:109F80008E0D9F1D20914C152817190609F05CF4C1
:109F900020914E152817190634F047E06B2D6E0DF1
:109FA0008A2D0F946428FFEFEF1AFF0A24E0E216CF
:109FB000F10429F70F5F1F4F0031110559F642E0F8
:109FC000C40ED11C2596CE31D10509F0B4CF8091B5
:109FD0004C158E3380F480914E158C3360F040E147
:109FE0006DE380919A060F94642840E16CE38091C0
:109FF0009A060F9464288091570B882309F414C1A2
:10A0000060918B06862F90E0019620914C152817C1
:10A01000190609F054F480914E15861730F022E0AD
:10A0200042E080918F060F942A2880914C158B3046
:10A03000D0F410924F15C9E0C09350158091D80606
:10A040009091D9060E943B328EE680934F15C093C3
:10A0500050152091990683E090E0821B910985506C
:10A06000994E0E94D94780913F0B10923F0B882355
:10A0700009F4DDC0DF91CF911F910F91FF90EF9018
:10A08000DF90CF90BF90AF900C9423431092570B6A
:10A090003FCF80918C0690918D0691958195910985
:10A0A00090938D0680938C0660E270E080E090E0F3
:10A0B0000F944F22DC01CB014097A109B1092091F7
:10A0C000880630918906820F931F909389068093AA
:10A0D000880660E872E0E2CE121613060CF0E2CEBB
:10A0E000DD53C130D24008F0DDCE80919A06C12FF9
:10A0F000C81BC03108F0D6CE319521953109309377
:10A1000089062093880660E773E083E090E00E9470
:10A110004DE68FEF809387068EEF8C0F8C3088F1A1
:10A1200080918C0690918D0631E0181619060CF07E
:10A1300030E021E0C2300CF020E09195819591094A
:10A14000321709F444C08091570B823009F0AACE2F
:10A1500080E4809398068FEF9FEF90939106809311
:10A160009006909393068093920690939506809321
:10A170009406909397068093960681E08093570B00
:10A1800091CEC43060F560E470E080E090E00F9420
:10A190004F22DC01CB0180549109A109B109209122
:10A1A0008C0630918D06820F931F81152EEF92073A
:10A1B0009CF090938D0680938C0680918C069091F4
:10A1C0008D06813092400CF4BECF80E092E09093F7
:10A1D0008D0680938C06B7CF80E09EEFEACFCC301F
:10A1E0000CF4B1CF60E470E080E090E00F944F2277
:10A1F00020918C0630918D06C901860F971F909390
:10A200008D0680938C0681159E4F34F480E09EEF7E
:10A2100090938D0680938C0680918C0690918D068C
:10A220008130924094F68FCF0E94DD47FECEDF91C1
:10A23000CF911F910F91FF90EF90DF90CF90BF9043
:10A24000AF900895EF92FF920F931F93CF93DF93F8
:10A25000CDB7DEB72C970FB6F894DEBF0FBECDBFDB
:10A2600010914F15009150152091880721111AC0A7
:10A270004CEE55E1602F812F0F947B2B80E090E016
:10A28000180F10934F15009350152C960FB6F89495
:10A29000DEBF0FBECDBFDF91CF911F910F91FF9019
:10A2A000EF900895E0901C15F0901D1528E135E120
:10A2B0003A832983212F30E03C832B83202F30E009
:10A2C0003E832D8318861F827A8769871C861B86AA
:10A2D0009E012F5F3F4F46ED5AE2BC01C7010F942C
:10A2E0008202B70188E195E10F94DB298F8198857F
:10A2F000C7CFEF92FF920F931F93CF93DF937B0112
:10A30000C42F622F0E94E8448823D1F1CC23F9F0B6
:10A3100001151105E1F4C7010E94664425E130E012
:10A32000A901481B5109CA0157FD019695958795CA
:10A33000C0E8DFE7D80F8D2F8C0F87FD09C060E2E2
:10A3400070E080E090E00E944945C150F4CFC0E841
:10A350006C2F70E0C7010E948247C81B01151105D0
:10A3600031F06C2F70E0C8010E942251C81BC73029
:10A3700038F060E270E080E090E00E944945F6CF5E
:10A38000DF91CF911F910F91FF90EF900895DF9291
:10A39000EF92FF920F931F93CF93DF9361E081E0E1
:10A3A0000E94EE33C091381485E0F82EFC0E81E057
:10A3B000D2E0DC1BE82EEC1ADC2ED194C11128C0AF
:10A3C000882389F08091370B18166CF0209139148E
:10A3D00030913A142F5F3F4F30933A142093391441
:10A3E0008F5F8093370B80916F02882349F010E0D4
:10A3F00000E020E041E06CEC7BE18D2D0E94795182
:10A4000080E0CF5FFC12DACF83E08093371421C065
:10A41000C13039F59091370B913079F080916F020E
:10A42000882371F381E0913009F080E020E241EC73
:10A430005BE16E2D0F94CF1CE3CF80913F0B109208
:10A440003F0B882359F3C0938007809134148823ED
:10A4500029F3DF91CF911F910F91FF90EF90DF9043
:10A460000895C23069F69091370B923069F080916F
:10A470006F02882329F281E0923009F080E020E227
:10A480004DEA5BE16D2FD6CF80913F0B10923F0BD1
:10A49000882369F3C093800780913414882339F3AB
:10A4A000D8CF0F931F93CF93DF9380916F028823B0
:10A4B00059F0609182077091830710E000E020E07E
:10A4C00041E081E00E94795180918B0781111AC08F
:10A4D00081E080938B07C0911215D091131540E055
:10A4E00060E081E592E50F94BD020E9494CE109247
:10A4F0008B0740E060E0CE01DF91CF911F910F917B
:10A500000D94BD02DF91CF911F910F9108956FEFD0
:10A510007FEF0C9422512F923F924F925F926F9255
:10A520007F928F929F92AF92BF92CF92DF92EF92E3
:10A53000FF920F931F93CF93DF934C016B015A014E
:10A5400060E085E00E94EE335090381453E0652EB1
:10A55000C114D10411F442E0642ED52D8EE0E82E12
:10A56000F12C92E0292E2EE3322E35E0432E7D2E63
:10A570007518D111D6C080916F02882399F080910F
:10A5800006026FEE7BE1823031F06FED7BE18330CC
:10A5900011F06DEC7BE110E000E021E041E0872D5F
:10A5A0000E947951C62DA114B10411F16D120CC095
:10A5B00080916F02882341F010E000E020E041E04C
:10A5C000B501872D0E947951C62DCF5F81E090E0C3
:10A5D000C114D10411F490E080E021E030E0A11436
:10A5E000B10411F430E020E0820F931F029781F054
:10A5F000CD130DC080916F02882349F010E000E078
:10A6000020E041E068E07CE1872D0E947951CF5F36
:10A61000CD1368C080916F02882309F461C010E0F7
:10A6200000E021E040E06DEF7BE1872D0E94795151
:10A630001091810793EF9E0D90937F078EEF8E0D03
:10A640008093B10B20914C152E151F0411F00CF0C6
:10A6500047C020914E15921708F042C030924F1516
:10A660008093501565E470E080E090E00E944945D9
:10A6700061E3610F062E000C770B880B990B0E948B
:10A68000494560E270E080E090E00E9449456091B9
:10A69000491470914A1480914B1490914C140F946A
:10A6A000BB46CB010E94D1E10E9487526FE270E06D
:10A6B00080E090E00E9449450E94F4E6811108C0C4
:10A6C000419EF0011124E25DFB4E8481811108C09E
:10A6D00080914D1490914E140E94D1E10E948752B6
:10A6E00020926F028CE0E80EF11CDF5F8AE4E8162E
:10A6F000F10409F03CCFCF5FC0933714DF91CF91C5
:10A700001F910F91FF90EF90DF90CF90BF90AF908F
:10A710009F908F907F906F905F904F903F902F9081
:10A720000895D13059F480916F02882309F43ACF0B
:10A7300010E000E020E041E0B40131CFC114D104C9
:10A7400009F430CFD23009F02DCF80916F028823E9
:10A7500041F010E000E020E041E0B601872D0E94CA
:10A760007951C3E0A114B10409F02FCF2FCFAF92DC
:10A77000BF92CF92DF92EF92FF920F931F93CF93EE
:10A78000DF935C016B010E946644E82EC6010E94C3
:10A790008844F12C03E110E0081B1109C5E20E15F5
:10A7A0001F050CF4CFE18C2F90E09C012E5F3F4FF2
:10A7B00040914C154217130609F094F50997209122
:10A7C0004E152817190664F110924F15C0935015B5
:10A7D000C5010E94D947D1E0C114D104B1F06AE3A8
:10A7E00070E080E090E00E9449450E151F05D4F40A
:10A7F000C45F80914C15C81740F020914E154C2F26
:10A800004950550B241715067CF4DF91CF911F9109
:10A810000F91FF90EF90DF90CF90BF90AF90089591
:10A82000D0E0DACFDD2389F3802F880F080F000FE7
:10A8300000934F15C093501560E270E080E090E007
:10A840000E944945C601DF91CF911F910F91FF9062
:10A85000EF90DF90CF90BF90AF900C948752CF9342
:10A86000DF93FC01EB018091391490913A1497FF2A
:10A8700004C010923A14109239144091430B509135
:10A88000440B6091450B7091460B80913914909167
:10A890003A14092E000CAA0BBB0B481759076A077C
:10A8A0007B0724F450933A144093391480916F023B
:10A8B0008823C1F02091391430913A146091470BEC
:10A8C0007091480B8091490B90914A0B620F731F56
:10A8D000811D911D1995BC0180914D0B90914E0BDE
:10A8E0000E94B75380913F0B811108C08091400BAB
:10A8F0008823A1F180916F02882381F180914B0B15
:10A9000090914C0B009791F02091391430913A14AA
:10A910004091470B5091480B6091490B70914A0B45
:10A92000420F531F611D711DFE011995E091410BEE
:10A93000F091420B309741F08091400B811103C0A0
:10A9400080913F0B8111199580913F0B10923F0B25
:10A95000882321F0DF91CF910C947434DF91CF9153
:10A96000089565E179E282E49DE20C942F5469E751
:10A9700079E288E69DE20C942F546FE479E284EE4C
:10A980009DE20C942F5469E379E28AED9DE20C94E8
:10A990002F5461EA79E287E89DE20C942F5465EB2D
:10A9A00079E284EA9DE20C942F5465E679E28EEE1A
:10A9B0009DE20C942F546DE879E28BE49DE20C94B7
:10A9C0002F5469EC79E288E59EE20C942F546DEDEA
:10A9D00079E285E29DE20C942F5468E079E28CE301
:10A9E0009EE20C942F546BEE79E28CEF9CE20C9477
:10A9F0002F542F923F924F925F926F927F928F923D
:10AA00009F92AF92BF92CF92DF92EF92FF920F93FD
:10AA10001F93CF93DF93EB01FC0180809180A28094
:10AA2000B380C501B40120E831E541E050E00F9466
:10AA3000EB44C9016DE671E00F946D486B017C0138
:10AA4000C501B40120E13EE040E050E00F94EB444A
:10AA5000CA01B90128E130E040E050E00F94EB4436
:10AA6000362E272E062F172F8CE3482E512C612CC3
:10AA7000712CC501B401A30192010F94EB44B62ED1
:10AA8000A72ECA01B901A30192010F94EB44CB0197
:10AA9000C114D10469F1AF92BF927F936F932F924B
:10AAA0003F92FF92EF92DF92CF9289EC93E19F93D6
:10AAB0008F93DF93CF930F948F408DB79EB70E96F1
:10AAC0000FB6F8949EBF0FBE8DBFDF91CF911F913F
:10AAD0000F91FF90EF90DF90CF90BF90AF909F903D
:10AAE0008F907F906F905F904F903F902F90089540
:10AAF000E114F104C9F0AF92BF927F936F932F924C
:10AB00003F92FF92EF9289EB93E19F938F93DF93B4
:10AB1000CF930F948F40EDB7FEB73C960FB6F894E5
:10AB2000FEBF0FBEEDBFD1CF012BB9F0AF92BF92E8
:10AB30007F936F932F923F928DEA93E19F938F9330
:10AB4000DF93CF930F948F408DB79EB70A960FB6C1
:10AB5000F8949EBF0FBE8DBFB8CF892BA9F0AF92DE
:10AB6000BF927F936F9385EA93E19F938F93DF93D7
:10AB7000CF930F948F40EDB7FEB738960FB6F89489
:10AB8000FEBF0FBEEDBFA1CFAF92BF9281EA93E1AE
:10AB90009F938F93DF93CF930F948F400F900F90DD
:10ABA0000F900F900F900F9090CF9091A11693FB64
:10ABB000882780F993FF06C081E090915F1491117E
:10ABC00001C080E008952F923F924F925F926F9262
:10ABD0007F928F929F92AF92BF92CF92DF92EF922D
:10ABE000FF920F931F93CF93DF93CDB7DEB762979A
:10ABF0000FB6F894DEBF0FBECDBF8D870E9477479A
:10AC00002D85211136C00E94F4E6409127149091C1
:10AC10006D02499FA0011124440F452F441F550B7D
:10AC2000519520910D0230910E0260914D1470915A
:10AC30004E14262737276091B6077091B70726274D
:10AC400037272427A9014827CA012091820630917D
:10AC500083068217930749F4E3EEF3E180E09191D4
:10AC6000992309F4AAC28927FACF90938306809387
:10AC700082060E94F4E68E870E9491DD4B015C0102
:10AC800050910D02598B80910E028A8B609149146C
:10AC900070914A1480914B1490914C140F94BB46C0
:10ACA0006B0120914D1430914E143B872A8760919F
:10ACB000B2077091B3078091B4079091B5070F94D4
:10ACC000BB462B01788B6F872090B6073090B70773
:10ACD0004A855B854115510569F04C155D050CF001
:10ACE00046C251E05887C6012A853B85821B930BDB
:10ACF00003970CF4188680910502817048858417AB
:10AD000009F43CC251E05C8781E00E941B470E942D
:10AD1000E645DF92CF9242E4E42E46E1F42EFF9224
:10AD2000EF928E010F5F1F4F1F930F930F948F4071
:10AD3000C8010E94DC440F900F900F900F900F906D
:10AD40000F9098859923B1F08AE10E94AA442B853F
:10AD50002F933A853F93FF92EF921F930F930F9497
:10AD60008F40C8010E94DC440F900F900F900F900D
:10AD70000F900F904C85442321F0688580E00E945D
:10AD8000D74680910502588550FB80F980930502D3
:10AD90002114310469F08F859889DD24D394281615
:10ADA00039060CF0EEC1C2018219930903970CF425
:10ADB000D12C8091050282FB882780F9CC24C39492
:10ADC0008D1101C0CD8481E10E941B470E94E645A0
:10ADD0005F924F9232E4E32E36E1F32EFF92EF9230
:10ADE0001F930F930F948F40C8010E94DC440F9073
:10ADF0000F900F900F900F900F90DD20A1F08AE13F
:10AE00000E94AA443F922F92FF92EF921F930F93BA
:10AE10000F948F40C8010E94DC440F900F900F9058
:10AE20000F900F900F90CC2021F06D2D81E00E94AB
:10AE3000D74680910502D0FA82F98093050280916D
:10AE40002714282F30E0398728873E8531110FC01D
:10AE500090916D0297FD0BC0899FC0011124AC0138
:10AE6000440F452F441F550B51955987488786E05D
:10AE70000E941B470E94E64524E648855985249F89
:10AE8000C001259F900D112481589F4F6FEF70E0F6
:10AE90000F9481487F936F9382E496E19F938F9301
:10AEA0001F930F930F948F40C8010E94DC4485E2EA
:10AEB0000E94AA4488E00E941B47C501B40120E11A
:10AEC0003EE040E050E00F94EB4469019CE3492EE2
:10AED000512C612C712CC501B401A30192010F9476
:10AEE000EB440F900F900F900F900F900F90CA01AE
:10AEF000B901A30192010F94EB4454E6C516D104A5
:10AF000008F043C17F936F93DF92CF9288E396E17D
:10AF10009F938F931F930F930F948F400FB6F894C6
:10AF2000DEBF0FBECDBFE5E0E00FF12FF11D80E2E7
:10AF300080830E94E64566E0C8010E94C84486E11D
:10AF40000E941B470E94E6453A893F9349894F93E7
:10AF500082E496E19F938F931F930F930F948F40FA
:10AF6000C8010E94DC4485E20E94AA440F900F9021
:10AF70000F900F900F900F9088859985892B79F00D
:10AF800085E00E941B470E94E6459E8516E09111D0
:10AF900014E080E00E94AA44812F0E94AA44121467
:10AFA00013040CF01E8680E10E941B470E94E645B8
:10AFB000121413040CF0FCC02E8512E0211110E0D5
:10AFC00080E00E94AA44812F0E94AA443D85332339
:10AFD00009F442CE1092E2130E9425470E94292DC7
:10AFE0008091A11682FF2AC00E94D555882309F4BA
:10AFF000EBC08091991690919A16A0919B16B091F2
:10B000009C160097A105B10509F4DEC0BC01CD0175
:10B010006D597F4F8F4F9F4F24E630E040E050E066
:10B020000F94EB4460919D1670919E1680919F162F
:10B030009091A0160F94EB4420938506C09085064E
:10B040004D85411105C0809186068C1509F474C0A8
:10B05000C09286068C2D69E10F94614850E1959F5E
:10B06000C001112469E170E00F94814880E090E80C
:10B070004C0102C0959487946A95E2F7DD24D3943D
:10B08000EC2CF12C6D2D8CE00E9487460E94E64549
:10B0900089E1A82EB12C712C0FEF1FEFEA14FB04ED
:10B0A00044F4C501499710E000E08E159F050CF4AB
:10B0B000840181E0D81609F48DC09DE0D91609F409
:10B0C00089C023E0721282C00160812F0E94AA44CD
:10B0D000802F0E94AA44739439E1A30EB11C44E06E
:10B0E0007412DACFD3945EE0D512CCCF8CE00E94FC
:10B0F0001B470E94E64580E20E94AA448E010F5F32
:10B100001F4F89E08C1508F068C0FF92EF9286E42B
:10B1100096E19F938F931F930F930F948F40C801D5
:10B120000E94DC448EE496E10E94BA440F900F9096
:10B130000F900F900F900F900E94774762960FB676
:10B14000F894DEBF0FBECDBFDF91CF911F910F915D
:10B15000FF90EF90DF90CF90BF90AF909F908F9037
:10B160007F906F905F904F903F902F90089531E0C7
:10B1700038878A859B858C199D09BACD8D858C87EA
:10B18000C3CDC1018419950911CE7F936F93DF92CE
:10B19000CF9280E396E19F938F931F930F930F9429
:10B1A0008F400FB6F894DEBF0FBECDBFE6E0BCCE39
:10B1B00080E20E94AA4480E207CF9091840689171A
:10B1C000E1F08093840606CF20E036CF71107DCF6A
:10B1D00010687BCF0FEF1FEF78CFFF92EF9282E4E2
:10B1E00096E19F938F931F930F930F948F40C80105
:10B1F0000E94DC448AE496E197CF0E94292D88239F
:10B2000009F4EECE0E942547EBCE4F925F926F92EB
:10B210007F928F929F92AF92BF92CF92DF92EF92E6
:10B22000FF920F931F93CF93109294051092930562
:10B230002FE3209397051092960510929505109292
:10B240008F051092900510929105109292059C0125
:10B25000F90190812F5F3F4F9032D1F39E34C9F4B2
:10B26000818190ED980F9A3020F08D3211F08B3261
:10B2700081F432969F012F5F3F4F808180538A3047
:10B2800008F475C09F012F5F3F4F8081803209F421
:10B2900070C0F093CA0BE093C90B8F010F5F1F4F73
:10B2A000C0816AE270E0C8010F94E048009731F075
:10B2B000FC01319780818032E1F31182CD3429F095
:10B2C000C43519F0C73409F042C0F80180810F5F1E
:10B2D0001F4F8032D1F380538A30C8F5C093970551
:10B2E00090E080E0AAE0AF014F5F5F4F2081022E27
:10B2F000000C330B20533109A89FB001A99F700D9A
:10B300001124C901860F971FFA01208120532A308A
:10B3100050F39093960580939505DF0131962C911B
:10B320002032D9F3CD3499F58737910524F5853747
:10B3300091054CF48C31910531F08E31910519F065
:10B340008731910521F5B0939405A0939305CF9192
:10B350001F910F91FF90EF90DF90CF90BF90AF9033
:10B360009F908F907F906F905F904F900895F9011C
:10B3700081CFF90187CF8A3223E0920744F08433EA
:10B38000E3E09E0704F3803AF3E09F07E1F21091B7
:10B39000C90BC12CD12C760150E040E0812C912CBE
:10B3A0005401839401C0DF01FD0131962C912223C9
:10B3B00009F481C02132E1F4CD34D1F48032910519
:10B3C000B9F4C0928F05D0929005E0929105F09269
:10B3D0009205F0939405E093930563E270E0CF014A
:10B3E0000F94E048009709F4B2CFDC011C92AFCF74
:10B3F00021542A3108F05AC0DF013D91303291F0DA
:10B4000060ED630F6A30E8F03E3271F43181305301
:10B410003A30B8F04115510519F4AF0141505109C6
:10B4200030E013C0FD01E8CF3D3211F03B3291F71F
:10B43000318160ED630F6A3020F03E3259F732817E
:10B44000E6CF3E2F311B309759F3622F70E0240175
:10B45000350104C0440C551C661C771C2A95D2F794
:10B46000C428D528E628F7286B587A4FDB013C938F
:10B47000208121542A3108F496CFDF01FD012D915E
:10B48000222309F490CF30ED320F3A30B8F333ED88
:10B49000320F323098F32B3289F39F012F5F3F4FE9
:10B4A0006081603209F07FCFF901F7CF4115510576
:10B4B000F9F6AD01DDCF5093940540939305C0920A
:10B4C0008F05D0929005E0929105F09292053FCFC2
:10B4D00080E1E3E5F2E0A8EBBBE001900D928A95F4
:10B4E000E1F708952F923F924F925F926F927F9271
:10B4F0008F929F92AF92BF92CF92DF92EF92FF9284
:10B500000F931F93CF93DF93CDB7DEB72F970FB66F
:10B51000F894DEBF0FBECDBF282E8B014B879AE07B
:10B52000492E97ED592E93E2692E9CE3792E80E007
:10B5300090E0A0E8BFE3222351F0412C512C80E899
:10B54000682E8EE3782E80E090E0A0EAB1E4898353
:10B550009A83AB83BC8380E090E0A8E4B2E421113D
:10B5600004C080E090E0A0EAB0E48D839E83AF83C6
:10B57000B8870E94685A812C912C540194E0299E2E
:10B5800010011124D101A854B44FBA87A987C8016A
:10B59000110FAA0BBB0B8C879D87AE87BF87A98530
:10B5A000BA85CD90DD90ED90FC902D813E814F814C
:10B5B0005885C501B4010F94F84087FF44C06C85DD
:10B5C0007D858E859F850F94FF40A30192010F9486
:10B5D0005E41A70196010F944F45E985FA85608386
:10B5E000718382839383E090C00BF090C10B009134
:10B5F000C20B1091C30B2091BC0B3091BD0B40913D
:10B60000BE0B5091BF0B6091B80B7091B90B80913C
:10B61000BA0B9091BB0BDE0111966D010E9458D4BC
:10B620000E9494CE83B182958170B1E08B27EB8527
:10B63000E81749F0A3019201C501B4010F944F45E9
:10B640004B015C01ACCFF101E854F44F6081718192
:10B65000828193812F960FB6F894DEBF0FBECDBFC7
:10B66000DF91CF911F910F91FF90EF90DF90CF90DE
:10B67000BF90AF909F908F907F906F905F904F9012
:10B680003F902F9008953F924F925F926F927F92DA
:10B690008F929F92AF92BF92CF92DF92EF92FF92E2
:10B6A0000F931F93CF93DF9300D000D01F921F9270
:10B6B000CDB7DEB7D82E4D835E836F837887322E69
:10B6C000270138010E94685A84E0D89EF0011124B5
:10B6D000E854F44F8D819E81AF81B885808391833A
:10B6E000A283B3839FEF391651F0A4E03A9EF00194
:10B6F0001124E854F44F4082518262827382BFEF7A
:10B70000CB1651F084E0C89EF0011124E854F44FA8
:10B7100080829182A282B3828090B80B9090B90B04
:10B72000A090BA0BB090BB0B20E030E041E953E4AD
:10B73000C501B4010F94F84087FFA5C020E030E0B8
:10B740004CE552ECC501B4010F94AF47181634F024
:10B75000812C912C3CE5A32E32ECB32E8092B80BB9
:10B760009092B90BA092BA0BB092BB0B4090BC0B5D
:10B770005090BD0B6090BE0B7090BF0B20E030E08E
:10B780004AE953E4C301B2010F94F84087FF82C035
:10B7900020E030E040EF51ECC301B2010F94AF471D
:10B7A000181634F0412C512C90EF692E91EC792E23
:10B7B0004092BC0B5092BD0B6092BE0B7092BF0BBF
:10B7C0008091C00B9091C10BA091C20BB091C30BA3
:10B7D0008D839E83AF83B88720E030E446E953E44D
:10B7E000BC01CD010F94F84087FF5BC020E030E042
:10B7F00040E050EC6D817E818F8198850F94AF473A
:10B80000181644F080E090E0A0E0B0EC8D839E83B9
:10B81000AF83B8878D819E81AF81B8858093C00B3F
:10B820009093C10BA093C20BB093C30B80E090E048
:10B83000A8E4B2E489839A83AB83BC83DE011196CA
:10B840006D01ED80FE800F811885A3019201C50175
:10B85000B4010E9458D428960FB6F894DEBF0FBEEC
:10B86000CDBFDF91CF911F910F91FF90EF90DF90AF
:10B87000CF90BF90AF909F908F907F906F905F9090
:10B880004F903F900895812C912C21E9A22E23E422
:10B89000B22E64CF412C512C8AE9682E83E4782E95
:10B8A00087CF80E090E4A6E9B3E4B0CF8F929F9277
:10B8B000AF92BF92CF92DF92EF92FF920F931F93BE
:10B8C000CF93DF93EC016A017B0120E030E040EA96
:10B8D00050E4688579858A859B850F944F45A7013B
:10B8E00096010F944F45AB01BC01812C912C540162
:10B8F000CC24CA94850174012FEF82E00E94435B3F
:10B90000EC80FD800E811F81488159816A817B8195
:10B9100021E080E00E94435BDF91CF911F910F9166
:10B92000FF90EF90DF90CF90BF90AF909F908F905F
:10B9300008954F925F926F927F928F929F92AF92F3
:10B94000BF92CF92DF92EF92FF920F931F93CF930C
:10B95000DF93EC016A017B0120E00F94171921E0CD
:10B96000B701A601CE010F94171923E0B701A60174
:10B97000CE010F94171924E0B701A601CE010F9450
:10B980001719488C598C6A8C7B8C88889988AA886E
:10B99000BB88A5019401C301B2010F944F4520E07B
:10B9A00030E040E05FE30F945E41688379838A83EF
:10B9B0009B838E01005C1F4FA3019201C501B4015E
:10B9C0000F944E4520E030E040E251E40F944E45A4
:10B9D000F8016083718382839383B701A601CE014E
:10B9E0000E94565C288139814A815B8160E070E861
:10B9F00082E893E40F944E456CAB7DAB8EAB9FAB6E
:10BA000018AE19AE1AAE1BAE288539854A855B85FE
:10BA100060E070E080E090EC0F944E456CAF7DAF3D
:10BA20008EAF9FAFDF91CF911F910F91FF90EF905D
:10BA3000DF90CF90BF90AF909F908F907F906F904E
:10BA40005F904F900895FF920F931F93CF93DF93D2
:10BA500000D000D0CDB7DEB78C01F090D80B8FEFBF
:10BA60008093D80B83E692E09A8389838091630266
:10BA700090916402A0916502B09166028B839C83D1
:10BA8000AD83BE831092630210926402109265022D
:10BA900010926602C8010E94995C0E9494CE60E0F8
:10BAA000C8010E945C2C62E0C8010E945C2C0E94CC
:10BAB0005AD5CE0101960E943A2CF092D80B2696C8
:10BAC0000FB6F894DEBF0FBECDBFDF91CF911F91AF
:10BAD0000F91FF9008952F923F924F925F926F9235
:10BAE0007F928F929F92AF92BF92CF92DF92EF920E
:10BAF000FF920F931F93CF93DF9300D000D0CDB769
:10BB0000DEB73C01D090D80B1092D80B83E6E82E1C
:10BB100082E0F82EFA82E9828091630290916402B9
:10BB2000A0916502B09166028B839C83AD83BE8336
:10BB300010926302109264021092650210926602E3
:10BB4000C3010E94995C0CEC1BE0F30124A135A118
:10BB500046A157A164A575A586A597A50F944F4545
:10BB600020E030E040E05FE30F945E41F801608345
:10BB7000718382839383F30180A991A9A2A9B3A9B8
:10BB8000F80184839583A683B783F30180A191A1F3
:10BB9000A2A1B3A1F80180879187A287B387CE01C4
:10BBA00001960E943A2C8FEF8093D80BFA82E9829B
:10BBB0008091630290916402A0916502B091660247
:10BBC0008B839C83AD83BE831092630210926402C8
:10BBD000109265021092660293E5692E92E0792E2A
:10BBE00020E030E040E450E4F30160857185828517
:10BBF00093850F944F454B015C0120E030E040E419
:10BC000050E4F30164817581868197810F944F45DB
:10BC10001B012C0120E030E040E450E4F30160819E
:10BC20007181828193810F944F45AB01BC0122E069
:10BC3000C22E8201710121E080E00E94435B20E07E
:10BC400030E040E450E4F30160857185828593859E
:10BC50000F944E454B015C0120E030E040E450E49D
:10BC6000F30164817581868197810F944E451B0194
:10BC70002C0120E030E040E450E4F3016081718168
:10BC8000828193810F944E45AB01BC018201710109
:10BC900021E080E00E94435BCE0101960E943A2C95
:10BCA000D092D80B26960FB6F894DEBF0FBECDBF4C
:10BCB000DF91CF911F910F91FF90EF90DF90CF9088
:10BCC000BF90AF909F908F907F906F905F904F90BC
:10BCD0003F902F9008950E94B32C882341F081E07B
:10BCE0002091640530916505232B09F480E00895C7
:10BCF000CF92DF92EF92FF926A017B010E946B5E0E
:10BD0000882331F0FF90EF90DF90CF900C942E338A
:10BD1000C701B601FF90EF90DF90CF900895CF92CA
:10BD2000DF92EF92FF920F931F93CF93DF938EE8F2
:10BD3000C82E82E0D82E98EBE92E9BE0F92E03E581
:10BD400012E0D0E0C0E0F60181916F010E946B5ECD
:10BD5000882309F473C00E942E33FE01E559FA4F7F
:10BD60002081211104C020917305222339F0F801AC
:10BD700020813181428153810F944F45F7016083C7
:10BD80007183828393832196F4E0EF0EF11C0C5FA4
:10BD90001F4FC430D105B9F640E050E0BA0186E447
:10BDA0000E94785E20E030E0A9010F94AF4718169A
:10BDB00084F40E942E3320E030E040E752E40F94F8
:10BDC000494660934F0270935002809351029093C2
:10BDD00052028091881183FD28C0809139098823FF
:10BDE00021F120915F0230916002409161025091F7
:10BDF00062026091C40B7091C50B8091C60B90914B
:10BE0000C70B0F944E452091460930914709409148
:10BE10004809509149090F944F4560934609709322
:10BE200047098093480990934909DF91CF911F9169
:10BE30000F91FF90EF90DF90CF900895F8018081EF
:10BE40009181A281B381F70180839183A283B3831F
:10BE50009ACFCF93DF93EB010E946B5E882319F09A
:10BE60000E94D032EB01CE01DF91CF910895CF93A4
:10BE7000DF93EB010E946B5E882321F0DF91CF916D
:10BE80000C94E032CE01DF91CF9108950E94D03220
:10BE900097FD0CC00E94D0326F3F7105810591055E
:10BEA00009F034F40E94D032862F089580E008957E
:10BEB0008FEF08950F931F93CF93DF9383E50E9435
:10BEC0006B5E882349F10E94465F823059F18330CE
:10BED00009F446C0813001F50EE812E0C0E0F80137
:10BEE00081918F010E946B5E882339F00E94465F2A
:10BEF0004FEF682F8C2F0F946D18CF5FC43079F7F8
:10BF000082E40E946B5E882339F00E94465F4FEF07
:10BF1000682F84E00F946D18DF91CF911F910F91DE
:10BF20000C9433C40EE812E0C0E0F80181918F0157
:10BF30000E946B5E882339F00E94465F482F6FEFA6
:10BF40008C2F0F946D18CF5FC43079F782E40E9474
:10BF50006B5E882309F30E94465F482F6FEFD9CFAD
:10BF6000CEE8D2E002E912E089910E946B5E811175
:10BF70000E94465F0C171D07B9F782E40E946B5EB2
:10BF8000882351F20E94465FC7CF8091640590914B
:10BF90006505892B41F00E94465F91E0811101C047
:10BFA00090E0892F089591E0FCCFCF93DF93C82FC5
:10BFB000D62F0E946B5E882321F0DF91CF910C94E5
:10BFC000C55F8C2F0E94B32C811101C08D2FDF9192
:10BFD000CF91089580E00E94CF33E2EBF4E180E05E
:10BFE00090E0A0E8BFE380839183A283B3831482AF
:10BFF0001582168217821086118612861386148681
:10C00000158616861786808B918BA28BB38B148A2C
:10C01000158A168A178A108E118E128E138E148E20
:10C02000158E168E178E80A391A3A2A3B3A3089595
:10C03000282FE82FF0E09091B30B892F90E0B0E02B
:10C04000A0E004C0B695A795979587952A95D2F755
:10C0500080FF14C08091840790918507860F971FF9
:10C060009093850780938407EE0FFF1FE855F84FE4
:10C0700080819181680F791F718360830895CF92C9
:10C08000DF92EF92FF926B017C0183E3C816D1042B
:10C09000E104F10470F082E3C81AD108E108F10864
:10C0A00062E370E080E090E00F9466240E9466C036
:10C0B000ECCFC701B6010F946624FF90EF90DF909C
:10C0C000CF900C9466C080912E04811107C00E940D
:10C0D0008DF9882319F081E080932E040895A7E25A
:10C0E000B4E11C92E6E8F7E0108211961C921182EE
:10C0F0000895CF93C82F80934D090E9447D6CC2333
:10C1000049F024982C9A65E070E080E090E0CF91AF
:10C110000D946624249A2C98CF9108958F929F9223
:10C12000AF92BF92CF92DF92EF92FF920F93CF9395
:10C13000DF931F92CDB7DEB75C017B0149016B0134
:10C14000C40ED51EF501808191810F94C544898369
:10C15000002311F0F7018083BE016F5F7F4FC401A0
:10C160000F949D01F50180819181019691838083D7
:10C17000FFEFEF1AFF0AEC14FD0421F780E00F90A7
:10C18000DF91CF910F91FF90EF90DF90CF90BF9014
:10C19000AF909F908F900895CF93DF93CDB7DEB788
:10C1A00060970FB6F894DEBF0FBECDBF9C01E62F9F
:10C1B000660FFF0BE653FC4CE491E750EC3008F0BF
:10C1C000C4C0F0E08827E851FF498F4F0D9495488F
:10C1D0002061F4604761456122617E617C61496153
:10C1E000A561A361A161806181E0FE0135969AE0BD
:10C1F000DF011D929A95E9F740EB50E05A8349839D
:10C2000041EB50E05C834B8343EB50E058874F8316
:10C2100044EB50E05A87498792E09F87888B80E102
:10C220003497D90101900D928A95E1F7C901609682
:10C230000FB6F894DEBF0FBECDBFDF91CF9108954A
:10C2400080E0D3CF81E08F5F40E950E0F901518376
:10C25000408341E950E05383428342E950E05583F3
:10C26000448348E950E0578346834AE950E05187C8
:10C2700040874CE950E05387428746E950E05587B4
:10C28000448793E096878787D1CF80E0DCCF80E03A
:10C29000DBCF81E08F5F40EA50E0D90111965C93DB
:10C2A0004E9341EA50E013965C934E93129742EA04
:10C2B00050E015965C934E93149748EA50E0179619
:10C2C0005C934E9316974AEA50E019965C934E930E
:10C2D00018974CEA50E01B965C934E931A9746EAE7
:10C2E00050E01D965C934E931C9794E01E969C9391
:10C2F0001E971F968C939ACF80E0CCCF80E0CBCF57
:10C3000081E08F5F40E251E0F9015183408341E2D7
:10C3100051E05383428342E251E05583448348E233
:10C3200051E0578346834AE251E0518740874CE20F
:10C3300051E05387428746E251E05587448795E0B4
:10C34000A1CF80E0DECF80E0DDCF80E1D9011D927A
:10C350008A95E9F76BCF9091C10095FD0CC0909143
:10C36000C00095FF08C08093C6008091C000806423
:10C370008093C000089520910C042F5F2F710FB699
:10C3800007FC27C090910D04921328C09091C00023
:10C3900095FF1EC090910D0440910C04941306C0AB
:10C3A0009091C1009F7D9093C10012C0E92FF0E0F1
:10C3B000E45FFB4F32819F5F9F713093C600909383
:10C3C0000D043091C00030643093C000491741F330
:10C3D000D9CF90910D04921301C0FBCFE0910C04D2
:10C3E000F0E0E45FFB4F828320930C048091C10056
:10C3F00080628093C1000895CF93DF93EC01FE012A
:10C4000084912196882319F00E94AB61F8CFDF91C7
:10C41000CF9108950F931F93CF93DF938B010E94C9
:10C42000FC61E8018991882319F00E94AB61FACF81
:10C43000DF91CF911F910F91089586E595E00C94BF
:10C44000FC614F925F926F927F928F929F92AF9218
:10C45000BF92CF92DF92EF92FF920F931F93CF93F1
:10C46000DF931F92CDB7DEB78091A11682FF1FC167
:10C470008091320B811102C010928006EE24E39469
:10C4800040919D1650919E1660919F167091A01636
:10C490008091991690919A16A0919B16B0919C1636
:10C4A000481759076A077B0708F4E12C10E000E001
:10C4B000AA24A39480E6982E9AE7C92E93E1D92E58
:10C4C00029E6822E8091320B853008F0F0C0E11011
:10C4D000EEC0E0908006E110EAC080916414909173
:10C4E0006514A0916614B091671480939D16909383
:10C4F0009E16A0939F16B093A01641E050E0BE0197
:10C500006F5F7F4F8CE594E10E94D3B70197D9F517
:10C51000898190E0F82E40909D1650909E16609074
:10C520009F167090A0164091991650919A1660919E
:10C530009B1670919C16BB24B39444165506660650
:10C54000770608F4B12C4416550666067706F0F413
:10C55000019609F468C08AE0F81609F46AC02DE073
:10C56000F21609F466C083E2F81619F02AE3F21213
:10C5700079C080917F06811175C023E2F21259C003
:10C58000A092800656C08FEF9FEFC4CF0E9494CE3A
:10C590008CE594E10E948AB780919816882379F1FE
:10C5A000815080939816889DC001112441E061E07C
:10C5B0008453974F0F941E30E091981684E0E89FC3
:10C5C000F0011124E853F74F40815181628173815A
:10C5D00040939D1650939E1660939F167093A016DD
:10C5E0008CE594E10E94A7B50F94902C8091A11640
:10C5F00082FD57C08DE893E10E94FC61BECF0F948D
:10C600007F2C0E94C3DD0E9491DD6D337105810591
:10C61000910520F0D0925009C0924F0910928506E2
:10C620000E94CCE6E3CF0E941D628EE793E10E9458
:10C63000FC6110927F060115110531F40E9466C05D
:10C64000EB2C10E000E03ECF80914E09989E000D4B
:10C65000111D1124F801EF5AF64F108280E00E945C
:10C66000BA2BEECF0F35110508F02CCF8BE3F81263
:10C6700003C0A0927F0626CF80917F06811122CF32
:10C6800080914E09F801989EE00DF11D1124EF5A9A
:10C69000F64FF082E12C0F5F1F4F14CF10927F06F0
:10C6A000CDCF23E2F212FACF10E000E069CF0F9075
:10C6B000DF91CF911F910F91FF90EF90DF90CF907E
:10C6C000BF90AF909F908F907F906F905F904F90B2
:10C6D000089580E595E00C94FC61CF93C82F82E02B
:10C6E000C11184E040E060E00E943BE80E94696381
:10C6F0008EE695E0CC2311F080E995E0CF910C9483
:10C70000FC619091881193FD0FC09091110C9111D3
:10C710000BC040914D1450914E1420916B023091FA
:10C720006C02421753074CF040E0682F8BE00E94E8
:10C730003BE861E080E00C9432EC0E9469638DE597
:10C7400095E00E94FC6180E008958F929F92AF92E5
:10C75000BF92CF92DF92EF92FF920F931F93CF93EE
:10C76000DF9300D000D01F921F92CDB7DEB76C01CF
:10C770005B017A01022F83EE95E00F94B301809163
:10C78000881183FD1CC020E030E0A901F701608121
:10C790007181828193810F94F840882381F01091F8
:10C7A000110C11110CC020914D1430914E14809138
:10C7B0006B0290916C02281739070CF45FC09091BE
:10C7C000C70881E0890F8093C7088091A11682FD78
:10C7D0007AC00E9484DE80E1E3E5F2E0A5E5B4E002
:10C7E00001900D928A95E1F70E9494CE20E030E00E
:10C7F000A901F60160817181828193810F94F840D3
:10C80000882319F18091110C811111C06091491494
:10C8100070914A1480914B1490914C140F94BB4624
:10C8200020916B0230916C026217730774F080E004
:10C8300090E0A0E2B1E489839A83AB83BC83BE011C
:10C840006F5F7F4FC6010E94E43241E061E081E00A
:10C850000E94B6D3811104C0B50182E00E941FF08E
:10C8600020E030E0A901F70160817181828193812C
:10C870000F94F84081112EC011E011C00E9469632D
:10C8800089EF95E00E94FC61002349F01092810736
:10C890000E946E3460E08AEE95E00E947AE6812F75
:10C8A00028960FB6F894DEBF0FBECDBFDF91CF91B3
:10C8B0001F910F91FF90EF90DF90CF90BF90AF90BE
:10C8C0009F908F9008958B7F8093A1169E5F909389
:10C8D000C7087FCF81E00E948163182F811107C0B4
:10C8E000002351F2109281070E946E34C5CF0023BD
:10C8F00029F040E061E083E00E943BE880E090E0C6
:10C90000A0E0B0E489839A83AB83BC8380E090E0AD
:10C91000A0ECB0E48D839E83AF83B887BE016F5FC8
:10C920007F4FCE0105960E94E4328090CC13909008
:10C93000CD13A090CE13B090CF1380E090E0A8EC80
:10C94000B1E48093CC139093CD13A093CE13B09306
:10C95000CF1380E090E0A0E0B1E489839A83AB83B9
:10C96000BC83F70180819181A281B3818D839E83F5
:10C97000AF83B887BE016F5F7F4FCE0105960E94DF
:10C98000E4328092CC139092CD13A092CE13B09249
:10C99000CF13149A64E670E080E090E00E943F605C
:10C9A0007ECFEC010E9476BD0E941D6280E395E07F
:10C9B0000E94FC61209711F4C7E2D5E00E942CE7A9
:10C9C00061E0CE010E947AE60E946E340E947747B1
:10C9D0000E9434460E947B4686E20E94F845809180
:10C9E000890784608860809389070E947747C09197
:10C9F0001915C695C69584E195E10E94B445DC2FD2
:10CA0000DD0F1D2F1C0F0F94332A10924F15C0936A
:10CA1000501583EE93E10E94875210924F15D093E8
:10CA200050158FE095E00E94D94710924F15109352
:10CA3000501582E095E00E94D94788E195E10F9476
:10CA4000A9298111E0CF8EE195E00F94B30189EE21
:10CA500093E030E6019729F0232F2A950000E9F7AB
:10CA6000F9CFF89489EE93E038EE019729F0232F5F
:10CA70002A950000E9F7F9CF0E9476BDA895FECF70
:10CA80007F928F929F92AF92BF92CF92DF92EF925E
:10CA9000FF920F931F93CF93DF931F92CDB7DEB713
:10CAA0007C0159018B016B01C40ED51E0C151D05AF
:10CAB000C9F1F70180809180F80171908F0179822E
:10CAC000C4010F94C544781601F1672DC4010F9479
:10CAD000CD44C4010F94C54499818917B1F00E94D7
:10CAE00069638DE694E00E94FC6181E00F90DF9124
:10CAF000CF911F910F91FF90EF90DF90CF90BF905B
:10CB0000AF909F908F907F900895BE016F5F7F4F91
:10CB1000C5010F949D01F701808191810196918358
:10CB20008083C4CF80E0E2CFCF92DF92EF92FF927A
:10CB30000F931F93CF93DF93CDB7DEB7A0970FB6B8
:10CB4000F894DEBF0FBECDBF61157105810591055B
:10CB500079F100E0C42ED12CF12CE12CA701960133
:10CB60000F94EB4411E0100FE1E0F0E0EC0FFD1F3B
:10CB7000E00FF11D07FDFA956083B901CA01012F8D
:10CB8000611571058105910549F7115010F1E1E03A
:10CB9000F0E0EC0FFD1FE10FF11D17FDFA959081FC
:10CBA00087E39A3008F480E3890F0E94AB61EDCFF0
:10CBB00080E3A0960FB6F894DEBF0FBECDBFDF9125
:10CBC000CF911F910F91FF90EF90DF90CF900C9439
:10CBD000AB61A0960FB6F894DEBF0FBECDBFDF915C
:10CBE000CF911F910F91FF90EF90DF90CF9008951C
:10CBF000CF92DF92EF92FF926A017B010E94FC616B
:10CC00004AE0C701B601FF90EF90DF90CF900C94FF
:10CC10009465CF93DF93EB010E94FC61BE0190E02D
:10CC200080E04AE0DF91CF910C949465CF92DF923F
:10CC3000EF92FF926B017C01F7FE0BC08DE20E9428
:10CC4000AB61F094E094D094C094C11CD11CE11C61
:10CC5000F11C4AE0C701B601FF90EF90DF90CF9042
:10CC60000C949465CF93DF93E091310BF0E0EE5A92
:10CC7000FA4E8081882309F447C082E492E10E9441
:10CC8000FC61C091310B80E6C89FE0011124CF5AAE
:10CC9000D64F88818E3479F480E20E94AB6189910D
:10CCA0000E94AB61899190ED980F9A30C8F38D3254
:10CCB000B9F38B32A9F38FE392E10E94FC6180917A
:10CCC000B0149091B114891B8F706FE070E0681BF5
:10CCD0007109072E000C880B990B0E9416668CE3D5
:10CCE00092E10E94FC618091320B65E070E0681B6C
:10CCF0007109072E000C880B990B0E9416668AE0BA
:10CD0000DF91CF910C94AB61DF91CF910895CF93D8
:10CD1000DF93EB010E94FC61BE01DD0F880B990BD4
:10CD2000DF91CF910C941666CF9384E50E946B5EE1
:10CD3000C0E08823F9F00E94465FC82F1816D4F48B
:10CD40000E9469638DE40E94AB61609195057091CA
:10CD50009605072E000C880B990B0E9416666C2F07
:10CD6000CC0F770B83E099E00E9487668AE00E94EF
:10CD7000AB61CFEF8C2FCF9108958F929F92AF929E
:10CD8000BF92CF92DF92EF92FF92CF936B017C0123
:10CD9000B42E20E030E0A9010F94F84087FF07C0CF
:10CDA0008DE20E94AB61F7FAF094F7F8F094C0E0DE
:10CDB00060E070E080E09FE3CB1541F02DEC3CECAF
:10CDC0004CEC5DE30F945E41CF5FF6CF9B01AC016D
:10CDD000C701B6010F944F456B017C010F94C24609
:10CDE0004B015C014AE00E949465CC2391F1C5019E
:10CDF000B4010F94FD409B01AC01C701B6010F9433
:10CE00004E456B017C018EE20E94AB61C15008F17E
:10CE100020E030E040E251E4C701B6010F945E41EA
:10CE20004B015C010F94BB466B01770FEE08FF08C6
:10CE3000C701B6010E941666C701B6010F94FF40F4
:10CE40009B01AC01C501B4010F944E456B017C01FF
:10CE5000DDCFCF91FF90EF90DF90CF90BF90AF905C
:10CE60009F908F900895CF92DF92EF92FF926A0188
:10CE70007B010E94FC6142E0C701B601FF90EF9088
:10CE8000DF90CF900C94BD668F929F92AF92BF922D
:10CE9000CF92DF92EF92FF920F931F93CF93DF9386
:10CEA00000D01F92CDB7DEB780913F0B10923F0BA1
:10CEB000882309F441C080910B0290910C0218164E
:10CEC00019063CF59A8389839E012D5F3F4F44E00C
:10CED00050E064EB7BE0CE0101960E9440650E9429
:10CEE00069634091B40B5091B50B6091B60B709192
:10CEF000B70B8BEA97E10E94336760910B02709148
:10CF00000C028AE997E10E94876688E997E10E940E
:10CF1000FC610E9423430F900F900F900F90DF91C0
:10CF2000CF911F910F91FF90EF90DF90CF90BF9026
:10CF3000AF909F908F90089581E080933614009178
:10CF4000391410913A140115110509F442C01092D8
:10CF50003A1410923914B801012E000C880B990B69
:10CF60000F94FF402091090C30910A0C40910B0C5A
:10CF700050910C0C0F945E412091B40B3091B50B85
:10CF80004091B60B5091B70B0F944F456B017C014C
:10CF900020E030E040E050EC0F94AF4787FD19C02F
:10CFA00020E030E040EA50E4C701B6010F94F840B9
:10CFB00018167CF0B80182E00E941860C092B40B91
:10CFC000D092B50BE092B60BF092B70B82E0809353
:10CFD0006F0280916F02882309F49DCF84EB9BE060
:10CFE0000E946FE0BC0187E798E10E94B753C090B0
:10CFF000B40BD090B50BE090B60BF090B70B8090CF
:10D00000790790907A07A0907B07B0907C07A501E4
:10D010009401C701B6010F94F8408823E9F020E09D
:10D0200030E0A901C701B6010F94F840882309F444
:10D030007DC0A5019401C701B6010F94F84087FD9A
:10D0400077C081E080937807C0927907D0927A0701
:10D05000E0927B07F0927C0780914C15813198F427
:10D0600080914E15833078F08091780744E0481B1A
:10D070005FE5E52E58E1F52E0CE022E062E488E160
:10D0800095E10F94CD2B80914C15853180F48091E2
:10D090004E15843160F04CE5E42E48E1F42E01E0B9
:10D0A00023E044E16CE388E195E10F94CD2B80917E
:10D0B0004C158F3308F02FCF80914E158F3208F426
:10D0C0002ACF8091780740E3481B82E4E82E88E16C
:10D0D000F82E0DE022E06AE588E195E10F94CD2B72
:10D0E0008091780741E3481B98E2E92E98E1F92EF8
:10D0F00022E065E088E195E10F94CD2B28EFE22E48
:10D1000027E1F22E00E123E04FE262E188E195E1C0
:10D110000F94CD2B38ECE32E37E1F32E23E04FE2D2
:10D1200067E688E195E10F94CD2BF5CE80E08ACFBC
:10D130008FEF88CF2F923F924F925F926F927F92A4
:10D140008F929F92AF92BF92CF92DF92EF92FF9217
:10D150000F931F93CF93DF93CDB7DEB7CB56D10993
:10D160000FB6F894DEBF0FBECDBF70E060E085E47F
:10D170000E94375F182F81E0810F8230E8F082EC47
:10D1800095E1C559DF4F0FB6F894DEBF0FBECDBF96
:10D19000DF91CF911F910F91FF90EF90DF90CF9093
:10D1A000BF90AF909F908F907F906F905F904F90C7
:10D1B0003F902F900C94FC6165E070E083E40E9446
:10D1C000375FB82E60E085E50E94D55F68968FAF27
:10D1D000689740E050E06CE872E417FD04C040E05E
:10D1E00050E066E173E483E50E94785E0F94BB46ED
:10D1F000072E000C880B990B0F94FF406D837E83E4
:10D200008F83AC969FAFAC970F9499246A8B7B8BDE
:10D210008C8B9D8B1F3F09F009C520E030E047E073
:10D2200053E46D817E818F81AC969FADAC970F9456
:10D23000AF4718160CF0D8C187E995E1A2CF612C51
:10D24000712C812C3EE3932E2C966CAE7DAE8EAE6F
:10D250009FAE2C974AE9642E49E9742E49E1842E49
:10D260004FE3942E60966CAE7DAE8EAE9FAE60970F
:10D2700061961FAF61972CE934E163963FAF2EAF03
:10D28000639747ED54E137C2A8A5B9A52C90119634
:10D290003C90119712960C9112971396BC91AB96F5
:10D2A000BFAFAB97BDC26796EEADFFAD679780830A
:10D2B00013C3E4E14E2E512C612C712CF4E1CF2EDE
:10D2C000D12CE12CF12CC1C36796EEADFFAD679771
:10D2D000808395C4D501C4012BAD3CAD4DAD5EAD91
:10D2E000821B930BA40BB50BB7FD65C061968FAD88
:10D2F00061970E94C3EB8AE00E94AB61D501C40133
:10D300008053984FAF4FBF4F8BAF9CAFADAFBEAF09
:10D310009FAD911186C024962CAD3DAD4EAD5FAD55
:10D320002497B101802FAB969FADAB970F94AF4779
:10D3300018160CF05EC0A4966CAD7DAD8EAD9FADA1
:10D34000A4970F94FF409101402FAB965FADAB9730
:10D350000F944F4524966CAF7DAF8EAF9FAF24974F
:10D360002AA93BA94CA95DA9280D391D4A1D5B1DA1
:10D3700028962CAF3DAF4EAF5FAF2897A8966CAD07
:10D380007DAD8EAD9FADA8970F94FF409B01AC0182
:10D390006D817E818F81AC969FADAC970F944E4589
:10D3A0009101402FAB965FADAB970F94F840881F6B
:10D3B0008827881F8FAFD501C401880F991FAA1F26
:10D3C000BB1F4A895B896C897D898AA49BA4ACA414
:10D3D000BDA4480D591D6A1D7B1D841B950BA60B12
:10D3E000B70B81389F44A241B105C8F18EE794E1A3
:10D3F0009DC2D501C40128962CAD3DAD4EAD5FADAB
:10D400002897821B930BA40BB50B65964EAD5FADB1
:10D41000659760E075E1B7FDCECF812F0E945BBEBE
:10D42000CACF20E030E040EA51E46D817E818F81F7
:10D43000AC969FADAC970F944E459B01AC01B101EA
:10D44000802FAB969FADAB970F94F84087FFB3CF7B
:10D4500063964EAD5FAD639767EC74E1DECFAA963D
:10D460008EAC9FACAA97A888B9888A149B040CF04C
:10D47000B8C09501233031050CF4B3C081E294E1CA
:10D480000E94FC611F3F09F090C041E154E15987BF
:10D4900048878FEF93E10E94FC61888599850E94FF
:10D4A000FC6149815A816B817C818DE194E10E940C
:10D4B00033678AE00E94AB618FEF93E10E94FC61C9
:10D4C000888599850E94FC6148A159A16AA17BA128
:10D4D00089E194E10E9433678AE00E94AB618FEF9B
:10D4E00093E10E94FC61888599850E94FC614CA1B2
:10D4F0005DA16EA17FA185E194E10E9433678AE07E
:10D500000E94AB6168966FAC68976620A1F12CEA27
:10D5100035EC47E25EE368A179A18AA19BA10F9453
:10D520005E416B017C012CEA35EC47E25EE36CA1C5
:10D530007DA18EA19FA10F9449461F3FD9F58980F7
:10D540009A80AB80BC808092B9079092BA07A09273
:10D55000BB07B092BC07C092BD07D092BE07E09255
:10D56000BF07F092C0076093C1077093C207809312
:10D57000C3079093C407C559DF4F0FB6F894DEBFB9
:10D580000FBECDBFDF91CF911F910F91FF90EF9014
:10D59000DF90CF90BF90AF909F908F907F906F90D3
:10D5A0005F904F903F902F90089580E194E199878C
:10D5B00088876FCF27E11202F0011124EB5BFB4E4D
:10D5C00069807A808B809C80638674868586968647
:10D5D000C786D08AE18AF28A638B748B858B968B9F
:10D5E000CACF0E94A3F9FDC083E895E10E94FC61C7
:10D5F0000E9476BD87E68093B80742E02CE330E0D6
:10D60000E5E0F0E057E6C52ED12CE12CF12C642E9C
:10D61000712CA6967FAE6EAEA697A8EEB3E00F94DF
:10D620003F456AAB7BAB8CAB9DAB6A887B888C88B3
:10D630009D88660E771E881E991E28966CAE7DAE5C
:10D640008EAE9FAE289781E0809349028EEC90E0E9
:10D65000A0E0B0E01F3F21F08FEF90E0A0E0B0E04D
:10D660009C01AD0124513109410951092FAB38AF5B
:10D6700049AF5AAF3C014D019594879477946794D4
:10D680006C966CAE7DAE8EAE9FAE6C979C01AD017C
:10D690002150310941095109A0962CAF3DAF4EAF41
:10D6A0005FAFA0971F3F09F0CACD5BEA652E5AEA2B
:10D6B000752E872C5EE3952E2C966CAE7DAE8EAECD
:10D6C0009FAE2C976DEC662E6CEC762E6CE4862E5D
:10D6D0006EE3962E60966CAE7DAE8EAE9FAE60977A
:10D6E00061961FAE619723EB34E163963FAF2EAF97
:10D6F00063974DEE54E165965FAF4EAF6597260197
:10D7000037018A899B89AC89BD898AA79BA7ACA769
:10D71000BDA78BAF9CAFADAFBEAF1CA21DA21EA21A
:10D720001FA218A219A21AA21BA219821A821B8276
:10D730001C82188690E49C87ACE1AA8FB6E4BB8F6C
:10D740001C8E1D8E1E8E1F8E1FAE24961CAE1DAE0F
:10D750001EAE1FAE24971EA61FA618AA19AA21E066
:10D760002E8B198A188A212C312C00E0AB961FAE23
:10D77000AB9737E11302C00111248B5B9B4EAC01C8
:10D78000465F5F4F67965FAF4EAF6797DC011496B9
:10D79000B9A7A8A7A6962EAD3FADA697032E000C5D
:10D7A000440B550BA4962CAF3DAF4EAF5FAFA49783
:10D7B000A6964EAD5FADA6974E0F5F1F4F5F5F4FB2
:10D7C000CA01550FAA0BBB0BA8968CAF9DAFAEAF8D
:10D7D000BFAFA8978B2CBB0C9908AA969FAE8EAEB4
:10D7E000AA9780914902882309F4A2C00F94992432
:10D7F0004B015C012091A7072EAB222309F47FC0C7
:10D800000E943FBE1F3F09F03FCD2090B2073090ED
:10D81000B3070091B4073091B507AB963FAFAB9714
:10D820002C8D3D8D4E8D5F8DB101802FAB969FADC0
:10D83000AB970F94AF4718163CF42C8E3D8E0E8F8D
:10D84000AB96EFADAB97EF8F28853C854A8D5B8D0E
:10D85000B101802FAB969FADAB970F94F84087FF37
:10D8600007C028863C860A8FAB96FFADAB97FB8F2F
:10D870002E89222309F477C09101402FAB965FAD2A
:10D88000AB976D817E818F81AC969FADAC970F94E5
:10D89000F84087FF34C0B501A4018AA59BA5ACA5BB
:10D8A000BDA5481B590B6A0B7B0BDB01CA018858CD
:10D8B0009341A109B109B7FD22C0D301C2018C195E
:10D8C0009D09AE09BF09B595A795979587951F3F07
:10D8D00009F0E9CC8093B8074EA75FA768AB79AB96
:10D8E000FD81FC8F2E812D8F3F813E8FAC964FADF9
:10D8F000AC974F8F8A8A9B8AAC8ABD8A1E8A20E0A9
:10D9000030E040EA51E46D817E818F81AC969FAD1D
:10D91000AC970F944F459101402FAB965FADAB97FD
:10D920000F94F84087FFD6CC8FE095E10E94FC6110
:10D93000C559DF4F0FB6F894DEBF0FBECDBFDF91E4
:10D94000CF911F910F91FF90EF90DF90CF90BF90FC
:10D95000AF909F908F907F906F905F904F903F908F
:10D960002F900C9476BD9101402FAB965FADAB9795
:10D970006D817E818F81AC969FADAC970F94AF4740
:10D9800018160CF0BCCFD501C4012A893B894C89FB
:10D990005D89821B930BA40BB50BAC01BD014858EC
:10D9A00053416109710977FDAACF48895989452BEF
:10D9B00009F416C12EA53FA548A959A9280F391F5A
:10D9C0004A1F5B1F2E8B3F8B488F598F2EA53FA57B
:10D9D00048A959A9281B390B4A0B5B0BC701B60193
:10D9E0000F94DB442E893F89488D598D0F940D4546
:10D9F000420E531E641E751E34E143165104610429
:10DA000071040CF456CC8FA998ADA9ADBAAD8415AC
:10DA10009505A605B70514F42C013D016C962CADB7
:10DA20003DAD4EAD5FAD6C977301620124153505B8
:10DA30004605570554F4A096CCACDDACEEACFFAC7B
:10DA4000A097C418D508E608F7088BE795E10E946F
:10DA5000FC61C301B2010E94166686E795E10E944F
:10DA6000FC61C701B6010E94166648855C856A8D17
:10DA70007B8D8FE695E10E9433674C8D5D8D6E8DB9
:10DA80007F8D88E695E10E94336748895989433044
:10DA900051050CF4A5C0C701B6010F94FF4020E06A
:10DAA00030E040E850E40F945E4169837A838B83D1
:10DAB0009C8328853C854A8D5B8D6C8D7D8D8E8DFC
:10DAC0009F8D0F944E452BED3FE049E450E40F94B9
:10DAD0005E4120E030E040E05FE30F945E419B0157
:10DAE000AC0169817A818B819C810F9449466C8756
:10DAF0007D878E879F876E897F89888D998D0F940A
:10DB0000FF402FE632E143E85AE30F945E41688715
:10DB100079878A879B8760962CAD3DAD4EAD5FAD12
:10DB200060976C857D858E859F850F945E416983A6
:10DB30007A838B839C839B01AC01688579858A8578
:10DB40009B850F945E412C962CAD3DAD4EAD5FADE7
:10DB50002C970F945E416CA37DA38EA39FA3298174
:10DB60003A814B815C81CA01B9010F944F452885E8
:10DB700039854A855B850F94494668A379A38AA3B2
:10DB80009BA34C855D856E857F8582E695E10E942D
:10DB90003367488559856A857B858CE595E10E94C8
:10DBA00033678CE495E10E94FC6149815A816B8165
:10DBB0007C8186E495E10E94336748A159A16AA15E
:10DBC0007BA180E495E10E9433674CA15DA16EA129
:10DBD0007FA18AE395E10E9433678AE00E94AB61EE
:10DBE000D701C601840D951DA61DB71DB595A79536
:10DBF000979587951F3F09F067CB8093B8072889D1
:10DC000039892F5F3F4F398B288B3D8138874E8173
:10DC10004C875F815A8FAC968FADAC978B8F8AA65D
:10DC20009BA6ACA6BDA69EA99E8B69CEE12E012E19
:10DC3000000CFF08F70183E0EE0FFF1F8A95E1F764
:10DC4000EF5BFD4F668177816F507109072E000CE5
:10DC5000880B990B0F94FF409B01AC016D817E8175
:10DC60008F81AC969FADAC970F94AF4718160CF40C
:10DC7000E3CA83E895E10E94FC610E9476BD87E1DA
:10DC80008E9DF0018F9DF00D1124EB5BFB4E8FE715
:10DC900082874AE028E230E0EAE0F0E09FE7C92E20
:10DCA000D12CE12CF12CB3CCAF92BF92CF92DF926A
:10DCB000EF92FF920F931F93CF93DF93CEE8D2E0C2
:10DCC0000CEC1BE058016E01FF24F394F6018191E6
:10DCD0006F010E94B32C882389F00E9494CE80911A
:10DCE000640590916505892B09F458C00E942E3374
:10DCF000F5016083718382839383F12CF4E0AF0E8E
:10DD0000B11C21E9C21622E0D20601F786E40E9486
:10DD1000B32C882339F10E9494CE0E942E336B01DC
:10DD20007C0120E030E040E85FE30F94AF47181635
:10DD3000CCF120E030E0A901C701B6010F94F84012
:10DD400087FF03C0C12CD12C760120E030E04FE7E3
:10DD500053E4C701B6010F945E410F94C24660932D
:10DD6000D80BF12C83E50E94B32C882311F10E947B
:10DD700094CE0E942E33609363027093640280936A
:10DD8000650290936602DF91CF911F910F91FF90F2
:10DD9000EF90DF90CF90BF90AF90089560E070E07B
:10DDA000CB01A6CFC12CD12C80E8E82E8FE3F82E32
:10DDB000CCCFFF2041F38FEB98E00E94FC61809173
:10DDC000D80B811104C08CEB98E00E94FC6183EBBE
:10DDD00098E00E94FC618091D80BE4E68E9FC00120
:10DDE000112481589F4F6FEF70E00F94814870E0CD
:10DDF00090E080E00F94FD4020E030E048EC52E4F9
:10DE00000F944946AB01BC018FE898E00E9433674C
:10DE100082E798E00E94FC6180E598E00E94FC6146
:10DE200080E20E94AB6189910E94AB61F80161912F
:10DE30007191819191918F0142E00E94BD668AE0CB
:10DE40000E94AB61F2E0C139DF0751F740916302F4
:10DE50005091640260916502709166028CE298E0D4
:10DE60000E9433678AE0DF91CF911F910F91FF905D
:10DE7000EF90DF90CF90BF90AF900C94AB618DE0AE
:10DE80000E94AB618AE00C94AB61E8E9F5E0808127
:10DE9000818385E492E10E94FC616091DE137091C0
:10DEA000DF138091E0139091E1136F5F7F4F8F4FED
:10DEB0009F4F0E9416660E943F6F0C9432660F932C
:10DEC0001F93CF938C01C62F81E192E10E94FC61E8
:10DED000C8010E94FC618AE30E94AB616C2F70E074
:10DEE00090E080E00E941666CF911F910F910C94F4
:10DEF0003F6FCF93DF93EC018991882319F00E9443
:10DF0000AB61FACFDF91CF910C943F6F8091980570
:10DF1000909199052FEF3FEF981751F0E92FF0E01E
:10DF2000E856FA4F228130E09F5F9F7790939905E2
:10DF3000C9010895CF92DF92EF92FF920F931F9342
:10DF4000CF93DF9300E68091320B853008F02DC12E
:10DF50008091980590919905891B8F7709F425C1C7
:10DF60000E94866FAC0197FDEECF2091DC133091BB
:10DF7000DD138A3019F08D3009F0E4C010927E066E
:10DF80002115310519F40E9466C0DDCF225E394F9C
:10DF9000F90110821092DD131092DC13CEE1D6E06D
:10DFA000FE018191803209F443C08E3409F0B6C07D
:10DFB00065E773E1CE010F9475407C01892B41F038
:10DFC0006EE470E0CE0104960F94E048009709F4E7
:10DFD000CE014AE050E070E060E001960F94F73D1A
:10DFE000AB01BC0140931A0650931B0660931C06BC
:10DFF00070931D068091DE139091DF13A091E013C2
:10E00000B091E1130196A11DB11D481759076A0788
:10E010007B0781F0EF2871F482E493E1DF91CF91E7
:10E020001F910F91FF90EF90DF90CF900D94A1047E
:10E03000EF01B6CF6AE270E0CE010F940F499C0168
:10E04000009701F1982F9C1B10E0992339F0915013
:10E05000FE01E90FF11D80811827F7CF4AE050E05B
:10E0600070E060E0C90101960F94F73DC12ED12CFC
:10E07000F12CE12C6C157D058E059F0531F083E2B6
:10E0800093E1CCCF89EF92E1C9CF80911A069091AC
:10E090001B06A0911C06B0911D068093DE13909381
:10E0A000DF13A093E013B093E11380913302811149
:10E0B0001CC067E470E0CE010F94E0480097A9F01F
:10E0C0004AE050E070E060E001960F94F73D643064
:10E0D00071058105910548F488E592E10E94FC6193
:10E0E00060E08EE492E10E947AE680911E068B3316
:10E0F00009F429CF8091320B853008F024CF80912C
:10E100004E09809FC00111246EE176E08F5A964F30
:10E110000F94EB4881E00E94BA2B15CF8091A11695
:10E1200080FFC3CF61E475E3CE010F947540009783
:10E1300031F0FC01838180538A3008F0B6CF8FEC38
:10E1400092E16CCF2F3531050CF0FDCE8C35C1F44A
:10E150000E94866F97FDF7CE20917E062111F3CEA7
:10E160002091DC133091DD13A9014F5F5F4F509375
:10E17000DD134093DC13225E394FF9018083E3CE37
:10E180008B3321F481E080937E06DDCE80917E0684
:10E190008111D9CEC90101969093DD138093DC13D0
:10E1A000225E394FF9014083CECEDF91CF911F918E
:10E1B0000F91FF90EF90DF90CF9008958F929F92F4
:10E1C000AF92BF92CF92DF92EF92FF920F931F9385
:10E1D000CF93DF93C82F0E94A3F90F9499246B016A
:10E1E0007C01D0910002DD23F1F080917405882339
:10E1F000D1F040912F04509130046091310470911E
:10E20000320497018601041B150B260B370BB9014D
:10E21000A80177FD1AC0833009F465C00CF054C022
:10E2200081300CF059C02D2F30E0A8EEB3E00F94F0
:10E230003F45C60ED71EE81EF91EC0922F04D0928D
:10E240003004E0923104F09232048091320B853038
:10E2500020F40E949A6F0E9421620F9499246B010E
:10E260007C0180916F0590917005A0917105B0912E
:10E2700072050097A105B105D9F14091C5075091EC
:10E28000C6076091C7077091C807840F951FA61F26
:10E29000B71FA7019601281B390B4A0B5B0BDA014C
:10E2A000C901B7FD25C00E941D626091C90B709124
:10E2B000CA0B88EC94E00E940A628AE00E94AB617B
:10E2C00090E080E00E94D164843009F0ACCF0E94DD
:10E2D000696387E894E004C00E94696386EB94E078
:10E2E0000E94FC61A0CF0E9469638FE994E0F8CF9F
:10E2F0008091010290910202A0910302B091040268
:10E300000097A105B10589F03091B0142091B114A6
:10E31000321709F4B3C00F9499246093C507709322
:10E32000C6078093C7079093C8070F9499248090DD
:10E33000370490903804A0903904B0903A049B01BF
:10E34000AC01281939094A095B0949015A01B7FC8E
:10E3500042C04B015C0134EC830E39E0931EA11CDA
:10E36000B11C8092370490923804A0923904B09284
:10E370003A04079B0AC0069B08C0059B06C0209173
:10E38000B807211102C0049908C060933304709348
:10E390003404809335049093360480903304909035
:10E3A0003404A0903504B090360481149104A10483
:10E3B000B10409F497C0681979098A099B09605664
:10E3C0007A4E8109910997FF8DC0749A6FEF70E0C2
:10E3D00082E00F9490238091430490914404A09193
:10E3E0004504B091460497018601081B190B2A0BBE
:10E3F0003B0BD901C801B7FD26C13091B0149091F3
:10E40000B11420916D0280916E0239136EC090910B
:10E410002714299F90011124220F232F221F330B31
:10E420003195D22F90912814899FC0011124880F13
:10E43000892F881F990B9195C82FDD2309F49FC060
:10E440000F94992480903B0490903C04A0903D044C
:10E45000B0903E0481149104A104B10409F071C08C
:10E460006C597F4F8F4F9F4F60933B0470933C04D8
:10E4700080933D0490933E04DFEF69C02091C7086C
:10E4800021112DC0C1112BC04091C5075091C60765
:10E490006091C7077091C807840F951FA61FB71F0B
:10E4A00097018601081B190B2A0B3B0BD901C801E8
:10E4B000B7FD15C080914704811137CF81E080936B
:10E4C0004704179A8091B30B8E7F8093B30B169AF3
:10E4D0008091B30B8D7F8093B30B149A26CF10924B
:10E4E000470423CF749860E072CF4091B11417E5D0
:10E4F000419FA00111244A5E534FFA01EF5AFF4F8A
:10E500009081299F90011124220F232F221F330B6A
:10E510003195D22F4E5A5F4FFA019081899FC001E9
:10E520001124880F892F881F990B9195C82F8091EE
:10E53000B1149091B014981709F47FCF8F5F8F704A
:10E54000F8CF681979098A099B0997FD95CF2D2F76
:10E5500030E050E040E02150310941095109A9EB78
:10E56000B0E00F942C452EEF30E040E050E00F94E7
:10E570000D452A5B3F4F4F4F5F4FB9010AC01092C4
:10E580003B0410923C0410923D0410923E0470E053
:10E5900060E088E00F94FE22CC23D9F10F949924F7
:10E5A00080903F0490904004A0904104B0904204B9
:10E5B00081149104A104B10471F46C597F4F8F4F01
:10E5C0009F4F60933F047093400480934104909365
:10E5D0004204CFEF06C0681979098A099B0997FDA3
:10E5E000F8CF2C2F30E050E040E0215031094109B4
:10E5F0005109A9EBB0E00F942C452EEF30E040E03C
:10E6000050E00F940D452A5B3F4F4F4F5F4FB901CC
:10E610000AC010923F0410924004109241041092DC
:10E62000420470E060E086E00F94FE22F4E6CF0E34
:10E63000D11CE11CF11CC0924304D0924404E0922E
:10E640004504F09246040E9466C08091A107813083
:10E6500009F072C00F9499246B017C0180914C04E5
:10E6600090914D04A0914E04B0914F049701860102
:10E67000081B190B2A0B3B0BD901C801B7FD3AC087
:10E680008090A2079090A307A090A407B090A50740
:10E690000E9491DDAB01BC014093A2075093A307F8
:10E6A0006093A4077093A50780913E0990913F095C
:10E6B000A0914009B091410988199909AA09BB099B
:10E6C000840F951FA61FB71F80933E0990933F09A3
:10E6D000A0934009B0934109D701C601805F984DCE
:10E6E000AF4FBF4F80934C0490934D04A0934E04C2
:10E6F000B0934F048091480490914904A0914A043A
:10E70000B0914B04A7019601281B390B4A0B5B0BF8
:10E71000DA01C901B7FD10C030E8C30E3EEED31ECA
:10E72000E11CF11CC0924804D0924904E0924A04D2
:10E73000F0924B040E94D1CD0E94F1E580916A05D0
:10E740008823C9F10F949924C0906605D09067057D
:10E75000E0906805F09069056C197D098E099F09A4
:10E7600097FD29C00F9499246B017C0120916A05C3
:10E7700030E0A8EEB3E00F943F45C60ED71EE81E6A
:10E78000F91EC0926605D0926705E0926805F09286
:10E79000690580E00E94C3EB8AE0DF91CF911F9171
:10E7A0000F91FF90EF90DF90CF90BF90AF909F9030
:10E7B0008F900C94AB61DF91CF911F910F91FF90DF
:10E7C000EF90DF90CF90BF90AF909F908F90089583
:10E7D0002F923F924F925F926F927F928F929F9271
:10E7E000AF92BF92CF92DF92EF92FF920F931F935F
:10E7F000CF93DF93CDB7DEB763970FB6F894DEBF44
:10E800000FBECDBF8091881183FD54C183E50E9466
:10E810006B5E8887882309F448C10E942E330F94C9
:10E82000BB466C3871050CF05EC17093B7076093FE
:10E83000B6070E94AFA86091B6077091B707072E80
:10E84000000C880B990B0F94FF402091B207309178
:10E85000B3074091B4075091B5070F94AF4718160E
:10E860000CF444C181EE93E160E00E947AE681E01D
:10E87000809349021A821B821C821D8219861A8685
:10E880001B861C8619821E862CE32F873CE1388B61
:10E8900046E4498B312C212C50E85A8B8FEB8B8B23
:10E8A00091E09D87812C912C54016091B607709165
:10E8B000B707072E000C880B990B0F94FF407B01C4
:10E8C0008C01232D322D4A895B890F94F8408823CF
:10E8D000B9F02091B2073091B3074091B40750913D
:10E8E000B507A885B701C801A11103C10F94F8406D
:10E8F000881F8827881F89833E2C2F2C0A8B1B8B0F
:10E900000F9499246B017C01DC01CB0129853A85A8
:10E910004B855C85821B930BA40BB50BB7FD2EC0FA
:10E92000D701C60188519C4FAF4FBF4F89879A8747
:10E93000AB87BC8780E00E94C3EB8DED93E10E9422
:10E94000FC6181149104A104B10409F4FAC0C50169
:10E95000B40168517C4F8F4F9F4F6C197D098E0910
:10E960009F0928EE33E040E050E00F94EB44CA01E9
:10E97000B9010E9416668AE00E94AB6180E00E94A5
:10E98000DE700F9499246093C5077093C607809337
:10E99000C7079093C8079091B2079E83A091B307D1
:10E9A000AF830091B4071091B507292F3A2FA80122
:10E9B000632D722D8A899B890F944E452B013C0152
:10E9C00020E030E0A9010F94AF4787FF04C077FA39
:10E9D000709477F8709420E030E040EA50E4C3018E
:10E9E000B20181149104A104B10409F0AEC00F94E6
:10E9F000F84087FF0BC0BD8546015701BB2331F0AE
:10EA000028EE820E23E0921EA11CB11C3981332313
:10EA1000A9F18A819B81AC81BD81892B8A2B8B2BAB
:10EA200061F0D701C6012A813B814C815D81821B47
:10EA3000930BA40BB50BB7FD21C02E813F81A8011C
:10EA40006E857F85888999890F944E4520E030E056
:10EA500040EC5FE30F94F84087FD4FC0D701C6013B
:10EA6000805A9541AF4FBF4F8A839B83AC83BD8350
:10EA70009E819E87AF81AF87088B198B8091490259
:10EA80008823D9F181149104A104B10461F0B8EE96
:10EA9000CB1AB3E0DB0AE108F108C818D908EA0884
:10EAA000FB08F7FE2AC01D8600CF82E50E946B5E40
:10EAB0008111B3CE63960FB6F894DEBF0FBECDBF03
:10EAC000DF91CF911F910F91FF90EF90DF90CF904A
:10EAD000BF90AF909F908F907F906F905F904F907E
:10EAE0003F902F9008956CE870E09FCE80EF93E107
:10EAF000BBCE0F94F84087FF1EC080914902882347
:10EB0000C9F263960FB6F894DEBF0FBECDBFDF919A
:10EB1000CF911F910F91FF90EF90DF90CF90BF901A
:10EB2000AF909F908F907F906F905F904F903F90AD
:10EB30002F900C94CCE63E2C2F2C0A8B1B8B198229
:10EB4000DFCE8FE30E94AB6116CF0F94AF4718164C
:10EB50000CF05CCF4601570159CFCF93DF93EC0106
:10EB60008881882349F18A3039F18D3029F18B333E
:10EB7000F9F08091320B8530D8F480914E0920E66F
:10EB8000829FC0011124BE018F5A964F0F94EB480B
:10EB900080E00E94BA2B0E946963BE018FE292E17D
:10EBA0000E940A628CE292E1DF91CF910C94FC61A9
:10EBB00080E00E94DE70D4CFDF91CF910895EF9274
:10EBC000FF920F931F93CF93DF9300D000D000D01C
:10EBD0001F921F92CDB7DEB77C0120917D07422F97
:10EBE000022E000C550B80917E078230A1F18330FC
:10EBF00059F184E49BE15F932F939F938F938E0150
:10EC00000F5F1F4F1F930F930F948F40C7010E94F8
:10EC10002BE881E080938B07C8010E94AD751092AC
:10EC20008B070F900F900F900F900F900F902B96D7
:10EC30000FB6F894DEBF0FBECDBFDF91CF911F910D
:10EC40000F91FF90EF90089580E59BE127FDD3CFD2
:10EC50008BE39BE1D0CF89E59BE1CDCFE0917D07B0
:10EC600087E1E802F0011124EB5BFB4E8085918582
:10EC70000C94DF75BF92CF92DF92EF92FF920F93C9
:10EC80001F93CF93DF9381E080937E0710927D07DF
:10EC900061E00E94EE33C091381485E0D82EDC0E7E
:10ECA00081E0D4E0DC1B93E0F92EFC1A92E0E92E1F
:10ECB000EC1AC82ECC1ABC2EB194C11128C08823DE
:10ECC00089F08091370B18166CF02091391430912F
:10ECD0003A142F5F3F4F30933A14209339148F5FCB
:10ECE0008093370B80916F02882349F010E000E099
:10ECF00021E041E062E67BE18B2D0E947951CF5FFC
:10ED000080E0DC12DACF85E08093371423C0C13075
:10ED100059F58091370B813089F080916F028823FB
:10ED200071F381E09091370B913009F080E024E09D
:10ED300048EA5BE16C2D0F94CF1CE1CF80913F0B33
:10ED400010923F0B882349F30E947434809134144D
:10ED5000882319F3DF91CF911F910F91FF90EF90CE
:10ED6000DF90CF90BF900895C23009F069C08091C4
:10ED7000370B823081F080916F02882309F4BFCF76
:10ED800081E09091370B923009F080E020E24DE86D
:10ED90005BE16E2DD0CF80913F0B10923F0B88230B
:10EDA00051F380919D0790919E070E94DF7580919D
:10EDB0003414882301F3CECF8091370B833081F058
:10EDC00080916F02882309F49ACF81E09091370BEC
:10EDD000933009F080E020E241E85BE16F2DABCF9A
:10EDE00080913F0B10923F0B882351F380919F0736
:10EDF0009091A0070E94DF7580913414882301F35D
:10EE0000A9CF80913F0B10923F0B882319F10F94EB
:10EE10005B2060917D0737E16302B0011124635BE1
:10EE20007B4E0EE216E722E231E048E750E082E74F
:10EE30009BE10F946E1E80913414882359F08ACF81
:10EE4000C33009F4B9CFC43009F059CF8091370BE2
:10EE50008430B9F280916F02882309F450CF11E019
:10EE60008091370B843009F010E020917D0737E165
:10EE70002303F0011124EB5BFB4E808591850E94FA
:10EE8000D1E19C0149E95BE16D2F812F0F94091DB0
:10EE900036CF2F923F924F925F926F927F928F92D6
:10EEA0009F92AF92BF92CF92DF92EF92FF920F9319
:10EEB0001F93CF93DF93CDB7DEB7C854D1090FB6F8
:10EEC000F894DEBF0FBECDBF382E0E948F5E82E564
:10EED0000E946B5E882309F44AC10E942E336B01A5
:10EEE0007C0120E030E0A9010F94F840882309F468
:10EEF0002EC1409053025090540260905502709081
:10EF00005602209157023091580240915902509177
:10EF10005A022D8B3E8B4F8B588F8091B80B90915E
:10EF2000B90BA091BA0BB091BB0B8D8F9E8FAF8F99
:10EF3000B8A32091BC0B3091BD0B4091BE0B5091FA
:10EF4000BF0B2DA33EA34FA358A79C01AD01C30146
:10EF5000B2010F94F84081110DC02DA13EA14FA127
:10EF600058A56D897E898F89988D0F94F8408823E4
:10EF700009F4EDC020E030E0A901C701B6010F940B
:10EF8000F840881F8827881F8311E8C080E090E040
:10EF9000A0E8BFE389A79AA7ABA7BCA7A3019201EA
:10EFA0006D8D7E8D8F8D98A10F944E4569A37AA3A8
:10EFB0008BA39CA32D893E894F89588D6DA17EA17D
:10EFC0008FA198A50F944E45698F7A8F8B8F9C8F58
:10EFD00029A13AA14BA15CA1CA01B9010F945E41DC
:10EFE0004B015C01298D3A8D4B8D5C8DCA01B901B5
:10EFF0000F945E419B01AC01C501B4010F944F45D4
:10F000000F94FD474B015C01AC019B0160E070E097
:10F0100080E89FE30F9449466DA77EA78FA798AB22
:10F0200020E030E040E05FE3C501B4010F945E41B1
:10F030004B015C01A7019601C701B6010F945E4127
:10F040006B017C01A5019401C501B4010F945E41DF
:10F050009B01AC01C701B6010F944E450F94FD47CB
:10F0600029A53AA54BA55CA50F945E414B015C0117
:10F07000698D7A8D8B8D9C8D90582DA53EA54FA5C1
:10F0800058A90F945E41A50194010F945E416B0154
:10F090007C012D8D3E8D4F8D58A1C301B2010F947F
:10F0A0004F4520E030E040E05FE30F945E419B017C
:10F0B000AC01C701B6010F944F45A30192010F9413
:10F0C0004E456B017C012DA13EA14FA158A56D8934
:10F0D0007E898F89988D0F944F4520E030E040E085
:10F0E0005FE30F945E412B013C012DA53EA54FA58A
:10F0F00058A969A17AA18BA19CA10F945E41A50199
:10F1000094010F945E419B01AC01C301B2010F94C5
:10F110004F452D893E894F89588D0F944E456D8BF3
:10F120007E8B8F8B988F20E030E0A901C701B6015C
:10F130000F94F8408111E8C020E030E0A9016D890A
:10F140007E898F89988D0F94F8408111DDC00E94CF
:10F150001D6286E192E10E94FC61AEC020E030E0D9
:10F1600040E85FEB29A73AA74BA75CA717CF89E434
:10F170000E946B5EC12CD12C7601882321F00E9465
:10F180002E336B017C018AE40E946B5E882309F4B4
:10F19000ADC00E942E33C3CF20E030E0A901C501ED
:10F1A000B4010F94AF4787FF22C2B7FAB094B7F803
:10F1B000B0941DC2498D5A8DBA0190E080E00F9441
:10F1C000FD4029A13AA14BA15CA10F945E414B01E6
:10F1D0005C010F9444466B017C01C501B4010F949E
:10F1E000EF474B015C01A70196016D8D7E8D8F8DE0
:10F1F00098A10F945E412B013C012D893E894F89D6
:10F20000588DC501B4010F945E41A30192010F9482
:10F210004F452B013C01A50194016D8D7E8D8F8D95
:10F2200098A10F945E414B015C012D893E894F8965
:10F23000588DC701B6010F945E419B01AC01C50119
:10F24000B4010F944E456DA37EA38FA398A759E1F7
:10F2500059A7E0C280E1E8EBFBE0DE0111960190E6
:10F260000D928A95E1F7C12CD12C80E8E82E8FE32E
:10F27000F82E8E010F5E1F4F9E01235F3F4FAE01A0
:10F28000475F5F4FBE016B5F7F4FCE0101960F94CA
:10F29000951780E1FE013196A3E5B2E001900D9251
:10F2A0008A95E1F70F9499246093C5077093C60778
:10F2B0008093C7079093C807C85BDF4F0FB6F894D9
:10F2C000DEBF0FBECDBFDF91CF911F910F91FF9099
:10F2D000EF90DF90CF90BF90AF909F908F907F90F6
:10F2E0006F905F904F903F902F90089520E030E016
:10F2F000A901C701B6010F94F840882309F427CF6C
:10F300001D8A1E8A1F8A188ED701C601B0588D8F9C
:10F310009E8FAF8FB8A32D893E894F89588D505845
:10F320002DA33EA34FA358A7A7019601C701B6017D
:10F330000F945E414B015C012D893E894F89588DA8
:10F34000CA01B9010F945E419B01AC01C501B40132
:10F350000F944F450F94FD4769AF7AAF8BAF9CAFC9
:10F360008091530290915402A0915502B09156029F
:10F3700089A39AA3ABA3BCA39C01AD01C701B601AD
:10F380000F944F456DA77EA78FA798AB209157028A
:10F39000309158024091590250915A0229A73AA738
:10F3A0004BA75CA72D893E894F89588D69A57AA501
:10F3B0008BA59CA50F944F4521966CAF7DAF8EAF6A
:10F3C0009FAF21978091B80B9091B90BA091BA0B88
:10F3D000B091BB0B89AB9AABABABBCAB2DA53EA53B
:10F3E0004FA558A9BC01CD010F944E456B017C017E
:10F3F0002091BC0B3091BD0B4091BE0B5091BF0BC7
:10F400002DAB3EAB4FAB58AF21962CAD3DAD4EADC5
:10F410005FAD21976DA97EA98FA998AD0F944E4538
:10F420004B015C0180915B0290915C02A0915D02B6
:10F43000B0915E0225968CAF9DAFAEAFBFAF259762
:10F440009C01AD016091C00B7091C10B8091C20B0A
:10F450009091C30B0F944E45698F7A8F8B8F9C8F41
:10F46000A70196016D8D7E8D8F8D98A10F945E41C1
:10F470002B013C01A50194016DA17EA18FA198A54E
:10F480000F945E419B01AC01C301B2010F944F4543
:10F490002B013C01A50194016D8D7E8D8F8D98A16E
:10F4A0000F945E414B015C01A70196016DA17EA105
:10F4B0008FA198A50F945E419B01AC01C501B401D9
:10F4C0000F944E45A30192010F94CE456B017C0130
:10F4D00020E030E0A9010F94F84087FF0AC02BED2F
:10F4E0003FE049EC50E4C701B6010F944F456B0172
:10F4F0007C012BED3FE049EC50E4C701B6010F94CD
:10F50000494620E030E040EC51E40F945E410F9416
:10F510002D460F94C2468B01672B11F401E010E0D9
:10F52000332051F02BED3FE049EC50E4C701B60128
:10F530000F944E456B017C0120E030E0A901C7012A
:10F54000B6010F94F840811122C029A93AA94BA90C
:10F550005CA969A17AA18BA19CA10F94F8408111AB
:10F5600016C02DA93EA94FA958AD69A57AA58BA5AE
:10F570009CA50F94F84081110AC008E110E02BED22
:10F58000C22E2FE0D22E29ECE22E20E4F22EA7018B
:10F59000960169AD7AAD8BAD9CAD0F945E414B0188
:10F5A0005C0120E030E0A901698D7A8D8B8D9C8D06
:10F5B0000F94F840882309F4EFCDA5019401C5010B
:10F5C000B4010F945E414B015C01298D3A8D4B8D46
:10F5D0005C8DCA01B9010F945E419B01AC01C5016C
:10F5E000B4010F944F450F94FD474B015C012FE68A
:10F5F00032E143E85AE3C501B4010F94F84087FDB6
:10F6000051CE40905F025090600260906102709015
:10F610006202C501B4010F94F1460F94C2461B016A
:10F620006017710708F41801B10190E080E00F94B1
:10F63000FD404B015C01AC019B01C701B6010F9479
:10F64000494669A37AA38BA39CA3A5019401698D64
:10F650007A8D8B8D9C8D0F94494669AF7AAF8BAFB5
:10F660009CAFA30192016091C40B7091C50B809176
:10F67000C60B9091C70B0F944E45A50194010F94B2
:10F68000494629966CAF7DAF8EAF9FAF299729A1D0
:10F690003AA14BA15CA1CA01B9010F945E4120E0DF
:10F6A00030E040E05FE30F945E419B01AC0160E01D
:10F6B00070E080E89FE30F944E4569AB7AAB8BAB6B
:10F6C0009CAB25962CAD3DAD4EAD5FAD2597298702
:10F6D0003A874B875C874D865E866F86788A609115
:10F6E0000D0270910E02072E000C880B990B0F94DF
:10F6F000FF4020914F0230915002409151025091B1
:10F7000052020F945E412AE037ED43E25CE30F942E
:10F710005E41698B7A8B8B8B9C8B0F9499249B0118
:10F72000AC0128533F4F4F4F5F4F2DAB3EAB4FAB1C
:10F7300058AF4D8C5E8C6F8C78A041E050E05A8FB2
:10F74000498F59E159A7898D9A8D8215930508F043
:10F7500081CD0E9466C00F9499242DA93EA94FA97E
:10F7600058AD621B730B840B950B97FD0FC00F9464
:10F7700099249B01AC0128533F4F4F4F5F4F2DAB56
:10F780003EAB4FAB58AF80E00E94DE7039A53150E0
:10F7900039A7332309F40ECD9201A30169A17AA1FF
:10F7A0008BA19CA10F945E416B017C012DA13EA118
:10F7B0004FA158A569A97AA98BA99CA90F945E416C
:10F7C0009B01AC01C701B6010F944F456B017C0151
:10F7D0009201A30169A97AA98BA99CA90F945E4102
:10F7E0004B015C012DA13EA14FA158A569A17AA1B1
:10F7F0008BA19CA10F945E419B01AC01C501B4019A
:10F800000F944E452B013C01C601D7018DA39EA349
:10F81000AFA3B8A79201A3016DA57EA58FA598A956
:10F820000F944F4569837A838B839C832DA13EA1DE
:10F830004FA158A521966CAD7DAD8EAD9FAD2197A2
:10F840000F944F456D837E838F83988729AD3AADA2
:10F850004BAD5CAD69857A858B859C850F944F4552
:10F8600069877A878B879C8729962CAD3DAD4EADF5
:10F870005FAD29976D857E858F8598890F944F455B
:10F880006D877E878F87988B80910702882321F070
:10F89000CE0101960E9424D3C12CD12C90E8E92EF0
:10F8A0009FE3F92E8E010F5E1F4F9E01235F3F4F96
:10F8B000AE01475F5F4FBE016B5F7F4FCE01019688
:10F8C0000F949517882309F4C5CC898D9A8D0196DC
:10F8D0009A8F898F38CF2F923F924F925F926F927B
:10F8E0007F928F929F92AF92BF92CF92DF92EF92D0
:10F8F000FF920F931F93CF93DF93CDB7DEB7C95F0E
:10F90000D1090FB6F894DEBF0FBECDBF81E00E94D3
:10F91000796041E061E081E00E94B6D3882311F074
:10F92000912C2EC08091CB0B811112C08CE3FE0173
:10F930003196DF011D928A95E9F73090CB0B8AE46E
:10F940000E94B32C982E882351F00E94EA5FE8CFE2
:10F9500060E08FE40E94D55F882341F3E1CF70E03F
:10F9600060E086E50E94375FCF52DF4F998388833E
:10F97000C15DD040059710F184E098E00E94FC61E1
:10F9800080E00E947960892DC750DF4F0FB6F89450
:10F99000DEBF0FBECDBFDF91CF911F910F91FF90C2
:10F9A000EF90DF90CF90BF90AF909F908F907F901F
:10F9B0006F905F904F903F902F90089560E084E4A7
:10F9C0000E94D55FC451DF4F8883CC5ED040CF52B8
:10F9D000DF4F08811981C15DD0400330110504F566
:10F9E00060E084E50E94D55FC351DF4F8883CD5E20
:10F9F000D04062E070E088E50E94375F182F62E037
:10FA000070E089E50E94375F082F80E50E946B5EF9
:10FA100081110DC0812F823071F08BED97E0AECF58
:10FA200011E0C351DF4F1883CD5ED040E2CF0E947A
:10FA3000E032082FF0CF82EB97E0023009F09ECF42
:10FA400040E050E86BEB75E483E50E94785E20E0CF
:10FA500030E040E752E40F94494660934B027093C4
:10FA60004C0280934D0290934E0288E40E94B32C86
:10FA7000882309F4A4C00E942E330F94BB468B0147
:10FA800077FF02C00F5F1F4F1595079511950195E0
:10FA9000110904571F4F5801063F2FEF120724F496
:10FAA00046EFA42EBB24BA946501C60ED71E30E2E1
:10FAB000C31631E0D30624F030E2C32EDD24D39404
:10FAC000073F4FEF140714F407EF1FEF7801E60E1E
:10FAD000F71E53E2E51651E0F5060CF0A3C0B8019D
:10FAE000012E000C880B990B0F94FF40C552DF4F7D
:10FAF000688379838A839B83CB5DD040B5010B2CCF
:10FB0000000C880B990B0F94FF40C152DF4F6883A4
:10FB100079838A839B83CF5DD040C552DF4F288194
:10FB200039814A815B81CB5DD0400E94CF2B8823F5
:10FB300009F47DC0B7010F2C000C880B990B0F94B2
:10FB4000FF402B013C01B6010D2C000C880B990BDA
:10FB50000F94FF40A30192010E94CF2BC551DF4FAC
:10FB60008883CB5ED040882309F461C0CF52DF4F39
:10FB700088819981C15DD040892B91F080E897E020
:10FB80000E94FC61C451DF4F9881CC5ED040992324
:10FB900021F086E797E00E94FC618AE00E94AB6159
:10FBA0000E9494CE80E00E94CF3381E00E9456D61E
:10FBB000882309F43FC0832D0E94CF33E1CE8CE42B
:10FBC0000E946B5E26EFA22EBB24BA94882329F0F4
:10FBD0000E942E330F94BB465B0182E50E946B5E50
:10FBE00090E2C92EDD24D394882329F00E942E337D
:10FBF0000F94BB466B0186E40E946B5E07EF1FEF1C
:10FC0000882329F00E942E330F94BB468B0182E497
:10FC10000E946B5E882331F00E942E330F94BB4606
:10FC20007B015DCF83E2E82EFF24F39458CF86E971
:10FC300097E0A4CE0E9439D460E085E40E94D55FAD
:10FC4000882309F418C3A1E0CD51DF4FA883C35E18
:10FC5000D040C551DF4FE881CB5ED040C952DF4F65
:10FC6000E883C75DD040CB53DF4F19821882C55C53
:10FC7000D0402FEF3FEFCB54DF4F39832883C55B54
:10FC8000D040CD52DF4F188219821A821B82C35D89
:10FC9000D040C354DF4F188219821A821B82CD5B79
:10FCA000D04031E0C353DF4F3883CD5CD04042E0D9
:10FCB000C753DF4F4883C95CD040CF54DF4F188211
:10FCC000C15BD040CA18DB08C601DD0CAA0BBB0B18
:10FCD000C251DF4F88839983AA83BB83CE5ED04015
:10FCE000E01AF10A8701FF0C220B330BCE50DF4FD5
:10FCF000088319832A833B83C25FD0402CE0CB5416
:10FD0000DF4F08811981C55BD040209FC001219F32
:10FD1000900D11248C01095A1A4EC754DF4F1983D4
:10FD20000883C95BD040CB54DF4F88819981C55B84
:10FD3000D0400196880F991F880F991F0DE610E09B
:10FD40000C0F1D1F080F191FC951DF4F198308839E
:10FD5000C75ED0400DE310E00C0F1D1F080F191FE8
:10FD6000CF53DF4F19830883C15CD040CB53DF4FA3
:10FD700028813981C55CD040032E000C440B550B03
:10FD8000CA50DF4F288339834A835B83C65FD040E4
:10FD9000C753DF4F0881C95CD040CF54DF4F188173
:10FDA000C15BD040011709F4C3C2C251DF4F688163
:10FDB00079818A819B81CE5ED0400F94FF406B0198
:10FDC0007C01612F110F770B880B990B0F94FF406B
:10FDD0009B01AC01C701B6010F945E41C152DF4FD8
:10FDE000288139814A815B81CF5DD0400F944F4596
:10FDF0004B015C01CE50DF4F688179818A819B8104
:10FE0000C25FD0400F94FF406B017C01CA50DF4FAE
:10FE1000688179818A819B81C65FD0400F94FF40C1
:10FE20009B01AC01C701B6010F945E41C552DF4F83
:10FE3000288139814A815B81CB5DD0400F944F4549
:10FE40006B017C0120E030E0A901C501B4010F94F1
:10FE5000F84087FF60C260E070E0CB01A50194012B
:10FE60000F944F450F94F146C755DF4F6883798350
:10FE70008A839B83C95AD04020E030E0A901C701A2
:10FE8000B6010F94F84087FF4BC260E070E0CB01F1
:10FE9000A70196010F944F450F94F146C355DF4FCC
:10FEA000688379838A839B83CD5AD040CB54DF4FBC
:10FEB00008811981C55BD0400F5F1F4FCB54DF4FC6
:10FEC00019830883C55BD040CF54DF4F1881C15BD5
:10FED000D040E12FEE0FFF0BCB53DF4F088119818C
:10FEE000C55CD040E00FF11FEE0FFF1F21EA30E0AC
:10FEF0002C0F3D1FE20FF31FCB54DF4F08811981F8
:10FF0000C55BD04011830083CF52DF4F2881C15D94
:10FF1000D040CD51DF4F4881C35ED040BE01635514
:10FF20007F4FCE0187559F4F0F94561AC354DF4F12
:10FF3000688379838A839B83CD5BD0409B01AC012E
:10FF40000F9441488111F1C1C354DF4F2881398199
:10FF50004A815B81CD5BD040CD52DF4F6881798192
:10FF60008A819B81C35DD0400F944F45CD52DF4FB6
:10FF7000688379838A839B83C35DD040C951DF4FF7
:10FF8000A881B981C75ED040C354DF4F2881398131
:10FF90004A815B81CD5BD0402D933D934D935D9322
:10FFA000C951DF4FB983A883C75ED040C755DF4F23
:10FFB000C880D980EA80FB80C95AD040CF53DF4F38
:10FFC000E881F981C15CD040C192D192E192F19275
:10FFD000CF53DF4FF983E883C15CD040C355DF4F77
:10FFE000288039804A805B80CD5AD040248635866F
:10FFF0004686578600E010E020E83FE3048F158F27
:020000021000EC
:10000000268F378FA701960169817A818B819C8128
:100010000F944F4569837A838B839C83A20191015E
:100020006D817E818F8198850F944F456D837E838E
:100030008F839887C354DF4F288139814A815B8140
:10004000CD5BD04069857A858B859C850F944F4523
:1000500069877A878B879C87A7019601C701B601BC
:100060000F945E419B01AC016D857E858F859889DB
:100070000F944F456D877E878F87988BA2019101E2
:10008000C201B1010F945E419B01AC0169897A897B
:100090008B899C890F944F45698B7A8B8B8B9C8BBA
:1000A000C354DF4F288139814A815B81CD5BD040C9
:1000B000CA01B9010F945E419B01AC016D897E8933
:1000C0008F89988D0F944F456D8B7E8B8F8B988F7A
:1000D000A2019101C701B6010F945E419B01AC01E1
:1000E000698D7A8D8B8D9C8D0F944F45698F7A8F9A
:1000F0008B8F9C8FA7019601C354DF4F6881798154
:100100008A819B81CD5BD0400F945E419B01AC0105
:100110006D8D7E8D8F8D98A10F944F456D8F7E8F45
:100120008F8F98A3A2019101C354DF4F6881798119
:100130008A819B81CD5BD0400F945E419B01AC01D5
:1001400069A17AA18BA19CA10F944F4569A37AA3C1
:100150008BA39CA36DA07EA00FA118A520E030E08A
:10016000A901C701B6010F94AF474601570187FFA8
:1001700004C0B7FAB094B7F8B094A5019401B301E4
:10018000C8010F94F84087FF02C034018501C30104
:10019000D8018DA39EA3AFA3B8A769A47AA40BA589
:1001A0001CA520E030E0A901C201B1010F94AF47C6
:1001B0005201410187FF04C0B7FAB094B7F8B09478
:1001C000A5019401B301C8010F94F84087FF02C054
:1001D00034018501C301D80189A79AA7ABA7BCA7A1
:1001E00020E030E040E85FE369AD7AAD8BAD9CADD7
:1001F0000F944F4569AF7AAF8BAF9CAFC754DF4FB9
:10020000E881F981C95BD040C486D586E686F78649
:10021000208A318A428A538AC354DF4F0881198168
:100220002A813B81CD5BD040048B158B268B378B8D
:1002300080E00E94DE70CF54DF4F0881C15BD04068
:10024000C353DF4F1881CD5CD040010FCF54DF4F37
:100250000883C15BD040C754DF4F08811981C95B57
:10026000D040045F1F4FC754DF4F19830883C95B19
:10027000D040312C8DCDB2E0CD51DF4FB883C35E7D
:10028000D040E7CCC354DF4F288139814A815B815C
:10029000CD5BD040CA01B9010F944148811152C0D1
:1002A00081E0C952DF4F1881C75DD0401827C9527D
:1002B000DF4F1883C75DD0401123D1F001E0C35355
:1002C000DF4F0883CD5CD04012E0C753DF4F188367
:1002D000C95CD040CF54DF4F1882C15BD04001E0F1
:1002E00010E0CB53DF4F19830883C55CD04006CDA7
:1002F0000FEFC353DF4F0883CD5CD0401FEFC753D0
:10030000DF4F1883C95CD04001E0CF54DF4F088332
:10031000C15BD040E4CF60E070E080E09FE39ECD21
:1003200060E070E080E09FE3B3CD832D0E94CF3387
:10033000CB53DF4F08811981C55CD04001301105D6
:1003400009F0A0CF80E00E9456D6882349F1832D82
:100350000E94CF3320E030E040EC5FE7C354DF4F32
:10036000288339834A835B83CD5BD0400E9420D4AD
:100370008091CB0B81110E945AD50E94A2ED992445
:100380009394C354DF4F288139814A815B81CD5BCF
:10039000D040CA01B9010F9441488111F1CAC0CAC5
:1003A000C354DF4F288139814A815B81CD5BD040C6
:1003B000CA01B9010F9441488111D8CFC9ACDAAC58
:1003C000EBACFCAC20E030E0A901C701B6010F9412
:1003D000F840882309F404C2A701960169817A8153
:1003E0008B819C810F944946CF54DF4F688379837A
:1003F0008A839B83C15BD04069837A838B839C8390
:10040000A70196016D817E818F8198850F94494661
:10041000CB54DF4F688379838A839B83C55BD0404D
:100420006D837E838F839887A701960169857A857E
:100430008B859C850F944946C754DF4F6883798329
:100440008A839B83C95BD04069877A878B879C8727
:10045000A70196016D857E858F8598890F94494601
:100460004B015C01CF54DF4F288139814A815B8188
:10047000C15BD040CA01B9010F945E419B01AC0140
:10048000C501B4010F944E45CF53DF4F6883798384
:100490008A839B83C15CD0406D877E878F87988BD2
:1004A000A701960169897A898B899C890F944946AD
:1004B0004B015C01CB54DF4F288139814A815B813C
:1004C000C55BD040CA01B9010F945E419B01AC01EC
:1004D000C501B4010F944E45CB53DF4F6883798338
:1004E0008A839B83C55CD040698B7A8B8B8B9C8B7A
:1004F000A70196016D897E898F89988D0F94494651
:100500004B015C01C754DF4F288139814A815B81EF
:10051000C95BD040CA01B9010F945E419B01AC0197
:10052000C501B4010F944E456D8B7E8B8F8B988FD8
:10053000A7019601698D7A8D8B8D9C8D0F9449460C
:100540004B015C01CB54DF4F288139814A815B81AB
:10055000C55BD040CF54DF4F688179818A819B8110
:10056000C15BD0400F945E419B01AC01C501B40159
:100570000F944E454B015C01898E9A8EAB8EBC8EDA
:10058000A701960169A17AA18BA19CA10F9449466C
:100590002B013C01C754DF4F288139814A815B819F
:1005A000C95BD040CB54DF4F688179818A819B81C0
:1005B000C55BD0400F945E419B01AC01C301B20109
:1005C0000F944E45C753DF4F688379838A839B839B
:1005D000C95CD04069A37AA38BA39CA3A701960111
:1005E0006D8D7E8D8F8D98A10F9449466B017C0196
:1005F000C754DF4F288139814A815B81C95BD04074
:10060000CF54DF4F688179818A819B81C15BD04063
:100610000F945E419B01AC01C701B6010F944E459A
:10062000C353DF4F688379838A839B83CD5CD0403B
:100630006D8F7E8F8F8F98A3CB53DF4F28813981A9
:100640004A815B81C55CD040CF53DF4F688179819F
:100650008A819B81C15CD0400F945E416B017C011B
:10066000A5019401C501B4010F945E419B01AC0149
:10067000C701B6010F944E456B017C0120E030E0CC
:10068000A9010F94AF472601370187FF04C077FA0D
:10069000709477F8709429A53AA54BA55CA56DA137
:1006A0007EA18FA198A50F944F452FEF36EE4BED0D
:1006B0005EE20F945E41A30192010F94AF4787FF62
:1006C0008FC0C753DF4F288139814A815B81C95C64
:1006D000D040C501B4010F945E412B013C01C353CE
:1006E000DF4F288139814A815B81CD5CD040CB537B
:1006F000DF4F688179818A819B81C55CD0400F94EE
:100700005E419B01AC01C301B2010F944E45A701AC
:1007100096010F9449462B013C014DA65EA66FA69B
:1007200078AAC353DF4F288139814A815B81CD5C30
:10073000D040C501B4010F945E414B015C01C75329
:10074000DF4F288139814A815B81C95CD040CF531A
:10075000DF4F688179818A819B81C15CD0400F9491
:100760005E419B01AC01C501B4010F944E45A70148
:1007700096010F9449466B017C01C9AADAAAEBAA3B
:10078000FCAAA3019201CF54DF4F688179818A814D
:100790009B81C15BD0400F945E41C754DF4F2881DD
:1007A00039814A815B81C95BD0400F944F454B0131
:1007B0005C01A7019601CB54DF4F688179818A8162
:1007C0009B81C55BD0400F945E419B01AC01C5018C
:1007D000B4010F944F4590586DAB7EAB8FAB98AF83
:1007E0008DA59EA5AFA5B8A9CB54DF4F888399836B
:1007F000AA83BB83C55BD040B058C754DF4F888302
:100800009983AA83BB83C95BD04009A91AA92BA9E4
:100810003CA9CF53DF4F088319832A833B83C15CF4
:10082000D04020E030E040E85EE3CD52DF4F688109
:1008300079818A819B81C35DD0400F945E41CD5206
:10084000DF4F688379838A839B83C35DD040CF5217
:10085000DF4F08811981C15DD040012B09F46BC2C3
:100860002DA93EA94FA958ADC951DF4F288339831F
:100870004A835B83C75ED04040906B1550906C15E7
:1008800060906D1570906E152091771530917815E8
:100890004091791550917A15C301B2010F944E45DC
:1008A000C952DF4F688379838A839B83C75DD040B9
:1008B000C0906715D0906815E0906915F0906A15A2
:1008C00020917315309174154091751550917615DE
:1008D000C701B6010F944E45C552DF4F6883798337
:1008E0008A839B83CB5DD040809063159090641584
:1008F000A0906515B090661520916F153091701518
:100900004091711550917215C501B4010F944E4577
:10091000C152DF4F688379838A839B83CF5DD04048
:1009200080915F1590916015A0916115B09162154D
:10093000CB53DF4F88839983AA83BB83C55CD040A8
:10094000A3019201BC01CD010F944E45CD51DF4F63
:10095000688379838A839B83C35ED04000915B1553
:1009600010915C1520915D1530915E15C753DF4FD6
:10097000088319832A833B83C95CD040A701960171
:10098000C753DF4F688179818A819B81C95CD040E0
:100990000F944E456B017C012091571530915815ED
:1009A0004091591550915A15C353DF4F288339830D
:1009B0004A835B83CD5CD040A5019401C353DF4FD4
:1009C000688179818A819B81CD5CD0400F944E45AE
:1009D0004B015C01C552DF4F288139814A815B811F
:1009E000CB5DD0400F945E412B013C01C152DF4FE3
:1009F000288139814A815B81CF5DD040C701B60132
:100A00000F945E419B01AC01C301B2010F944E45AE
:100A1000CF54DF4F688379838A839B83C15BD04047
:100A2000C152DF4F288139814A815B81CF5DD0403F
:100A3000CD51DF4F688179818A819B81C35ED0402F
:100A40000F945E412B013C01C952DF4F288139814F
:100A50004A815B81C75DD040C501B4010F945E41FE
:100A60009B01AC01C301B2010F944E452B013C0127
:100A7000C952DF4F288139814A815B81C75DD040EF
:100A8000C701B6010F945E416B017C01C552DF4F77
:100A9000288139814A815B81CB5DD040CD51DF4FC8
:100AA000688179818A819B81C35ED0400F945E41C9
:100AB0009B01AC01C701B6010F944E456B017C014F
:100AC00020917B1530917C1540917D1550917E15BC
:100AD0000F945E414B015C0120917F153091801590
:100AE0004091811550918215C301B2010F945E416E
:100AF0009B01AC01C501B4010F944F454B015C0152
:100B0000209183153091841540918515509186155B
:100B1000CF54DF4F688179818A819B81C15BD0404E
:100B20000F945E419B01AC01C501B4010F944F4588
:100B30004B015C01C353DF4F688179818A819B81BE
:100B4000CD5CD0409058A70196010F945E41C353ED
:100B5000DF4F688379838A839B83CD5CD040C75302
:100B6000DF4F288139814A815B81C95CD040C30154
:100B7000B2010F945E419B01AC01C353DF4F68810A
:100B800079818A819B81CD5CD0400F944E45C753BB
:100B9000DF4F688379838A839B83C95CD040CB53C2
:100BA000DF4F288139814A815B81C55CD040CF54B9
:100BB000DF4F688179818A819B81C15BD0400F942E
:100BC0005E419B01AC01C753DF4F688179818A8107
:100BD0009B81C95CD0400F944E459B01AC01C5017F
:100BE000B4010F944F454B015C0120E030E0A901B6
:100BF0000F94AF47181624F0B7FAB094B7F8B09432
:100C0000A7019601C701B6010F945E416B017C01FB
:100C1000A3019201C301B2010F945E419B01AC019B
:100C2000C701B6010F944F456B017C01CF54DF4FD4
:100C3000288139814A815B81C15BD040CA01B901F9
:100C40000F945E419B01AC01C701B6010F944F4563
:100C50000F94FD479B01AC01C501B4010F944946B7
:100C6000AB01BC018FE497E00E9433678AE00E94E9
:100C7000AB6103E913E0D8018D918D01882319F050
:100C80000E94AB61F8CF48E0C754DF4F688179819B
:100C90008A819B81C95BD0400E94BD6609EA13E04E
:100CA000F80181918F01882319F00E94AB61F8CF80
:100CB00048E0CF53DF4F688179818A819B81C15C95
:100CC000D04090580E94BD660EEA13E0D8018D9185
:100CD0008D01882319F00E94AB61F8CFC951DF4F15
:100CE000688179818A819B81C75ED040905848E0B5
:100CF0000E94BD66CF52DF4F08811981C15DD0408F
:100D000003301105ACF003EB13E0D8018D918D0198
:100D1000882319F00E94AB61F8CF48E0CD52DF4F35
:100D2000688179818A819B81C35DD0400E94BD66C4
:100D30008AE00E94AB61C451DF4F0881CC5ED04095
:100D40000111E9C1CB54DF4F288139814A815B8190
:100D5000C55BD040CB56DF4F288339834A835B8302
:100D6000C559D040CF53DF4F88819981AA81BB817B
:100D7000C15CD040C756DF4F88839983AA83BB8369
:100D8000C959D040C12CD12C70E8E72E7FE3F72E53
:100D9000C356DF4FC882D982EA82FB82CD59D04048
:100DA000CE018B569F4F0F942A33C757DF4FC8820F
:100DB000D982EA82FB82C958D040C357DF4F1882DC
:100DC00019821A821B82CD58D040C754DF4F088148
:100DD00019812A813B81C95BD040CF56DF4F088300
:100DE00019832A833B83C159D040CE0187579F4F37
:100DF0000F942A33CB56DF4F288139814A815B819A
:100E0000C559D040CF54DF4F288339834A835B8351
:100E1000C15BD040C357DF4F88819981AA81BB81D4
:100E2000CD58D040CB54DF4F88839983AA83BB83AE
:100E3000C55BD040C756DF4F488059806A807B80B1
:100E4000C959D040C757DF4F088119812A813B819A
:100E5000C958D040C754DF4F088319832A833B8386
:100E6000C95BD040C356DF4F88809980AA80BB8081
:100E7000CD59D040CF56DF4FC880D980EA80FB8063
:100E8000C159D040A7019601C301B2010F945E4140
:100E9000CF53DF4F688379838A839B83C15CD040C3
:100EA000A5019401CB54DF4F688179818A819B81B0
:100EB000C55BD0400F945E419B01AC01CF53DF4F27
:100EC000688179818A819B81C15CD0400F944E45B5
:100ED000C358DF4F688379838A839B83CD57D04083
:100EE000A5019401C754DF4F688179818A819B8174
:100EF000C95BD0400F945E414B015C01A701960194
:100F0000CF54DF4F688179818A819B81C15BD0405A
:100F10000F945E419B01AC01C501B4010F944E4595
:100F2000CF57DF4F688379838A839B83C158D04032
:100F3000CB54DF4F288139814A815B81C55BD0402A
:100F4000CF54DF4F688179818A819B81C15BD0401A
:100F50000F945E416B017C01C754DF4F28813981BA
:100F60004A815B81C95BD040C301B2010F945E41ED
:100F70009B01AC01C701B6010F944E45CB57DF4F23
:100F8000688379838A839B83C558D040CE01835878
:100F90009F4F0F942A33C757DF4F088119812A8149
:100FA0003B81C958D040C357DF4F488059806A8081
:100FB0007B80CD58D040CF56DF4F88809980AA8063
:100FC000BB80C159D040C358DF4F88819981AA8125
:100FD000BB81CD57D040CF54DF4F88839983AA83FC
:100FE000BB83C15BD040CF57DF4F88819981AA81F5
:100FF000BB81C158D040CB54DF4F88839983AA83EB
:10100000BB83C55BD040CB57DF4F88819981AA81D4
:10101000BB81C558D040C754DF4F88839983AA83CA
:10102000BB83C95BD040CB56DF4FC880D980EA80F4
:10103000FB80C559D040C756DF4F488159816A812E
:101040007B81C959D040C356DF4F88819981AA81DD
:10105000BB81CD59D0400093B2141093B3142093A8
:10106000B4143093B5144092B6145092B7146092F1
:10107000B8147092B9148092BA149092BB14A092D2
:10108000BC14B092BD14CF54DF4F088119812A815E
:101090003B81C15BD0400093BE141093BF142093DA
:1010A000C0143093C114CB54DF4F088119812A81B9
:1010B0003B81C55BD0400093C2141093C3142093AE
:1010C000C4143093C514C754DF4F088119812A8195
:1010D0003B81C95BD0400093C6141093C714209382
:1010E000C8143093C914C092CA14D092CB14E092A1
:1010F000CC14F092CD144093CE145093CF1460933F
:10110000D0147093D1148093D2149093D314A093DD
:10111000D414B093D514C351DF4F1881CD5ED040A5
:10112000112309F4D6C18CE896E00E94FC616E019F
:1011300023EAC20ED11CCF54DF4FD982C882C15BD3
:10114000D04002E0C353DF4F0883CD5CD040212C58
:1011500010ECC754DF4F1883C95BD04009E7CF5369
:10116000DF4F0883C15CD04014E4CB53DF4F1883BA
:10117000C55CD040CF54DF4F08811981C15BD0409E
:10118000CB54DF4F19830883C55BD040C753DF4F73
:101190001882C95CD040CB54DF4FA881B981C55BB0
:1011A000D0400D911C917801EE0CFF1CEE0CFF1C41
:1011B000EDE6F0E0EC0FFD1FEE0DFF1D40805180CD
:1011C00062807380CD52DF4F288139814A815B81F3
:1011D000C35DD040C301B2010F944E454B015C0189
:1011E000E1E0F0E0EC0FFD1FEE0DFF1D84AD95ADCD
:1011F000A6ADB7ADC358DF4F88839983AA83BB835D
:10120000CD57D040F8013496EE0FFF1FEE0FFF1FB1
:1012100001E010E00C0F1D1FE00FF11F84AD95AD34
:10122000A6ADB7ADC757DF4F88839983AA83BB8329
:10123000C958D040CB56DF4F188219821A821B82C0
:10124000C559D0409E012B563F4FAE0147575F4FC7
:10125000BE0163587F4F82EB94E10E94CEDACB56F9
:10126000DF4F288139814A815B81C559D040C30154
:10127000B2010F944E457B018C01222DC754DF4FE4
:101280003881C95BD040CF53DF4F4881C15CD0402B
:10129000CB53DF4F5881C55CD0400F94F84087FF97
:1012A00010C02E2CC754DF4FF882C95BD040CF53FB
:1012B000DF4F0883C15CD040CB53DF4F1883C55C40
:1012C000D04020E030E0A901C501B4010F94AF4740
:1012D00087FDF1C089E896E00E94FC6145E0C50108
:1012E000B4010E94BD66CB54DF4F08811981C55BF4
:1012F000D0400C5F1F4FCB54DF4F19830883C55B71
:10130000D040C753DF4F1881C95CD040113009F07D
:10131000CBC08AE00E94AB61CF54DF4F08811981B6
:10132000C15BD04002501109CF54DF4F19830883AD
:10133000C15BD040C353DF4F1881CD5CD04011302A
:1013400009F0ABC08AE00E94AB61CF52DF4F088149
:101350001981C15DD0400430110509F0BAC080E6A2
:1013600096E00E94FC6142E0B42E7601A12CD701E8
:101370008D919C918C01000F111F000F111FE1E056
:10138000F0E0EC0FFD1FE00FF11F44AD55AD66AD71
:1013900077ADC358DF4F488359836A837B83CD572A
:1013A000D040FC013496EE0FFF1FEE0FFF1F21E02F
:1013B00030E02C0F3D1FE20FF31F84AD95ADA6ADBD
:1013C000B7ADC757DF4F88839983AA83BB83C958BA
:1013D000D040CB56DF4F188219821A821B82C55922
:1013E000D0409E012B563F4FAE0147575F4FBE0185
:1013F00063587F4F82EB94E10E94CEDAEDE6F0E095
:10140000EC0FFD1FE00FF11FCB56DF4F2881398114
:101410004A815B81C559D04060817181828193810D
:101420000F944E45222DC754DF4F3881C95BD04001
:10143000CF53DF4F4881C15CD040CB53DF4F588141
:10144000C55CD0400F944E452B013C0120E030E0BC
:10145000A9010F94AF4787FD38C08DE596E00E9443
:10146000FC6145E0C301B2010E94BD6634E0E30EB9
:10147000F11C41E0A41226C08AE00E94AB6152E058
:10148000C51AD10881E0B8121AC08AE00E94AB6187
:101490008EE396E00F94A03B24C001E0C353DF4FDE
:1014A0000883CD5CD04066CE11E0C753DF4F188370
:1014B000C95CD04070CE80E20E94AB610FCFBB24EC
:1014C000B39453CFAA24A39452CF80E20E94AB617D
:1014D000C8CFCF52DF4F08811981C15DD040012BA9
:1014E000B9F6C451DF4F1881CC5ED040111188C0CD
:1014F0008CE0E3E5F2E0DE01A358BF4F01900D92CE
:101500008A95E1F781E08093CB0BCE0183589F4F02
:101510000E9436DCC755DF4F288139814A815B81C3
:10152000C95AD04060915302709154028091550283
:10153000909156020F944E456B017C012DEB37E3E1
:1015400046E855EB0F94AF4787FD4BC02DEB37E3D3
:1015500046E855E3C701B6010F94F84018160CF49D
:1015600040C0C355DF4F288139814A815B81CD5A04
:10157000D040609157027091580280915902909129
:101580005A020F944E456B017C012DEB37E346E880
:1015900055EB0F94AF4787FD24C02DEB37E346E8AA
:1015A00055E3C701B6010F94F8401816D4F0C354A0
:1015B000DF4F288139814A815B81CD5BD0406091CA
:1015C0005B0270915C0280915D0290915E020F94CB
:1015D0004E45CB57DF4F688379838A839B83C558F9
:1015E000D0408CE0FE01E358FF4FA3E5B2E001904C
:1015F0000D928A95E1F7C551DF4F3880CB5ED04020
:101600003092CB0B0C94B6818F929F92AF92BF9287
:10161000CF92DF92EF92FF920F931F93CF93DF93BE
:1016200000D01F92CDB7DEB76C017B018A01B22ECC
:10163000A090321410922E1410922F141092301485
:1016400010923114109232140F94A52420E030E04F
:10165000A901F80160817181828193810F94F84022
:10166000882319F1A11015C08091110C811111C0AE
:101670006091491470914A1480914B1490914C14CC
:101680000F94BB4620916B0230916C026217730776
:1016900064F081E00E948163811197C081E08093B2
:1016A0000602109281070E946E3440E060E088E0FC
:1016B0000E943BE820E030E0A90160916104709154
:1016C000620480916304909164040F94F84087FF52
:1016D0000FC080E090E0A0E2B1E489839A83AB83FD
:1016E000BC83BE016F5F7F4F81E694E00E94E432CD
:1016F00080E090E0A8ECB2E489839A83AB83BC835A
:10170000AE014F5F5F4F69E574E085E594E00E94AC
:1017100019D580E090E0A0EAB0E489839A83AB8396
:10172000BC83BE016F5F7F4F8DE594E00E943BD587
:101730008091610490916204A0916304B09164046B
:1017400080935F0290936002A0936102B093620263
:101750008093C40B9093C50BA093C60BB093C70B9B
:1017600084EC9BE00E94A5CE109281070E946E340B
:101770008AE096E00F94B3018091C708815080936E
:10178000C708882339F00F94902C8091C7088150A6
:101790008093C7088091A107823011F40E944CDE2B
:1017A0000E94CCE60E946E340F900F900F900F9025
:1017B000DF91CF911F910F91FF90EF90DF90CF902D
:1017C000BF90AF909F908F900895AA2029F140E09C
:1017D00061E084E00E943BE80E94696382E196E058
:1017E0000E94FC6161E08B2D0E945B32A090740529
:1017F00083E08093740581E080938D0780918D074D
:10180000882341F060E08B2D0E945B3281E00E94D2
:10181000DE70F4CFA092740540E061E085E00E94A4
:101820003BE820E030E0A901F6016081718182810E
:1018300093810F94F840882371F080E090E0A0EC51
:10184000B0E489839A83AB83BC83BE016F5F7F4F13
:10185000C6010E94E43220E030E0A901F701608176
:101860007181828193810F94F840882351F1809097
:10187000CC139090CD13A090CE13B090CF1380E0F6
:1018800090E0A8ECB1E48093CC139093CD13A09397
:10189000CE13B093CF1380E090E0A0E0B0E4898352
:1018A0009A83AB83BC83BE016F5F7F4FC7010E94E9
:1018B000E4328092CC139092CD13A092CE13B092CA
:1018C000CF13812C912CA12C80E4B82E93E0E92E2B
:1018D00020E030E0A901F80160817181828193816B
:1018E0000F94AF4718167CF440E060E086E00E9459
:1018F0003BE889829A82AB82BC82BE016F5F7F4FD8
:10190000C8010E94E432F0907405E09274051092D0
:101910008D0740E060E087E00E943BE8809180070F
:10192000811104C081E00E94DE70F8CFF09274054E
:10193000813071F2BACE0F931F93CF93DF93D82FDC
:10194000C62F0E946D6361E08C2F0E945B320F9462
:10195000992460527C468B4F9F4F60932E14709356
:101960002F148093301490933114109232141091EC
:10197000740583E08093740581E080938D0701E016
:1019800080918D07882309F447C060E08C2F0E9466
:101990005B32809132148823D9F140E060E08AE024
:1019A0000E943BE80E9469638CEB95E00E94FC6119
:1019B00080918D07882321F081E00E94DE70F8CFAE
:1019C00010922E1410922F14109230141092311481
:1019D000109232140F94A52480E00E9481638D2F11
:1019E0000E946D630F94992460527C468B4F9F4FE9
:1019F00060932E1470932F148093301490933114AD
:101A00001092321400938D0761E08C2F0E945B329C
:101A100081E00E94DE70B4CF10937405DF91CF9106
:101A20001F910F910895CF92DF92EF92FF92CF9383
:101A3000DF93CDB7DEB76C970FB6F894DEBF0FBE5D
:101A4000CDBF8CE40E94B32C882309F4B3C00E945C
:101A50002E336B017C0120E030E0A9010F94AF47E9
:101A600087FF04C0F7FAF094F7F8F094F7FAF094CF
:101A7000F7F8F094C98EDA8EEB8EFC8E80E090E061
:101A8000A8ECB2E489839A83AB83BC8380E090E0C6
:101A9000ABE8B3E48D839E83AF83B88780E090E0AA
:101AA000A0EAB1E489879A87AB87BC8788E50E9462
:101AB0006B5E882351F040E050E0BA0188E50E9457
:101AC000785E69837A838B839C8389E50E946B5E51
:101AD000882351F040E050E0BA0189E50E94785E29
:101AE0006D837E838F8398878AE50E946B5E88234F
:101AF00051F040E050E0BA018AE50E94785E6987C3
:101B00007A878B879C87F090A116F2FAFF24F0F871
:101B100040E061E080E00E943BE880E50E946B5E6F
:101B2000E82E1D861E861F86188A8091C70881119F
:101B300034C02E2DAE01435F5F4FBE016F5F7F4FFC
:101B4000CE0149960E94A563882339F1FF2011F048
:101B5000EE2019F160E080E00E949B8C80E090E034
:101B6000A0E0B0E48D8B9E8BAF8BB88F198A1A8A58
:101B70001B8A1C8A1D861E861F86188A8091C708AC
:101B8000882359F020E0AE014B5E5F4FBE016F5ECF
:101B90007F4FCE010D960E94048B6C960FB6F89481
:101BA000DEBF0FBECDBFDF91CF91FF90EF90DF90F2
:101BB000CF900895C12CD12CE12C80E4F82E56CF83
:101BC0001F920F920FB60F9211240BB60F922F9304
:101BD0008F939F93EF93FF9380910D0420910C04BA
:101BE000821306C08091C1008F7D8093C10012C016
:101BF000E82FF0E0E45FFB4F92818F5F8F7190934D
:101C0000C60080930D049091C00090649093C00032
